:10689E000025327800253478000C2573000C436FE8
:1068AE006465206178656C000C546F6F206D616EAD
:1068BE00790A676F737562000C4E6F740A617661A8
:1068CE00696C61626C65000C4D656D6F7279206646
:1068DE00756C6C000C42617474657279456D7074E0
:1068EE0079000C46756E6374696F6E0A6572726F0D
:1068FE0072000C4E6F2070726F6772616D000C54D7
:10690E0061626C65206572726F72000C4D656D6F01
:10691E007279206572726F72000C0025635965736F
:10692E00004E6F2563004E72203A252E3473000AF6
:10693E00252E32732E252E32732E252E3473004DB6
:10694E00656D6F7279206672656520256C644B00EB
:10695E000A4261726D616E4C20003132384B62001A
:10696E003531324B6200313032344B62000A2573BE
:10697E00000A4261726C61732025632E25630050FC
:10698E0072696E74203F004D6573736167652028D0
:10699E002563256329002573002A2A2A2A2A2A001C
:1069AE00245356594A4D504144472B2C2554575A7F
:1069BE004B4E514245482D3B3A55582A4C4F524367
:1069CE0046492F3FAE80A66FCD3EFBC641862603BD
:1069DE00CC8062AE80A677CD3EFBC641862603CC28
:1069EE008062AE80A67FCD3EFBAE80A68ECD3EFBF6
:1069FE00C641862603CC804AAE80A696CD3EFBAE1F
:106A0E0080A699CD3EFBC641862703CC801EAE8064
:106A1E00A6A1CD3EFBAE80A6B0CD3EFBAE80A6BA03
:106A2E00CD3EFBCC801EAE80A6BDCD3EFB5343417A
:106A3E004E2020011F070041910100011F07004158
:106A4E008A01001FFF020080690500806E01580058
:106A5E000001011F070041844B00000108011F07C0
:106A6E000041858E001FFF032C44004D00592A68FB
:106A7E003A6D3A73113F090040000001002C0001ED
:106A8E00040001054C5443204F5320312E3020007A
:106A9E0000000107170000FF689EFF689E0000407F
:0A6AAE0007010000FF689EFF689ECC
:10E1ED00410C5E00410C5600410E9E00410D920007
:04E1FD00410C5C0075
:107855007A68799F7BFF901B03122A2A7B0122FFFE
:10786500E43EFE900D8EE0FAA3E02FF582EA3EF5A8
:1078750083EDF0901D32E0FEA3E0FF900D8EE0FC5D
:10788500A3E02FF582EC3EF58322901B520229F3EB
:10789500FD901D32E03400FC900D8EE0FAA3E02D42
:1078A500F582EA3CF583227A6979297BFF901AD320
:1078B500747FF0227A1B7971901B06022A2AE490C4
:1078C5000D83F0900D7F7480F0A3E4F022900C38C6
:1078D5007414F0900C40227BFF7A69792F901AD3AB
:1078E500747EF02278367C1C7A6A799E7F0D7D0144
:1078F5007BFF7E0002260DE92408F9E43AFA22E02E
:10790500FEA3E0900D79FFE0FCA3E0FD22F0900CD2
:10791500507401F0227B01901AD3022A2A901B96FB
:10792500E02497F582E4341BF58322F07BFF7A6926
:10793500792722900C3CE4F0900C50F022900C5EDC
:107945007401F0E4900C56F022900C46E475F001B9
:1079550002279FE0FF900D8EE0FCA3E0FDF5828CF1
:107965008322E0FF8D828C8375F009EE1229E7A34F
:1079750022900E9FE0FF901D98E0C39FD394302284
:10798500900C3CE0900D91F022900C38740FF0E4CF
:10799500900C40F07F0722EFF0901D2D0229F39007
:1079A5000C38E0640F221227F7900C6C022999908D
:1079B5000D84E0FEA3E0FFC322F0900C55745FF048
:1079C50022F07B017A1A79B222900D88E00475F0D5
:1079D50009A4FF222FFFEC3EF0A3EF22E0FEA3E077
:1079E500FFF5828E8322900C59E0FF900D8DE022E9
:1079F500900C627401F022900D837401F0227BFFDC
:107A05007A6A799222900C6C022981E4900D83F0B8
:057A1500900C38F02286
:10F6F800E4FF740F2FF8E4F60FEFB401F5E4FFEF21
:0EF70800C394005009742A2FF8E4F60F80F124
:01F7160022D0
:10B77E00127913EF24FB606514607114607B24FC56
:10B78E00606A240A600302B83B7F0112A2889019F6
:10B79E006EE0900C3CF0900C4EE0FF700302B83E51
:10B7AE00900C3CE0B42003743AF0900C3CE0B42EC4
:10B7BE0003743BF0900C3CE0FEEF75F00CA4247289
:10B7CE00F582E43469F583E5822EF582E43583F55E
:10B7DE0083E493900C3CF0E4900C4E800A7F0112AF
:10B7EE00A288900C3C74881279BE80447F0112A20C
:10B7FE0088900C3C7487F080377F0112A288E49009
:10B80E000D91F0900D8BE0700F74FF1279C6128FB0
:10B81E005F900C5CE0FF8010E4900D8BF07BFF7A64
:10B82E0068799E128F5F7F0412DE7380031279385F
:04B83E0012798522D4
:10E50500EF24FB602014602A24FE600E0470311293
:10E515007913900C3C742BF08026127913900C3CE7
:10E52500742DF0801B900D83E06015900C3C748970
:10E53500800B900D83E06008900C3C748A12791270
:0CE545001279857F0112A2881279BF2292
:10BFDA00EF24FE602114602E14604624FB6057246F
:10BFEA0008600302C074900C4EE0B40102801E90F7
:10BFFA000C4E74018022900C4EE0B40202800E9026
:10C00A000C4E74028012900C4EE0B40306E41279CE
:10C01A00BE8057900C4E7403F0900C55745EF080FD
:10C02A0049900C67E0700474FF8004E4900C67F098
:10C03A00FF125DC58034900C4FE0B40119900D9148
:10C04A00E0B42E1D12F9FF4018E4900C4FF012FDD7
:10C05A002812D488800B12F9FF5006900C487401FC
:10C06A00F0127913900C3C7481F07F0112A288E4DB
:05C07A00900D91F02281
:06FDED00901E2AEFF02237
:10FA44007F0112A288127985E4900D83F0900C3C1A
:06FA5400748E12791222EB
:0DFC6D00900C73E0FFE4FBFA7D4902BA73CE
:0652EB00901B52122A2A5A
:1052F100122633645360030255F112788F90000136
:1053010012264C24CF603324F870030255EB240994
:1053110060030255F190000212264C642B600302D7
:1053210055F1901B551278CB900C5EF0900C560401
:10533100F0900C68740AF00255F1900C56E070037D
:10534100FEFF2212C749EF4E7003FEFF2212788F33
:10535100E92402F9E43AFAC003C002C00112785507
:105361007A1B79591278BDD001D002D003124CF3C7
:1053710012788FE92404F9E43AFAC003C002C001AB
:105381007A6879A31278597A1B795B1278BDD001BA
:10539100D002D003124CF3901B5DE0FEA3E0901B02
:1053A1005B12790BB50707ECB506030255F1D3ED96
:1053B10094FFEC94414003025543ED8CF0122AEE28
:1053C100544029F353FD3EF254183EF95462410111
:1053D100546F4111547D4121548B413154994141C4
:1053E10054A7415154B5416B54C3419454D541EE36
:1053F10054F741F3551D41FF000055F112788F120A
:1054010078FCC003C002C0017BFF7A6879A31278DF
:105411005B7A0D7984801912788F1278FCC003C0F1
:1054210002C0017BFF7A6879A312785B7A0D7979E2
:105431001278BDD001D002D003124CF30255F11203
:10544100788F1278FCC003C002C00112785512781F
:10545100B9D001D002D0031255F6900C68F0025574
:10546100F112788F7D1012CA2EE4FFFE806012784F
:105471008F7D1012CA2E7F107E00805212788F7D90
:105481001012CA2E7F207E00804412788F7D101268
:10549100CA2E7F307E00803612788F7D1012CA2E80
:1054A1007F407E00802812788F7D1012CA2E7F5097
:1054B1007E00801A12788F7D0612CA2E7F6A7E00C6
:1054C100800C12788F7D1112CA2E7F937E0012C438
:1054D100430255F112788F1278FCC003C002C0015B
:1054E1001278551278B9D001D002D0031255F69036
:1054F1000D9BF00255F112788F1278FCC003C002A7
:10550100C0011278551278B9D001D002D003124CE3
:10551100F3901B72E09007B1F00255F112788F12EF
:1055210078FCC003C002C0011278551278B9D001CD
:10553100D002D003124CF3901B72E0900D88F00260
:1055410055F17F05125BE4EFF46004E4FEFF229065
:105551001B5974FF75F0FD12279F901B6FE4F0A398
:105561007408F0901B59E07002A3E0606E12788F0E
:10557100901B6FE0FEA3E029F9EA3EFAC003C002E6
:10558100C0011278557A1B79571278BDD001D0022B
:10559100D003124CF3901B55E0FEA3E0FFBEFF0EBB
:1055A100BFFF0B1278D2746A127947FEFF22901B5B
:1055B10058E0FF901B55E475F0011227B585F08284
:1055C100F583EFF0901B5974FFF5F012279F901BA4
:1055D1006FE475F00212279F025564901B5BE0FF98
:1055E100A3E0A3CFF0A3EFF0800612794212DDB55C
:0455F1007E007F01B8
:0955F50022124CF3901B72E0221B
:10C1C800E4901E2BF0900C4BE0FEA3E0FF900C7166
:10C1D800E0B50618A3E0B50713900C53E0FF900DE7
:10C1E8009AE0B5070712E87AE4FEFF22900D9AE07C
:10C1F800FF125BE4901E2BE02491F582E43406F5EF
:10C2080083E4F0900C71E0FFA3E0900D89CFF0A3D8
:10C21800EFF0900C711279E1E0FD901E2BE0FC0428
:10C22800F074912CF582E43406F583EDF0BEFF1628
:10C23800BFFF13900D9AE004F0E0FF125BE4900C4E
:10C24800711278CB8006900C71127951901E2BE0F8
:0FC258002490F582E43406F583E070B6FE7F0192
:01C2670022B4
:10FB4000900D89E0FFA3E0900C71CFF0A3EFF012CD
:03FB5000C1C82207
:06A86600901D2D122A2AAC
:10A86C00900D88E0FF700302A94A900E9EE0B50798
:10A87C0002E4F0900C59E0FF125BE4900E9EE07540
:10A88C00F009A4FF901D32E5F0F0A3EF127877E009
:10A89C00FDEF2406127864A3E0FDEF240712786420
:10A8AC00A3A3E0FDEF2408FFE43EFE900D8EE0FA3A
:10A8BC00A3E02FF582EA3EF583ED12799D12263343
:10A8CC00FF901D33E0240312789512799C900001BF
:10A8DC0012264CFF901D33E0240412789512799CBB
:10A8EC0090000212264CFFF4901D33600AE0240500
:10A8FC00127895EFF08010E02405FF901D32E034C3
:10A90C0000FE127880E4F0901D32E0FCA3E0FD9094
:10A91C000D8EE0FAA3E0FB1278A4E0FEEB1278A413
:10A92C00A3E07C002400FFEC3E900C46F0A3EF1259
:10A93C007877A3A3E0900D8DF07E007F0122127832
:07A94C00D27469F0E4FEFF84
:01A9530022E1
:10AEAE00900D8DE0FF125BE47B017A1579B412C030
:10AEBE007FEF700302AF6F64037035900D8E1279C1
:10AECE00B7900C47E09F900C46E09E40081279EB3D
:10AEDE00B507028058900C461279E1E4F0BEFF0BE4
:10AEEE00BFFF0812AF741278CB80BD12794E80B8B6
:10AEFE007B017A1579B412FADB9016B4EFF0E49078
:10AF0E0016B3F09016B4E0FF9016B3E0FDC39F5059
:10AF1E0097900D8EE0FEA3E0FF900C46E0FAA3E0C2
:10AF2E00FBC39FEA9E40101279EBB5070A1278D246
:10AF3E00746AF0E4FEFF2274B42DF582E43415F544
:10AF4E0083E08B828A83F0BAFF0BBBFF0812AF74CB
:10AF5E001278CB800312794E9016B3E004F002AF54
:05AF6E00117E007F01CF
:10AF730022900D8DE004F0E0FF125BE4900C46227A
:10D65900900E9EE004F0900C46E0FEA3E0FFFD90E2
:10D669001E02EEF0A3EDF0900D88E0FD900E9EE015
:10D67900B50516900C44EEF0A3EFF0900D8DE090F7
:10D689000C51F012CE0A12E87A900C59E0FF125BA5
:10D69900E4901E02127958C083C082900E9EE0FE6B
:10D6A900D082D08375F0091229E7EFF0901E03129A
:10D6B9007967EFF0900D8D127967A3EFF07E007F07
:01D6C900015F
:01D6CA00223D
:09FD3C00E4900E9EF0FE7F01220E
:10C6160012F6F8781D7C1D7AFD79AC7F081278F346
:10C626001288827F23125BE4EF70157F13125BE49E
:10C63600EF900C6170057407F0800B7413F08006A0
:10C64600900C617423F012E7A27BFF7A6979D2908D
:10C656001D36122A2A901D341278CB7F05125BE410
:10C66600901D34E0FEA3E0AA06F8AC027D01A312F9
:10C6760029F37E017F5412260D900D841278CB90FB
:10C686000D797481F0A37460F01279429007B104B9
:10C69600F0900D9B7407F0E4900D88F012DDB51252
:0AC6A600F97312E46B7F0702DCF366
:10F655007A0C797412791A7BFF7A6879A71237E2E6
:10F66500900C6BE070057F5F12A486E4900C4EF061
:01F675002272
:10F88D0012F9FF5007E4900C38F08006900C387494
:0AF89D000FF012C3A77F0602DCF390
:0EFC430012FD281278E91299017F0602DCF307
:0BFCDE00900D7D7401F07F0602DCF346
:10D48800900C4FE07059900401E07053900C62E0EA
:10D49800FF6401600AEF7031900D8CE0B4452A906A
:10D4A8000C5AE07024900C62F0900D95F012C3A70E
:10D4B800900C3F7401F0900C3D7449F0900D8CF085
:10D4C8001278C3900C38F080261279F512F0F71212
:10D4D800E46B12798E12DCF37F0612DCF380109075
:10D4E8000401E0B401097D147C007F0612CF9EE49C
:05D4F800900D91F022EF
:10C90A00900C4FE07006900401E06008900C5DE026
:10C91A006401707812FC7A900C62E0FF6401600A8C
:10C92A00EF702D900D8CE0B44926900C5AE07020DF
:10C93A00900C62F012C3A71278C3900C3F04F090D7
:10C94A000C3D7445F0900D8CF0E4900C38F0803C6E
:10C95A001279F5900D95F07F667E0012D572E94A3C
:10C96A004B60217F677E0012D57212263360151242
:10C97A00C3A7900D837409F07F0812A288E4900C73
:10C98A0038F0800312DED27F0612DCF3E490040151
:02C99A00F02289
:10F58400900D8BE0B4FF1B901AB6E0FF900D92E053
:10F594006F600F1279A4600A900D92EF1279C6126F
:03F5A4008F5F2254
:06FDF30012FD2802F7E8F2
:0CFCAE00901DD8EFF0A3EDF0A3EBF022C6
:10F29600901E2CEFF0900D8BE0B4FF0D1279A46058
:10F2A60008901E2CE0FF12DE73901E2CE0900C5C82
:0BF2B600F0B40306900D7E7401F022FE
:10F71700900D8BE0B4FF0A1279A46005E4FF12DEB6
:0FF7270073E4900C5CF0900D7EF0900D90F0224A
:1058FE00900C38E0122AC8591E00596405599E0FA3
:10590E0059BB145A60195A7F1E5B6A2300005BCD87
:10591E00900D90E06401603C900D83E06003025BAB
:10592E00C7900C5EE064017024900E9EE0FF900D17
:10593E0088E0B50711125BCE642A900C38600474AF
:10594E0019F022025A7B1278D27469F0221278D2A0
:10595E007468F0228033900C48E0B40103025BC4FB
:10596E00900D90E064016021900C5AE06401601289
:10597E00900C4FE0B4010312FC5F7F05125BE40252
:10598E00A7711278D274C9F0221278D274CAF0229A
:10599E0012F9BA7F667E0012D572E94A4B6009127F
:1059AE005BD960047FFF8002E4FF02F457900C4045
:1059BE00E0122AC859E10159E90259F1035A1E674A
:1059CE005A26685A2E695A366A59F9C95A01CA00B6
:1059DE00005A3F7BFF7A6879AB80537BFF7A6879F8
:1059EE00B6804B7BFF7A6879C680437BFF7A6879F5
:1059FE00D5803B7BFF7A6879E21237E212FD28E40C
:105A0E00FF125DC57F3C7E0012FD6912F98B80216D
:105A1E007BFF7A6879F080167BFF7A697900800EB9
:105A2E007BFF7A69790C80067BFF7A6979191237C8
:105A3E00E27F0A12A288E4900C4FF012F9FF4003A5
:105A4E0012D48812798E12DCF37D147C007F06024C
:105A5E00CF9E900D95E0B401111291ECEF64014EC2
:105A6E006003025BCD900D95F022900C387405F01A
:105A7E0022900C3CE0FFB48E08E4900C38F0025BF0
:105A8E0066EFB42E10125BCE642A6009900C387447
:105A9E0023F0025B66900C48E0B4010312DED29054
:105AAE000C3CE0FFB42B06900D83E014F0EFB42D08
:105ABE0006900D83E004F0900D83E0FF900D96E0CC
:105ACE006F60061279311237E2900D83E0900D96D9
:105ADE00F0E4FDFF12A183900D83E0122AC85B143F
:105AEE00005B19015B2E025B38035B3D045B4205D4
:105AFE005B4A085B4C095B510A5B590B5B5B0C5BA9
:105B0E00590D00005B661279FC804D125BD9600561
:105B1E0012A9548043900D837402F012E2908038E3
:105B2E0012E290E4900E9FF0802E12D0A7802912E0
:105B3E00E7EA8024900D837404F0801C800512EC3B
:105B4E00958015900D837409F0800D800512E19AF1
:105B5E008006900D83740CF012793822900D95E02A
:105B6E007057900D78E0640170301279311237E27F
:105B7E007F407E0012D57212CF197D03E4FF12A171
:105B8E00831278AC1237E27D037F0D12A183127857
:105B9E00DC1237E2E4900D78F022900C3CE0B489F0
:105BAE000E900D957401F07F0712A28812DED2902E
:105BBE000C3CE0B48A0902DED2900C38741EF0223E
:105BCE007F6A7E0012D572122633227F677E001204
:065BDE00D57212263322ED
:10F1B400900C4FE07027900401E07021900C40E027
:10F1C400701B127A0312FADBC374109FFF7D0312C3
:0EF1D400A183127A031237E27F0712DD542264
:0100120022CB
:01001A0022C3
:10E7A20012F7E812FD28E4900C3BF07EFC7F6D121C
:10E7B200DB6A900C73EFF012F8A712FDF912FD0A52
:10E7C200900C517405F0900C441278CB900D88F0A7
:10E7D20012CE0A1279F5E4900D88F0900C68740A52
:08E7E200F0900D8B74FFF02292
:10C3A700900C68E075F014A4FFAEF012FD6912F965
:10C3B7008BE4900C67F012FDF9900D8BE0B4FF133E
:10C3C7001279A4600E1279C7128F5F900C5CE0FFA0
:10C3D70012DE737F667E0012D572E94A4B60117FC9
:10C3E700677E0012D57212263360057FFF12F4575D
:10C3F700900C5F7401F0900C66F0900C54F0900C68
:10C4070070F0900C60F0900D99F0E4900C5DF09056
:10C417000C4D04F0900D78F0E4900C48F0900D83EB
:10C4270004F0900D9612793B900C40F0900E9FF01F
:0CC4370012FD281278E912990102F7E8C2
:10E87A00900C44E0FEA3E0FF900C4BEEF0A3EFF007
:10E88A00900D9CEEF0A3EFF0900C71EEF0A3EFF078
:10E89A00900D89EEF0A3EFF0900C51E0900D9AF0F4
:10E8AA00900C52F0900C53F0900D74122981127949
:07E8BA00AEE4900C5AF022BD
:10CE0A00900C44E0FFA3E0901E04CFF0A3EFF09053
:10CE1A000C51E0FF900C61E0C39FFFE49400FEE434
:10CE2A00FCFDFB7A80F9F8122805EF249BFFEE340B
:10CE3A00FFFEE43DFDE43CFCC004C005C006C0079B
:10CE4A00901E04E0FEA3E0FFE4F8F9AA06AB07D0BF
:10CE5A0007D006D005D0041279AB900D88E0602186
:10CE6A00127A0AC004C005C006C0071279CEAEF015
:10CE7A00E4F8AA06AB07D007D006D005D004127989
:0ACE8A00AB127A0A900D7402299988
:10EE2A00900C517405F0900D97127904900C4412CD
:10EE3A0079D9F01279B4ED9FFFEC9EFEE4B5071084
:10EE4A00EEB4800C900C517406F0900C441278CBFE
:06EE5A0012CE0A02E87A64
:10BD3900900C61E0900C59F0900D7BE0FFA3E0902E
:10BD49000D8ECFF0A3EFF01279CEC3E49FFFE495F7
:10BD5900F0900D8E8FF012279F900D84127904C3F5
:10BD69009FEC9EC39480900C4150157405F0900D82
:10BD790097E0FEA3E0FFED900D811279D9F08009DB
:10BD89007406F0900D811278CB900D81E0FEA3E04E
:10BD9900FF900C69EEF0A3EFF0900D86EEF0A3EFA3
:10BDA900F0900C41E0A3F0900C43F0901E06EEF0E9
:10BDB900A3EFF0900C59E0FF125BE4901E06127994
:10BDC90058EFF0901E07E08D828C83A3F0900C4110
:08BDD900E08D828C83A3A3F02E
:01BDE100223F
:10DDB5001279B4E49F900D98F074809E900D97F0C1
:10DDC500900D7B74FFF0A3749BF0E4900E9EF09091
:10DDD5000D88E0600512BD39800312EE2A900D848E
:10DDE500E0B48318A3E0B41213900C49E4F0A374D3
:10DDF5000CF0900D93E4F0A37424F022900C49E408
:0FDE0500F0A37410F0900D93E4F0A37440F0229A
:06C74900901CCE122A2A0A
:10C74F00E92402F9E43AFAC003C002C00112785595
:10C75F007A1C79D21278BDD001D002D003124CF3DB
:10C76F00901CD3E0901CD6F0901CD17404F0901C58
:10C77F00D2E07002A3E06046901CCE1229F3901C09
:10C78F00D1E07E0029F9EE3AFAC003C002C00112CF
:10C79F0078557A1C79D41278BDD001D002D003120B
:10C7AF004CF3901CD5E0FFA3E02FF0901CD274FF48
:10C7BF00F5F012279F901CD1E02402F080B0901C5E
:0FC7CF00D6E024E9F46004E4FEFF227E007F013F
:01C7DE002238
:0BCA2E00901B92122A2A901B95EDF03D
:10CA3900E4A3F0901B95E0FFA3E0FEC39F5043EEF3
:10CA490075F002A42408FFE435F0FE901B92122928
:10CA5900F3E92FF9EA3EFAC003C002C00112785582
:10CA69007A1B79A81278BDD001D002D003124CF3F9
:10CA7900901BA9E0FF127922EFF0901B96E004F0D9
:10CA890080B1901B95E0B41120E4A3F0901B96E0CF
:10CA9900FFC39411501374972F127928E0645C60D6
:10CAA90008901B96E004F080E3127922E4F07B0100
:04CAB9007A1B7997D4
:01CABD002256
:10E29000E4FFFE12D57212CF1912F6337D02E4FFAD
:10E2A00012A18312000EE92403F9E43AFA12791C50
:10E2B0007BFF7A6979341237E212E5517A0479FDED
:10E2C00012791A7A057900901AD6122A2A7A0579D3
:10E2D00003901AD9122A2A7BFF7A69793D0237E224
:10D0A700E4FB7A04F9F8127A0A122890901AD3123C
:10D0B70029997BFF7A69794D1237E27BFF7A697983
:10D0C7005E1237E2900C61E024ED601024F06014EA
:10D0D700241C70197BFF7A697968800E7BFF7A6957
:10D0E700796E80067BFF7A6979741237E2127A03C8
:10D0F70012791C7A69797B1237E212000E900007C9
:10D1070012264CFFC00712000E90000812264C9002
:10D117001AD4F0901AD3D0E0F07BFF7A69797F02B6
:02D1270037E2ED
:10E7EA007BFF7A69798D1237E27D03E4FF12A183F8
:10E7FA001278AC1237E27D037F0D12A1831278DC06
:10E80A001237E2900C3CE0B4890E900C3B74011272
:10E81A0079301237E2127A10900C3CE0B48A031273
:08E82A00DED2E4900C50F02254
:10EC95007F307E0012D57212CF197D03E4FF12A1D9
:10ECA500831278AC1237E27D037F0D12A1831278AF
:10ECB500DC1237E2900C3CE0FFB489031279FCEFDB
:0CECC500B48A03127A10E4900C50F02284
:10A95400E4901D97F07F67FE12D572901D99122A1C
:10A964002A7A6979951278B0A314F01237E2901D0F
:10A97400991229F312FADB901D98EFF0900C3CE049
:10A98400648A702412797650147F667E0012D57220
:10A99400E94A4B6008900D83740CF0800B127976B1
:10A9A4004006900E9FE004F0900C3CE0B4891390B4
:10A9B4000E9FE0D394004005E014F080057F06125A
:10A9C400A288901D977401F0901D97E0FFC3940432
:10A9D4005066900E9FE0FD901D98E0C39DFDE494A9
:10A9E40000FCEF1475F010A4FFC3ED9FE5F0648044
:10A9F400F8EC6480984039901D97E0FDE4FF12A1C3
:10AA0400837F677E0012D572901D97E01475F01055
:10AA1400A4FF900E9FE07C002FFFEC35F0FEE92FA1
:10AA2400F9EA3EFA12791C7BFF7A6979A41237E2BB
:0DAA3400901D97E004F08090E4900C50F02D
:01AA410022F2
:10E19A007F207E0012D57212CF197D03E4FF12A1EF
:10E1AA00831278AC1237E27D037F0D12A1831278B5
:10E1BA00DC1237E2900C3CE0B48918E4FF12F45701
:10E1CA007B007A0079007F667E0012C443900D833B
:10E1DA007402F0900C3CE0B48A031279FCE4900CCF
:03E1EA0050F022D0
:1091EC00900C4DE0640170441279311237E2E49036
:1091FC000C4DF0789E7C0D7D017BFF7A6979A7126E
:10920C002D92E4900E9DF0900C50F0900C74F07F29
:10921C0050FE12D57278747C0C7D01122D927B015C
:10922C007A0C797412FADB900D73EFF0900C50E01D
:10923C006401600302931D900C48E0B4010612DE39
:10924C00D202931D900C3CE0FF648E6005EF6488A5
:10925C007052E4900C50F0900C3C04F0900C4DF0DB
:10926C007F6A7E0012D572C003C002C0017F6A7E85
:10927C000012D57212FADB901D2BEEF0A3EFF07BEF
:10928C00017A0D799E901D28122A2AD001D002D085
:10929C000312DB03EF7004FE7F01227F0212A2880F
:1092AC00E4FEFF22900C3CE064877024900E9DE05D
:1092BC00605514F0E0249EF582E4340DF583742A95
:1092CC00F0900D73E0141279301237E2803E803743
:1092DC00900E9DE0C39406502E900D73E0FF04F0A9
:1092EC0074742FF582E4340CF583742AF0900C3CE2
:1092FC00E0FF900E9DE0FE04F0749E2EF582E434A7
:10930C000DF583EFF080057F0612A288E4900C50D7
:10931C00F0900D73E02474F582E4340CF583E4F0E2
:03932C0012D88ACA
:01932F00221B
:10F127000C000D003031323334353637383941422F
:10F13700434445464748494A4B4C4D4E4F50515220
:0FF14700535455565758595A2D2E20242F2B25E7
:1044BC00E0FF04F0901B32E0FCA3E02FF582E43C1B
:1044CC00F583E0FF901B2EE475F0011227B585F003
:1044DC0082F583222F24F7F582E4340AF583E0FF7A
:1044EC009009F7E0FE04F074F82EF582E43408F538
:1044FC0083227B017A1B7991901C64022A2AF58312
:10450C00E0FDEFFBEEC39BFFE49400FE74AC2FF5D3
:10451C008274133EF583EDF09014ADE004F022901C
:10452C001BAAE0FFA3E0900D7FCFF0A3EF22901C1D
:10453C000FE475F00102279F901C0FE0FEA3E0FF33
:10454C00F5828E83E022E0FF900C3AE0FE04F074DA
:10455C00F72EF582E4340AF583229009F7E0FF90F8
:10456C001BB0E02FFFE433CF2401CF3400FED3EF98
:10457C0094EBEE64809480229014ABE0FFFDA3E0FA
:10458C002DFDE433FCA3D3E0FE9DEC6480F8748035
:10459C009822EEF0A3EFF0901BB2E0FFA3E0FD2217
:1045AC00901BAEE0FFA3E0FD22E01475F009A4FF20
:1045BC00900D8FE02FFF900D8EE035F0FE9008F6F9
:1045CC00F0A3EFF022F583E0FF9013A8E0FCA3E04A
:1045DC002EF582E43CF58322540F2430FE901D45C9
:1045EC001229F3EE1226CE901D451229F302263322
:1045FC00901B30E0FEA3E0FF901BB0E022F0901B7C
:10460C00BCE0FEA3E022901BBBE0FF901B39E02234
:10461C00EFF0901DA0E004F022E0FF900D73E0FE9F
:10462C0004F074742EF582E4340CF58322900C396A
:10463C007401F022E0FFA3E0901C0DCFF0A3EFF08B
:10464C0078147C1C7D017B0122901C0F74FFF5F00B
:10465C0002279F901BBCE0C4F854F0C8A3E0C454DC
:10466C000F4822901C0F7480F0A3E4F022F0901BF2
:10467C00BCE0C4540F22D3901BB0E0FF901B36E07B
:10468C009F229013AAE0FF9014ADE0FEC39F2290EE
:10469C001D73E0FEA3E0AA06F922E0FFA3E0CF9091
:1046AC001C0BF0A3EFF022901BB0E0FF901DA0E0DC
:1046BC00C39F2224FEFEE0347F901C0FF0A3CEF0AB
:1046CC00901C15E014F022901BBCE0C41322901C2B
:1046DC0009E0FEA3E0FF901C0FE0221227F7901BCD
:1046EC003A022999901B30E0FEA3E0F5828E8322DA
:1046FC00E0FEA3E0FFD39401EE9480227FFF901B99
:10470C003A12298DD3022930EFF0901B30E475F06A
:10471C00010227B574742EF582E4341BF5832290C4
:10472C001BB6E0FFA3E0FD2274E42FF582E434080D
:10473C00F58322EF2CF582E43EF583E0FD22EFF0C9
:10474C00900D88E0FEEFD39E22F07BFF7AF1792763
:10475C00227C002FFFEC3ECF2400CF3480F0A3EF5F
:10476C00F022901BAFE0FF900C3AE022901C14E07A
:10477C00FFA322900C397402F022901C0FE0FEA3D0
:10478C00E022EEF0A3EFF0901BB0E022F583EDF009
:10479C00900EA2E004F022EF24FEFFEE34FFF0A313
:1047AC00EFF022EE9F9014ACFFE0FEEFC39E229040
:1047BC001E08E0FFD3941022901E08E0FFC3940162
:1047CC0022900C39F0901BADE022901C09E0FCA368
:1047DC00E0FD22A804A905AA06AB07229014ABE0C1
:1047EC009014ADF022901BBCE0C31322E0FDEFC38C
:1047FC009DFDE4940022901BB4E0FD900EA2E0FC21
:10480C00C39D22E0FFA3E0901C09CFF0A3EFF022A0
:10481C00E0FFA3E0900D9CCFF0A3EFF022E0FFA30C
:10482C00E0900C69CFF0A3EFF022E0FFC374FF9F80
:10483C00FF74FF9400FE22901B36E004F0229009D6
:10484C00F7E02FFFE433227D017BFF02260D900C55
:10485C0058E0FF900C57E02FFF22F582E43412F55C
:10486C008322FD901D4C1229F3ED0226CE901C08DC
:10487C00E0FF901C11E06F227A0C7951FE7F03024D
:10488C00260D900C4BF0A3EFF022901B31E02FFF84
:10489C00901B30E022EEF0A3EFF0E422900C5F745A
:1048AC0001F0900C3D22E4900C74F0900D73F0220A
:1048BC00901E087401F022901E087410F022F0E48F
:1048CC009013A0F022FFE0FCA3E0FD22EEF0A3EF9A
:1048DC00F0901BB4E022901B367401F022900C5B1C
:1048EC00E0FD9014ADE0227B017A0A79F722E0FF1B
:0848FC00901C8DE0FEC39F2219
:10F3BB001289F3901DB0122A2A12FADB901DB3EFBB
:10F3CB0012467930E00312F8A7901DB01229F39082
:07F3DB001DB3E0FD02A38B4E
:10667E00E4901DDDF0900C5FE06401600302674B57
:10668E0012F7E81245AC12F9A3901DDB1248A19047
:10669E000AF7F0900C3AF012F8A7E4900C5FF09025
:1066AE000D7DF09008E204F0E4900BF6F09008E314
:1066BE00F09008E1F012E908901BB5E0FF127D6F33
:1066CE00901BB6E0FF127D6F901BB7E0FF127D6F3F
:1066DE00900D94E024FFFF900D93E034FFFE901B8D
:1066EE00B0E0FDD39FEE124597400C900D94E0FF65
:1066FE00ED9F14901DDDF0901BB0E0FF901DDDE0CE
:10670E00FEC39F5013901DDB1245D8124625EFF0A5
:10671E00901DDDE004F080DF900D73E024741246CE
:10672E0031E4F012D88A9008E3E0701178277C1CCF
:10673E007A6A79ABFE7F0D124853128573900C5016
:10674E00E0640160030268819008E2E0B401079002
:10675E000C3CE0B48E079008E3E0B4010B900BF60E
:10676E007401F0E49008E2F0900BF6E064017061C1
:10677E0012F7E8900C3CE0FF648E6004EFB48808DA
:10678E001248A8744BF08041EFB48719900C3AE090
:10679E006033900D73E014F0900C3AE014124755EC
:1067AE001237E28020900C3AE0D394E65012900C0F
:1067BE003C124625EFF0900C3C124552EFF080054E
:1067CE007F0612A28812452BF0E4900C50F002685E
:1067DE0085900D7DE0700612452B0268799010B2FF
:1067EE00E0644560030268747F0112A288901BB8B2
:1067FE00E0B401091247561237E21248B2E4901D76
:10680E00DDF09010B3E0FF901DDDE0C39F5033E04C
:10681E00FF24B5F582E43410F583E0FE900D73E0AD
:10682E00FD04F074742D124631EEF074B52FF5821E
:10683E00E43410F583124552EFF0901DDDE004F0C4
:10684E0080C012F7E81248A87452F0E4900C50F091
:10685E009010F6E0FF12ADD712467A30E0191247CB
:10686E00561237E280119008E27401F07F0612DDB5
:10687E0054800412452BF0900C3AE024F712455E3A
:10688E00E4F0900D73E02474124631E4F002D88ADD
:106AB800E4901B73F07B017A1B7974901B8E122A69
:106AC8002AE4901B91F012E551901BADE0FF901B5A
:106AD80091E0FE2474124723EFF0124720E070067D
:106AE800124720742EF0901B91E004124609780298
:106AF800CEC313CE13D8F930E0091244FE901BAE72
:106B0800126C6412460A7803CEC313CE13D8F93038
:106B1800E0091244FE901BAF126C6412465F30E02D
:106B2800091244FE901BB0126C7312460A7805CE07
:106B3800C313CE13D8F930E0091244FE901BB112EA
:106B48006C7312460A7806CEC313CE13D8F930E018
:106B5800091244FE901BB2126C8212460A7807CEC4
:106B6800C313CE13D8F930E0091244FE901BB312B8
:106B78006C82901BBCE030E0091244FE901BB412FA
:106B88006C911247F130E0091244FE901BB5126C6B
:106B980091901BBCE01313543F30E0091244FE905F
:106BA8001BB6126CA0901BBCE0131313541F30E0EB
:106BB800091244FE901BB7126CA012467A30E00905
:106BC8001244FE901BB8126CAF1246D3540730E043
:106BD800091244FE901BB9126CAF1246D31354032A
:106BE80020E04E901B91E0FF12484AFED3EF94E656
:106BF800EE648094805036E4FF901B91E0FEEFC372
:106C08009E501A74742F124723E0FE9009F7E0FD96
:106C180004F074F82D1244F6EEF00F80DC9009F7BA
:106C2800E024F81244F6E4F0900C39F022124639C8
:106C380022901BBAE0FFA3E0FD12F9A3901B91E09C
:106C4800F582758300AA06A907A801AC027D017B1D
:0B6C5800017A1B79747E00FF12260DEC
:106C630022E0901C67F0901B8E1229F312C99C221C
:106C7300E0901C67F0901B8E1229F312C99C22E04E
:106C8300901C67F0901B8E1229F312C99C22E0908E
:106C93001C67F0901B8E1229F312C99C22E0901CF2
:106CA30067F0901B8E1229F312C99C22E0901C6797
:0B6CB300F0901B8E1229F312C99C22E6
:10B1FE00E4901DDEF0900C4BE0FFA3E0901DDFCF3E
:10B20E00F0A3EFF0900C53E0FF900C52F0125BE4C1
:10B21E00901DDEE0FF04F074F82F1244F6E0FF906C
:10B22E001DDFE0FAA3E0FBF5828A83EFF0900C6C51
:10B23E00122981EF24FFFFEE34FFFEED34FFFDEC0B
:10B24E0034FFFC900C6C122999BAFF16BBFF1390B9
:10B25E000C52E004F0E0FF125BE4901DDF12467228
:10B26E008006901DDF12453D901DDEE024F7F5822D
:10B27E00E43408F583E0709812FD0A900D9BE0FF10
:10B28E0012A2887FFF12FC07901DDFE0FFA3E0CF24
:10B29E0012488E900C52E0A3F0E47FFFFEFDFC906E
:10B2AE000C6C12298DC31229305006900C5A740161
:0EB2BE00F0900D7EE0B40106900D907401F04A
:01B2CC00225F
:10DED20012F8A712F0F712FD0A12FDF9E4900AF700
:10DEE200F0900D7F124672900D7B74FFF0A3749B2D
:10DEF200F012FB9912FBB9E4900401F0900C3BF094
:10DF0200900C4FF0900C62E07017900C3FF0900D67
:10DF12008CE0B4450312C90A900D8CE0B4490D801F
:0DDF22000812F9FF500302F4A412D4882263
:10A28800EF122AC8A2BA01A2C002A2C803A2D0042F
:10A29800A2D805A2E006A2E907A2F808A30709A325
:10A2A800250AA35514A35915A35D16A36117000029
:10A2B800A3667B017D0F80047B017DC87F01801E22
:10A2C8007B017D0F7F0880167B017DC87F08800E8B
:10A2D8007B017D0F7F1080067B017DC87F1002E621
:10A2E800331248BC1247BB507512A37304F080F4B4
:10A2F8001248C31247C4406612A37314F080F412C4
:10A3080048BC1247BB500712A36704F080F41248F8
:10A31800C31247C4404812A36714F080F4E4901EA7
:10A3280009F01248BC1247BB500712A37F04F08003
:10A33800F41248C31247C4400712A37F14F080F4F4
:10A34800901E09E004F0E0C3940540D622E4FF80A3
:0EA358000A7F0180067F0280027F03125CA054
:10A36600227B017D0512E633901E08E0227B017DEB
:10A376000C12E633901E08E0227B017D0512E633BF
:05A38600901E08E0221A
:107BCA0012465F20E003027C55901BAEE0FEA3E064
:107BDA007C002400FFEC3EFEEF8EF0122AEE7C08B9
:107BEA0041827C0D41837C1C41847C1741857C2128
:107BFA0041877C26418A7C12419100007C2E900CA0
:107C0A0039801C900C3A8017900C3B8012900C3CE7
:107C1A00800D900C3D8008900C3E8003900C3FE054
:107C2A00900EA0F0901BB0E0FF900EA0E0FEB5070A
:107C3A0006E4A3F0027D18EEC39F900EA1500674CD
:107C4A0001F0027D187402F0027D18901BAEE06408
:107C5A0040704BA3E0900EA2F0900C3AE0FF900E19
:107C6A00A2E0F9C39F5020E0FF24F712455EE0FE30
:107C7A00901BAF1247F8FC74A32DF582740E3CF5E5
:107C8A0083EE12479B80D2901BAFE0FFE9C39FFFB0
:107C9A00E49400FE74A32FF582740E3E80281245E8
:107CAA00AC12F9A3E4900EA2F01248025010124747
:107CBA003F74A32CF582E4340E12479880EB74A328
:107CCA002CF582E4340EF583E4F01245A312F9A3ED
:107CDA00E4900EA2F0124802501012473F74A22CF0
:107CEA00F582E4340F12479880EB74A22CF582E4F3
:107CFA00340FF583E4F07B017A0F79A2901D5312B9
:107D0A002A2A7A0E79A3129594900EA1EFF0900D7B
:107D1A007F1246F3A3A3A3E024DC602D24FD6010A8
:107D2A0024FD601724047033900EA1E0602D8013A7
:107D3A00900EA1E07025900D7F801A900EA1E0644C
:107D4A00016018900D7FE4800C900EA1E06402603F
:107D5A000A900D7FE475F00312279F900D7FE4755A
:057D6A00F00502279F57
:10EFCF00900C66E0B40113E4900C50F0900C6612B4
:10EFDF0047551237E212D88A8013900C50E0B401D3
:10EFEF000C900C667401F0E4900C50F02212452B3B
:02EFFF00F022FE
:106CBE00E4900C39F0901BBCE020E003026DD19003
:106CCE001BB0E0F97074A3124771FDC39FFFE494EB
:106CDE0000FE9009F7E07A002FFFEA3ECF24021261
:106CEE0045764003026EBC901BB8E0FF600512446F
:106CFE00ECEFF0901BB1E0C39D4006900C3AE060C3
:106D0E0033E4901DA0F0901BB1E0FFFD900C3AE033
:106D1E001247FBCD2401CD3400FC901DA0C31245BB
:106D2E00935011EE2F24F6F582E4340A1244E81241
:106D3E00461C80D2026EB0026EBC9009F7E0FFE9ED
:106D4E0012456F507B901BB8E0FF60051244ECEFCC
:106D5E00F0900C3AE0FF6065901BAFE0FEC3EF9E33
:106D6E00A31247B44021E4901DA0F0901BB0E0FFA9
:106D7E00901DA0E0FEC39F5044901BAFE0FFEE12AB
:106D8E0044E012461C80E4E4901DA0F012476EC34E
:106D9E009FFE901DA0E0FDC39E5009ED1244E0122F
:106DAE00461C80E81246B350149009F7E0FF04F039
:106DBE0074F82F1244F6742012461D80E7026EB04E
:106DCE00026EBC1245AC12F9A3901D9CEEF0A3EF1F
:106DDE001246097805CEC313CE13D8F920E02F1230
:106DEE0045665027901BB8E0FF60051244ECEFF0AB
:106DFE00E4901DA0F01246B3500E901D9C1244D389
:106E0E001244EA12461C80ED026EB0026EBC1245B0
:106E1E00A312F9A312F774EF24FFFFE434FF901DC1
:106E2E009C8FF012279F1247F130E04D12472B1224
:106E3E00F9A3901D9EEEF0A3EFF012F77412484ADC
:106E4E001245795031901BB8E0FF60051244ECEF0B
:106E5E00F0E4901DA0F0901D9EE0FEA3E0FF12F75F
:106E6E00741246B8500E901D9C1244D31244EA126E
:106E7E00461C80E2802C026EBC1245665030901B80
:106E8E00B8E0FF60051244ECEFF0E4901DA0F012A4
:106E9E0046B3500E901D9C1244D31244EA12461C67
:106EAE0080ED9009F7E024F81244F6E4F022124641
:016EBE00399A
:016EBF0022B0
:10F8A7001247561237E2900C55745FF0E4900C6BD8
:0AF8B700F07F5F12A4861248B2220F
:10EE9600E4FF1247CD7003A3E0FF900C4BE0FCA308
:10EEA600E0FD900C44E0B50411A3E0B5050C900C10
:10EEB60053E0FE900C51E06E6007AD07E4FF024F91
:04EEC600C4124639F3
:01EECA002225
:10CE9400E4901E0BF0900C391246097803CEC313AC
:10CEA400CE13D8F930E00A901BAFE0901E0AF08050
:10CEB4001D1245A312F9A312F774901E0A12474AD1
:10CEC4005006901E0AE07006900C397404F0900C21
:10CED40039E07040901BADE0702712460A7802CE0C
:10CEE400C313CE13D8F930E00A901BAEE0901E0BAA
:10CEF400F0800E12472B12F9A312F774901E0BEF59
:10CF0400F0901E0A1245B512C7DF901E0BE0FD7F9C
:04CF140001124FC4F3
:01CF180022F6
:084FC400901C07EFF0A3EDF0D3
:104FCC00E4901C11F0901C13F0EF7018900C44122C
:104FDC00480F900D9C1246A6900C4B1246407A0C32
:104FEC0079638016900D8112480F900C691246A6B9
:104FFC00900D861246407A0C79417E007F03122672
:10500C000D901BADE01470030251A61470030252F4
:10501C003024827003025230248060030252549078
:10502C001C15E0FF125BE4901C08E0D39480500345
:10503C00025136901C117480F0901C0B1246FC40EF
:10504C0008901C0F1247A3800F901C0CE0901C0BB7
:10505C001246BFE0FF125BE4900C39E06003025093
:10506C00EA1248796078901C09E0FEA3E0FFD39027
:10507C001C10E09F901C0FE09E500A124778E0B580
:10508C00070312477F12454460261247D6EFB50539
:10509C000BEEB50407124778E06F6014124786B424
:1050AC000009EEB480051252CB80DA12465580D539
:1050BC00901C11E004F01246DAB5060CA3E0B5071B
:1050CC0007124778E06F6090124786B4000AEEB47E
:1050DC0080061252CB025064124655025064900C5A
:1050EC0039E060030252541246DAB5061BA3E0B550
:1050FC000716901C14E0FDA3E0B5050CEE1246ABB0
:10510C00901C15EDF0025254124786C394FEEE9497
:10511C00FF400A1252DF901C0F74808004901C0F09
:10512C00E475F00212279F025228901C0BE0FFA39B
:10513C00E0901C0FCFF0A3EFF0900C39E0704F1201
:10514C004879604A124544901C12F0BEFF0BBFFF19
:10515C00081252DF12466F800312453A901C12E07F
:10516C0070E2901C11E004F0901C0DE0FEA3E0FF37
:10517C00A3E0B506C4A3E0B507BF901C16E0FF90F2
:10518C001C15E06F70B3900C397403F080AB900C6D
:10519C0039E06003025254025228901C07E070065A
:1051AC0012464C124884901C16E0901C15F0901C72
:1051BC000D1246FC400EEF24FEFFEE34FFA3F0A3CD
:1051CC00EFF0800A901C0EE0901C0D1246BF901C54
:1051DC0015E0FF125BE412454460331247D6EFB57D
:1051EC00050BEEB50407124778E06F602112478675
:1051FC00B40016EEB480121246CCE0FF125BE474DD
:10520C00FF901C0FF0A3F080CD12465580C81246BB
:10521C00DA6E7003A3E06F600312453A901C0F1214
:10522C0046A68024901C07E0700612464C12488457
:10523C00124778F01247D6A3ECF0A3EDF0901C0FB8
:10524C00ECF0A3EDF0125BE4900C39E070701245B9
:10525C0044FD901C13E0FC04F074F72C12455EED39
:10526C00F0901C12F0BEFF11BFFF0E901C15E00455
:10527C00FF125BE412466F800312453A901C12E059
:10528C0070CCA3E014900C3AF0901C07E0901C0B2F
:10529C00701612481C78637C0C7D017B017A1C799A
:1052AC00147E007F0302260D124829901C15E090F5
:0E52BC000C42F09008F6E0FEA3E0FF12EA605C
:1052CA0022901C15E014F0E0FF125BE474FF901CBE
:1052DA000FF0A3F022901C15E004F0E0FF125BE44B
:0152EA0022A1
:10C6B000900C54E064017054901BAEE075F002A43D
:10C6C000FDACF0901BADE075F014A42DFFE5F03C3F
:10C6D000AD07FC901BB0E0D394024017901BAFE075
:10C6E000D39407400974022DFDE43CFC80050DBD88
:10C6F00000010C900C73E0FFAB05AA047D5212BA46
:10C7000073E4900C50F0900C54F0803812465F2087
:10C71000E014900C73E0FF12F0C7BF4907900C546F
:10C720007401F022801E900C50E06401600B900CAC
:10C7300073E0FF12F0C7BF490BE4900C50F0900C6F
:08C740005404F02212452BF015
:01C7480022CE
:10DFE800780C7C1E7AF179297E007F0212485390C2
:10DFF8000C5D7401F01289F39007AE122A2A90087A
:10E00800DFE0F460F912F6769008DFE0F460F912C8
:10E0180046D31313540120E0167B017A1E790C9025
:10E0280007AE122A2A12F6769008DFE0F460F9E4C7
:09E03800900C5DF07F0602DCF3A0
:1063E4009012A074011248CAA3F01247CD6006901F
:1063F400129DF0801A1245A312F9A312F774901299
:106404009D12474A500690129DE0700312477F90F8
:106414000C39E0600302665690129D1245B512C70E
:10642400DF900D81124829900C41E0A3F012485AE4
:10643400900C5BE02F0490129FF0901BBCE020E0D6
:10644400030264CBE0FEA3E07805CEC313CE13D8D9
:10645400F930E014901BB1E0B40106900C3AE080EE
:106464001912476EC39F8012900C3A124602FED353
:106474009F400D901BAFE0FDEF9D9013A2F08005AF
:106484009013A2EEF0E49013A1F0901BAFE09013F0
:10649400A0F09013A2E0FF9013A1E0FEC39F50224E
:1064A4009013A0E024F712455EE0FF9013A1E0FDF5
:1064B40004F074A12D124866EFF09013A0E004F0EC
:1064C40080D074A12E80397F05125BE41245AC1292
:1064D400F9A3901BB0E09013A21248CA901BB0E03D
:1064E400FD9013A0E0FCC39D501312473F74A12CF0
:1064F400124866EDF09013A0E004F080DF74A12C44
:10650400124866E4F0124639900C42E0FF125BE454
:10651400900C58E0FF9013A2E0D39F40030266560C
:10652400900D86E0FEA3E0900C691248D1B50713E4
:10653400ECB5060F900C43E0FF900C42E06F700343
:106544000266569012A0E064016003026656900C45
:1065540042E090129EF0900C57124836D3ED9FEC17
:106564009E401290129E126657900C57E090129A19
:1065740012475D8018900C57E0FF900C6AE02FFEE4
:10658400900C69E0340090129AF0A3CEF07B017A6B
:106594001279A190129AE0FCA3E0FD90129EE09083
:1065A4001D5CF012D023EF640170709012A0F09083
:1065B4000C39F0900C69E0FFA3E090129ACFF0A39D
:1065C400EF1248CA900C42E0FF125BE490129A1258
:1065D4004547FD9013A0E0FC04F074F82CF582E428
:1065E4003409F583EDF090129CF0BEFF14BFFF1147
:1065F400900C42E004FF125BE490129A12467280FF
:106604000690129A12453D90129CE070BF9008F6D5
:10661400E0FEA3E0FF12EA6002652490129F124894
:1066240036900C69E0FCA3E0D39FEC9E4013900CE1
:106634004212665790129FE0900C6912475D026502
:106644002490129FE0FF900C69E48FF012279F02C0
:026654006524BB
:1066560022E004F0E0FF125BE4900C69E0FEA3E0A8
:10666600FF9013A3EEF0A3EFF0C3E49FFFE49EFEBA
:08667600C3E49FFFE49EFE2235
:10B39700900C60E06401600302B43A1245AC12F904
:10B3A700A3901DE112478E901DE312467930E0030A
:10B3B70012F8A7901DE112469E7B01A3E0FD12A3A0
:10B3C7008BE4900C60F090040104F0E4901A98F07C
:10B3D70012FB9912FBB9901BB2E024FE6037146090
:10B3E7002C14604414601614600B14703BE4FB7D4E
:10B3F700017F028039E4FB7D017F038031E4FB7D1F
:10B40700017F048029E4FB7D017F058021E4FB7D2A
:10B41700017F068019900C387414F0900C40740367
:10B42700F0E4900401F0802CE4FB7D017F05128796
:10B437002E802112F9FF401C900C607401F09007D8
:10B44700AE1229F3E41226CE12FA5A7BFF7AF67966
:08B457007602F39312452BF07D
:01B45F0022CA
:10E23F00900D99E06401702D1245AC12F9A3901D59
:10E24F00E412478E901DE612467930E00312F8A7CC
:10E25F00901DE412469E7B01A3E0FD12A38BE49078
:10E26F000D99F0801712F9FF5012900D997401F06B
:10E27F0012FB9912FBB9E4900C3BF02212452BF0E4
:01E28F00226C
:06FDF900E4900C3CF02236
:106EC000900D9CE0FEA3E0FF901D3BEEF0A3EFF0E1
:106ED000A3EEF0A3EFF0900C64E0901D3FF0A3F060
:106EE000900C4BE0FEA3E0FF900C44E06E7003A317
:106EF000E06F70030270A5901D3FE0FF125BE4900D
:106F00001D3B124547901D41F0BEFF0EBFFF0B1207
:106F100070A9901D3B1246728006901D3B12453DA4
:106F2000900C6C122981EF2401FFE43EFEE43DFD4C
:106F3000E43CFC900C6C122999901D41E070C090CB
:106F40000C4BE0FEA3E0FF901D3BE0B50611A3E073
:106F5000B5070C900C53E0FF901D3FE06F6064900C
:106F60001D3FE0FF125BE4901D3B124547901D4121
:106F7000F0BEFF0EBFFF0B1270A9901D3B124672B0
:106F80008006901D3B12453D901D40E0FF125BE4E2
:106F9000901D41E0901D3D1248D1F5828C83EFF0A9
:106FA000BCFF17BDFF14901D40E004F0E0FF125B32
:106FB000E4901D3D124672026F3F901D3D12453D0B
:106FC000026F3F901D3DE0FEA3E0FFEE12488E9061
:106FD0001D40E0900C53F0900D9CE0FCA3E0FD6F91
:106FE0007002EC6E600302709F900C44E0FEA3E020
:106FF000FFED6F7002EC6E700302709A900C53E01C
:10700000900C52F0900C4B1246FC4008901D3D1223
:1070100047A38017900C4CE024FEFE900C4BE0340C
:107020007F901D3DF0A3CEF01270B5900C52E0FFA2
:10703000125BE4901D3D124547603D900C44E0FC1E
:10704000A3E0FDEFB5050EEEB5040A900C51E0FF8C
:10705000A3E06F6023901D3DE0FEA3E0B40011EEBD
:10706000B4800D1270B574FF901D3DF0A3F080C385
:10707000901D3D12465880BB900C44E0FEA3E0FFFB
:10708000901D3DE06E7003A3E06F6006901D3D1201
:10709000453D901D3D12481C8005E4FF12FC07E4AD
:0870A000900C39F02212477F29
:1070A80022901D3FE004F0E0FF125BE422900C52B6
:0970B800E014F0E0FF125BE42299
:0AFD0A00E49009F7F09008F8F022E9
:10D7AD00900C5D7401F0900C70E064017028900A8B
:10D7BD00F7F0900C3AF0901BADE075F014A4FBAAB5
:10D7CD00F0900C73E0FF7D5212BA73E4900C70F080
:10D7DD009008F5F08030900C73E0FF12F0C7EF6405
:10D7ED0049600C901BAEE0FF9008F5E0B50717906F
:10D7FD000C707401F0900C5DF0900C3AE024F7126F
:0FD80D00455EE4F0800412452BF07F0602DCF349
:10DF8C00901E2EEFF0901A98E07022901E2EE0FF5B
:10DF9C00640D600C124554EFF09008F5E004F0228B
:10DFAC00900C73E0FFE4FBFA7D4902BA73901E2ECD
:10DFBC00E0FF640D901A976011E0FE04F074542E8B
:10DFCC00F582E4341AF583EFF022E02454F582E470
:0CDFDC00341AF583E4F0901A9904F02246
:10F001001247F1A3E01330E00A12FC5F900C4F7439
:10F0110001F022900C68E075F014A4FFAEF012FD2F
:10F021006912F98BE4900C4FF012F9FF400312D4EE
:02F03100882233
:103C0800E4901B37F0A3F0A3F01245AC12F9A3908F
:103C18001B2E12459E12F9A3901B301248A1900C3E
:103C28003912467920E01EE4901B36F0C312468311
:103C3800400302402012471685F0821244CCEFF070
:103C480012484380E712472B12F9A3901B321248FF
:103C5800D864027003023DBE901BB8E024D56070A2
:103C680024FE7003023D1D240360030240207B01F3
:103C78007A1B794612E759C004C005C006C0077B05
:103C8800017A1B793E12E759D003D002D001D00047
:103C9800121FE7901B4E1229997F207EBC7DBE7CA7
:103CA8004C901B4E12298D1220ED600540031246E0
:103CB8003912403EC004C005C006C007124021D0DA
:103CC80003D002D001D0001228051246EA023DA214
:103CD80012403EC004C005C006C007124021D003F0
:103CE800D002D001D0001227EA1246EA7EE07DF524
:103CF8007C051247084008901BB0E064086010E497
:103D0800FEFDFC124708400A901BB0E0B403031202
:103D18004639023DA2901B321245FFFD12C875C0FC
:103D280004C005C006C0071245FCFD12C87512473D
:103D3800DFD007D006D005D004C3122930901B323B
:103D48001245FFFD401F12C875C004C005C006C05B
:103D5800071245FCFD12C875D003D002D001D0006F
:103D68001246E7803512C875122922C004C005C062
:103D780006C0071245FCFD12C875D003D002D00159
:103D8800D0001227EAE42FFFEE34E1FEED34F5FD12
:103D9800EC3405FC1246EA124639901B3A12298186
:103DA800901C48122999901BB0E0FD901B2EE0FE54
:103DB800A3E0FF02B12D1246D3540730E003023EC0
:103DC80058901BBAE0FF1248963400CF24FFCF3436
:103DD800FF901B34F0A3EFF0901B34124547FDB45D
:103DE8002014901B30E06E7003A3E06F6008901BF6
:103DF8003412465880E2EDB42006901B377401F067
:103E08001248E2124682503BA3E0701E1246F0129E
:103E180044CE124714FE901B34E06E7004A3E06594
:103E2800F0701A901B3704F080131246126F600767
:103E38001244BCEFF080061244D07420F0124843BC
:103E4800023E0B124612C39F4003024020023F8FDE
:103E5800901BB9E0146065147003023F41147003AD
:103E6800023F96240360030240201248E212468271
:103E7800503DA3E07020A3E0FF04F0901B301244F3
:103E8800C3EFF0901BBAE0FF901B38E06F701A90F8
:103E98001B3704F080131246126F60071244BCEF00
:103EA800F080061244D07420F0124843023E751286
:103EB8004612C39F4003024020023F8F901BBAE086
:103EC80024FFFFE434FFFE1248963E901B34F0A313
:103ED800EFF0901B341246F3E0B42008901B341224
:103EE800465880EE901B3412453D1248E212468235
:103EF800503BA3E0701E1246F01244CE124714FE47
:103F0800901B34E06E7004A3E065F0701A901B37C4
:103F180004F080131246126F60071244BCEFF08061
:103F2800061244D07420F0124843023EF51246129D
:103F3800C39F4003024020804E901BB8E0901B3284
:103F4800B42B1B124067C004C005C006C00712404E
:103F580032D003D002D001D0001227EA80191240D3
:103F680067C004C005C006C007124032D003D002A3
:103F7800D001D0001227F71246EA7F3F7E7E7D05EA
:103F88007C0012470A4004124639220240081240B7
:103F98004FC004C005C006C00712405B1247DFD0FF
:103FA80007D006D005D004C3122930401812404F5C
:103FB800C004C005C006C00712405BD003D002D0C1
:103FC80001D0008038901B30E0FEA3E0FF12C57BD3
:103FD800EF2480FFEE3451FEED3401FDE43CFCC0DB
:103FE80004C005C006C007901B32E0FEA3E0FF1224
:103FF800C57B1247DFD007D006D005D0041246E7AC
:10400800901B3A122981901B2EE0FBA3E0901BD64F
:08401800CBF0A3EBF012B5F0B0
:1040200022901B30E0FEA3E0FF901BB0E0FD12C821
:104030007522901B30E0FEA3E0FF12C57B22901B8F
:1040400032E0FEA3E0FF901BB0E0FD12C8752290A5
:104050001B32E0FEA3E0FF12C57B22901B30E0FE86
:10406000A3E0FF12C57B22E0FEA3E0FF12C57B2286
:105E9500901BB6E07006126130EF8004901BB6E0EF
:105EA500149014ABF0901BB9E0700A126130901495
:105EB500ACEFF08008901BB9E09014ACF0901BAEED
:105EC500E024C16033146003025F4F9014AB1247A6
:105ED50071FED39F401F1247AF5002EFF01247E803
:105EE5001245844003025F8D74F72EF582E4340A6F
:105EF50012450A80EB025F8812610EFDD3EF9D7497
:105F050080F86E98404112610EFDC3EF9DFFEE943F
:105F150000FEA3E0FDC3EF9D7480F86E9850137BDF
:105F2500017A0979F812FADB9014ABE0FEC3EF9E13
:105F3500A3F01247E8124584504E74F82EF582E41A
:105F4500340912450A80EE025F881245AC12F9A3A6
:105F55009013A5EEF0A3EFF09014AB124602FED31A
:105F65009F40201247AF5002EFF01247E8124584D8
:105F750050169013A5E0FCA3E02EF582E43C1245F3
:105F85000A80EAE49014ACF0901BB1E0644360032E
:105F950002603C901BADE060069013ABF0801A12D6
:105FA50045A312F9A312F7749013AB12474A500692
:105FB5009013ABE0700312477F9013AB1245B512F7
:105FC500C7DF900C42E0FF125BE412485AE433FE4F
:105FD500900C6AE02FFF900C69E03EFE900C5BE0B0
:105FE500FD9014ACE0C39D5036E4A3F09014ACE0F2
:105FF500FDA3E0FCC39D500812611C12452480ECF2
:106005009014ACE0A3F01248E9C39D400302610D72
:106015008F828E837420F012F73612452480E7E4D0
:106025009014ADF01248E9FCC39D400302610D12C6
:10603500611C12452480ED1245A312F9A39013A803
:106045001248D89013AAF07F05125BE49013AAE0DA
:10605500FF9014ACE0C39F40030260F2901BB5E0D3
:10606500640270419014ADF09014ACE0FFA3E0FE23
:10607500C39F501D74AC2EF582E43413F583E0FD07
:106085009013A8E0FAA3E02EF582E43A12452080A9
:10609500D79014ADEFF012468E506D1245D5742091
:1060A50012452380F1E49014ADF09014ACE0F99022
:1060B50013AAE0C399124692500A1245D5743012BC
:1060C500452380E69014ADEFF012468E503A9014B9
:1060D500AC1247F8FCEEC39DFDE49CFC74AC2DF5B9
:1060E5008274133C1245D1EF12452380DCE49014F1
:1060F500ADF012468E501174AC2EF582E4341312B5
:0861050045D1EF12452380EAA9
:10610D00227B017A0979F812FADB9014ABE0227444
:10611D00AC2CF582E43413F583E08F828E83F0127C
:10612D00F73622A3E0FFA3E0FD12F9A312F77422C4
:1090A700E4901DE7F0A3F0A3F0901BADE024FE6071
:1090B7002314602D14603B14603C1470030291E08C
:1090C700240560030291EB900C3AE0FDB40802809E
:1090D700180291DC900C3AE0FDB40D02800B02916E
:1090E700DC900C3AE0FDB40C061248F30291E8025A
:1090F70091DC12477F22E4FF900C3AE014FEEFC3A5
:109107009E40030291AD74F72F12455EE0FEC394B3
:1091170030400BEED394395005EE24D0801674F707
:109127002F12455EE0FEC394414014EED3945A508B
:109137000EEE24C9FDE434FF901DE78DF0806074C6
:10914700F72F12455EE0122AC8917B209184249163
:109157009F2591962B91692D91722E918D2F00004D
:1091670091A9901DE7E475F0248034901DE7E4751C
:10917700F025802B901DE7E475F0268022901DE7EF
:10918700E475F0278019901DE7E475F028801090AA
:109197001DE7E475F0298007901DE7E475F02A12B2
:1091A700279F0F0290FF901DE7E0FEA3E0FF7C00E2
:1091B7007D2B122714A3EDF0E090F12B93FF900C79
:1091C7003AE024F6F582E4340AF583E0B50706E4CD
:1091D700900C39F022124639221248F3900C3AE0EB
:0491E700FD12C12490
:0191EB002261
:10F736000FEFAC0670010E14FDBCFF12BDFF0F905B
:0FF746000C42E004F0E0FF125BE47E807F0022C3
:10946400901C777430F0A3F0A31246097802CEC39F
:1094740013CE13D8F930E0231245AC1295887D0839
:1094840012C875901C6E12459E1295887D0812C8EC
:1094940075901C70EEF0A3EFF08008901C70E4F05F
:1094A400A304F0901BB8E0603412472B12F9A39088
:1094B4001C721248A1FF901BB8E0FEEFC39E50102F
:1094C400901C721244D3E0FE124734EEF00F80E693
:1094D400124734E4F07B017A0879E480067B007A51
:1094E400007900901C74122A2A1246D3540730E0E3
:1094F4003A901BB9E0FF12FC51901C77EFF0124632
:10950400D313540330E00D901BBAE0FF12FC5190CA
:109514001C78EFF01246D31313540130E00D901B66
:10952400BBE0FF12FC51901C79EFF0901C77E0FF38
:10953400A3E0FD901C6EE0FBA3E0901BF9CBF0A32D
:10954400EBF0901C70E0FBA3E0901BFBCBF0A3EBD3
:10955400F0901C741229F3901BFD122A2A1248F36E
:10956400901C00122A2A901C79E0FB1296BB900CE6
:1095740039EFF0700E901A97E0900C3AF0900C3D91
:039584007454F02C
:0D9587002212F9A3901C72EEF0A3EFF02267
:109D5D001247F130E00A74FF901C86F0A3F0800EDC
:109D6D001245AC129E59901C86EEF0A3EFF01245F1
:109D7D00A3129E59901C89EEF0A3EFF0901BB8E052
:109D8D00603C901BB6129E48E4A3F0901BB812489D
:109D9D00FA5018901C8B1244D3E0FF74E42E124736
:109DAD0037EFF0901C8DE004F080E0901C8DE024E6
:109DBD00E4124737E4F07B017A0879E480067B00F2
:109DCD007A007900901C8E122A2A901BB9E0FF129E
:109DDD00FC51901C88EFF0901BBA129E48E4A3F042
:109DED00901BB41248FA501C901C8B1244D3E0FF08
:109DFD0074F72EF582E4340BF583EFF0901C8DE0B3
:109E0D0004F080DC901C8DE024F7F582E4340BF532
:109E1D0083E4F0901C88E0FF901C86E0FCA3E0FD3D
:109E2D007B017A0B79F7901C97122A2A901C8E12BF
:0A9E3D0029F312BC8E900C39EFF0EF
:109E470022E0FFA3E0FD12F9A3901C8BEEF0A3EF35
:109E5700F02212F9A3901C8BEEF0A3EFF07D08120D
:039E6700C8752299
:06E2E000901D42122A2AE3
:10E2E600E4FF901D48E0FEEFC39E503D901D421294
:10E2F60045F6C41245E4D3943940057407122679CD
:10E30600901D4612453D901D421245F61245E4D336
:10E31600943940057407122679901D4612453D90A2
:09E326001D4312453D0F02E2E81F
:01E32F0022CB
:06D4FD00901D49122A2ACD
:10D50300E4FE901D4FE0FDEEC39D5062901D491255
:10D5130045F6FDD394394005ED24C98008901D4993
:10D523001245F624D012486E901D49E475F001129D
:10D5330029FC122633C454F012486E901D4912453B
:10D54300F6FDD394394006ED24C9FF800612263335
:10D5530024D0FF901D4C1245F64F1226CE901D4D40
:0ED5630012453D901D4A12453D0E0E02D505A3
:01D571002297
:10B9BB001245AC12F9A3901D7312459E12F9A39078
:10B9CB001D7512478E901D77F0901BB1E0901D787E
:10B9DB00F0E4FF901D78E0FEEFC39E5011901D75B3
:10B9EB00E0FCA3E0F5828C837420F00F80E5E41279
:10B9FB0047CD64017037EE75F002A4FF901D77E020
:10BA0B00D39FE5F01245974002803612469B7B018F
:10BA1B00C002C001A312469E901D4C122A2A901DF3
:10BA2B0077E0901D4FF0D001D00202D4FD901D772E
:10BA3B00E075F002A4FFA3E0C39FE5F01245975019
:10BA4B00041246392212469B7B01C002C001A3128D
:10BA5B00469E901D45122A2A901D77E0901D48F0B6
:07BA6B00D001D00212E2E05D
:01BA720022B1
:108CBB00901D531229F3122633FF901D501229F3E6
:108CCB0002263314F5828E83E022E0FCA3E0FD2420
:108CDB0006F582E43CF58322E0FF04F074742FF573
:108CEB0082E4340CF58322E0FF901C611229F3908F
:108CFB001C6DE0FE04F08E82758300EF22901CD772
:108D0B001229F38F8275830012264C24D0FDE43494
:108D1B00FF901CDB8DF012279F0F0F22C39FC39474
:108D2B0000901D56227C002400FFEC3EF0A3EFF0D8
:108D3B00901E0EE022EF2405F582E43EF583E0223F
:108D4B00901D79E0FEA3E0F5828E8322E47B107AFE
:108D5B000E901BD2F9F8122981022890901BBCE0CF
:108D6B00FEA3E022E475F00102279F901DA1E4759C
:108D7B00F0011229FC122633FF22901BBCE0C41316
:108D8B0022E004FFF07E00900C49E0FCA3E0FD1212
:108D9B002769ED4C221227EAA804A905AA06AB07FE
:108DAB0022122981901C48022999A3E024D0FFE4C8
:108DBB0034FFFE22AC00AD01AE02AF03901BE0020C
:108DCB002999E024D075F00AA422901CDBE0FEA3C5
:108DDB00E0FF7C002274B42FF582E43414F5832277
:108DEB00901BBCE0131322EEF0A3EFF0A322122989
:108DFB0081E47B0AFAF9F822F0A3EFF0900C59E02A
:0C8E0B00FF22901CDAE014FEEFC39E2250
:107A1A00AD07AC068D828C83E0FEA3E07A002400D9
:107A2A00FFEA3E901BBCF0A3EFF074022DFDE43C8C
:107A3A00FC0DEDAE0470010C128CCE901BACF090D4
:107A4A001BBCE0C313A3E01330E00E0DEDAE0470CF
:107A5A00010C128CCE901BADF0128D677802CEC34A
:107A6A0013CE13D8F930E00E0DEDAE0470010C12EE
:107A7A008CCE901BAEF0128D677803CEC313CE1353
:107A8A00D8F930E00E0DEDAE0470010C128CCE90D8
:107A9A001BAFF0901BBCE0C4F854F0C8A3E0C45478
:107AAA000F4830E00E0DEDAE0470010C128CCE9032
:107ABA001BB0F0128D677805CEC313CE13D8F930F8
:107ACA00E00E0DEDAE0470010C128CCE901BB1F0DD
:107ADA00128D677806CEC313CE13D8F930E00E0D97
:107AEA00EDAE0470010C128CCE901BB2F0128D67B1
:107AFA007807CEC313CE13D8F930E00E0DEDAE04DD
:107B0A0070010C128CCE901BB3F0901BBCE030E0DD
:107B1A000E0DEDAE0470010C128CCE901BB4F090D9
:107B2A001BBCE0C31330E00E0DEDAE0470010C1265
:107B3A008CCE901BB5F0128DEB543F30E00E0DED5C
:107B4A00AE0470010C128CCE901BB6F0128DEB13A2
:107B5A00541F30E00E0DEDAE0470010C128CCE9065
:107B6A001BB7F0901BBCE0C4540F30E00E0DEDAE15
:107B7A000470010C128CCE901BB8F0128D8554073C
:107B8A0030E00E0DEDAE0470010C128CCE901BB9D4
:107B9A00F0128D8513540330E00E0DEDAE04700122
:107BAA000C128CCE901BBAF0128D8513135401302F
:107BBA00E00DAE04AF058F828E83E0901BBBF022EE
:10F774008F828E83A3128DCDFD8F828E83E024D061
:0DF7840075F064A42DFDA3A3E024D02DFF9B
:01F791002255
:08C87500901C7A128DF2EDF027
:10C87D00901C7E1229A500000000901C821229A593
:10C88D0000000001901C7D7401F0901C7CE0FFA362
:10C89D00E0D39F5061A312298DC000C001C002C01A
:10C8AD0003901C7DE0FF901C7CE0C39FFFE494008F
:10C8BD00FE901C7AE0FCA3E02FF582EC3EF583128E
:10C8CD008DB6E4FCFD901C8212298D122805D00333
:10C8DD00D002D001D0001227EA901C7E1229999027
:10C8ED001C82128DF9122805901C82122999901C18
:0CC8FD007DE004F08094901C7E122981E4
:01C90900220B
:09B12D00901C45128DF2EDF0FBBF
:10B13600901C4D1229A500000064BB080A901C4D06
:10B146001229A500989680E4901C4CF0901C47E0CC
:10B15600FF901C4CE0C39F400302B1FDA312298D52
:10B16600901C48128D61901C51EFF02430FFE4339F
:10B17600FED3EF9439EE648094804010E02426A339
:10B18600F0D39439400EE024BAF08008901C51E0C8
:10B196002430A3F0901C52E0FF901C4CE0FE901C63
:10B1A60045E0FCA3E02E128CDCEFF0901C4812293F
:10B1B60081C004C005C006C007901C51E0FFE4FC36
:10B1C600FDFE901C4D12298D122805128DA3D00765
:10B1D600D006D005D0041227F7901C481229999062
:10B1E6001C4D128DF9122890901C4D122999901C15
:07B1F6004CE004F002B1522D
:01B1FD00222F
:06C99C00901C61122A2A22
:10C9A2007B017A1C7968901C6A122A2A901C6412F4
:10C9B2008CC8901C6DF0901C67E0FD6443601EED16
:10C9C20064596019ED644D6014ED6444600FED64C8
:10C9D20068600AED646D6005ED6473701C901C6AFA
:10C9E2001229F312D39B901C68128CF21226E0904B
:10C9F2001C69E0FF128CFA8021901C67128CF212E3
:10CA020026E0901C6DE07E0029F9EE3AFA90FFFFD5
:10CA120012264C700890FFFF742E1226E0901C6DB7
:0CCA2200E0FF901C641229F3EF0226CE06
:10D39B00ED122AC8D3B843D3DC44D3D04DD3C459F0
:10D3AB00D3E868D3F46DD400730000D41190050357
:10D3BB00E01226CE9005048046900505E01226CE9D
:10D3CB00900506803A900500E01226CE900501806C
:10D3DB002E9004FDE01226CE9004FE8022901AB20D
:10D3EB00E01226CE901AB38016901AB5E01226CE14
:10D3FB00901AB6800A901AB8E01226CE901AB9E0AD
:07D40B009000011226E0224F
:107D6F00EF122AC87DB3417DBD427DC6437DCF440E
:107D7F007DD8457DE1477DEB4A7DF44B7DFA4C7E06
:107D8F000B4D7E154E7E1F4F7E2C507E39517E46F9
:107D9F00527E53537E63547E6C557E74567E80584C
:107DAF0000007EB8D270901E33740F027E5AD270CC
:107DBF00901E337401803BD270901E337405803255
:107DCF00D270901E33740D8029D270901E33740EB2
:107DDF008020D270901E337418027E5AD270901E7B
:107DEF00337409800D9008E3027EB5D270901E3374
:107DFF007403F012FA9C9008E1027EB5D2707404FD
:107E0F00127ED1027EB5D2707407127ED1027EB57A
:107E1F00D2707408127EDC9008E1027EB5D27074C5
:107E2F0006127EDC9008E1027EB5D270740C127ED1
:107E3F00E49008E1027EB5D270740B127EE49008D4
:107E4F00E1027EB5D270901E33741B127EF990083A
:107E5F00E1027EB5D270901E337414800F127EC56E
:107E6F009008E18041D270901E337415127EF98014
:107E7F0038D270740F127EEC7418F012FA9CD27113
:107E8F00901E34740FF012FAB1127EC5D2707405C1
:107E9F00127EEC740D127F09740E127F097409F0B3
:107EAF0012FA9C9008E17401F09008E1E0B401052A
:107EBF00E49008E3F022D270901E337402F012FAAD
:107ECF009C22901E33F012FA9C9008E122901E33F0
:107EDF00F012FA9C22901E33F012FA9C22901E335D
:107EEF00F012FA9CD270901E3322F012FA9CD271CB
:107EFF00901E34740FF012FAB122F012FA9CD27065
:047F0F00901E33226B
:10ADD700EF122AC8AE3710AEA011AE6112AE6813DB
:10ADE700AE3E20AE7D21AE6F30AE7640AE5A50AE4D
:10ADF7008B60AE8470AE4580AE9281AE4C90AE5300
:10AE0700A0AE30B0AE99B1AEA7B2AE30B8AE99B978
:10AE1700AEA7BAAE30D0AE99D1AEA7D2AE30E0AEC3
:10AE270099E1AEA7E20000AEAD900C3E7441F0226E
:10AE3700900C3E7442F022900C3E7443F022900C2A
:10AE47003E7444F022900C3E7445F022900C3E7400
:10AE570047F022900C3E744AF022900C3E744CF05E
:10AE670022900C3E744DF022900C3E744EF02290CE
:10AE77000C3E744FF022900C3E7450F022900C3E22
:10AE87007451F022900C3E7452F022900C3E745391
:10AE9700F022900C3E7454F022900C3E7455F02230
:07AEA700900C3E7456F022EE
:06959400901D50122A2A6E
:10959A00E4901D56F0901D56E060030296B5901DAA
:1095AA0053128CC824DD700302963524FD70030221
:1095BA00964C24E7604214605924E46021243B60FD
:1095CA0003029666128CC5FF12F872500302966D5A
:1095DA00128CBB128D27501D029683029688128C1C
:1095EA00C5FF12FC16500302966D128CBB128D2712
:1095FA005003029683029688128CC5FF12FC2550EE
:10960A000302966D128CBB128D27500302968302B9
:10961A009688128CC5FF12F8725002802E128CBBEB
:10962A00128D275003029683029688128CC5FF1268
:10963A00FC1650028015128CBB128D2750028039FD
:10964A00803C128CC5FF12FC255005901D51801CD0
:10965A00128CBB128D275002801F8022128CBBFEF7
:10966A00B5070E901D51128D6F901D54128D6F808B
:10967A0010EEC39F901D5650057401F080037402CA
:10968A00F0128CC5600B901D53128CC860030295B2
:10969A009F901D53128CC8FF6421600CEF645C60BC
:1096AA0007EF643F600280037F0122901D56E0FFAE
:0196BA00228D
:10C7DF00901E0EEE128E03125BE4901E0E128CD57D
:10C7EF00E0FEED2407128CDCE0900C69128D30FC1A
:10C7FF00A3E0F5828C83E0FEA3E0900D81128D30D3
:10C80F00FCA3E02409128CDCE0FEED240A128CDC80
:10C81F00E07C002400FFEC3E900D86128D37FEA3C6
:10C82F00E0FF2408128D43900C42F08F828E83A379
:10C83F00A3E0900C41F0901E0EA3E0240B128D4349
:10C84F00900C43F08F828E83A3A3A3E0900C57F03C
:10C85F00901E0EA3E02404128D43900C58F0128DFD
:06C86F0040900C5BF0227A
:08EA6000901DB4EEF0A3EFF0ED
:10EA6800900C69E0FFA3E0901DB6CF128E03125BF5
:10EA7800E4901DB6E0FF901DB4128CD5EFF0901D08
:10EA8800B7E0FFED2407128CDCEFF0900C42E0FFBA
:08EA9800ED2408128CDCEFF004
:01EAA0002253
:0ED02300901D57122A2A901D5AECF0A3EDF032
:10D03100E4901D5DF0901D5CE0FF125BE4901D57D4
:10D04100128D79901D5AE0FCA3E0FDF5828C83E0FE
:10D05100FE6F6005EE643F704ABCFF19BDFF16907C
:10D061001D5CE004F0E0FF125BE4901D5A7480F057
:10D07100A3E4F08006901D5A128D6F901D5DE004AF
:10D08100F0901D57128CC870B4900C58E0FF901DA1
:10D091005DE06F600B901D5A128D4EE0643C709DF7
:05D0A1007F01227F0069
:01D0A6002267
:0BC12400901CD7122A2A901CDAEDF0C4
:10C12F00E4A3F0A3F0A3F0900C3AE020E00AE4902F
:10C13F001CDEF0A304F08009901CDE7401F0E4A370
:10C14F00F0901CDEE0FF128E0D5005128D0880F668
:10C15F00128DD57D03122702901CDBEEF0A3EFF0BA
:10C16F00901CDFE0FF128E0D5005128D0880F61225
:10C17F008DD57D0A122714AF05A3EFF06007E0FFFE
:10C18F00C3740A9FF0901CDDE02430F0901CDAE0BD
:10C19F0024FFFFE434FFFE901CD71229F38F828E09
:10C1AF008312264CFF901CDDE0B50706E4900C3996
:08C1BF00F022900C397401F02C
:01C1C7002255
:1089F300E49014B2F0A3F0128D677806CEC313CEC1
:108A030013D8F930E00C901BB2128B49EF14901479
:108A1300B2F0128DEB543F30E00B901BB6128B4932
:108A23009014B3EFF0901BBCE020E003028AAF90F8
:108A33001BB0E0702E9014B3E07028901BAEE0B42E
:108A4300400D901BB1E0FF900C3AE0C39F80117B77
:108A5300017A0979F812FADB901BB1E0FEC3EF9EAD
:108A630004800A9014B3E0FF901BB0E02F9015B37D
:108A7300F0901BAEE09014B2B4400FE0FF901BAF38
:108A8300E024F7F582E4340A800DE0FF901BAFE0A9
:108A930024F8F582E43409F583E5822FF582E43581
:108AA30083AF829014AEF0A3EFF08043901BB0E04D
:108AB30060028016901BB5E0FF600B901BB1E0FED7
:108AC300C3EF9E0480049014B3E09015B3F0901BA1
:108AD300AEE0FFA3E0FD12F9A39014AEEEF0A3EF16
:108AE300F09014B2E0FF9014AEE48FF012279F12BF
:108AF3008D8513540330E0219014AE128D4EE0B4F3
:108B030030179015B3E0D39401400E9014AE128D3C
:108B13006F9015B3E014F080DFE4FF9015B3E0FE2F
:108B2300EFC39E50159014AEE0FCA3E02F128CDC33
:108B3300E0FE128DE0EEF00F80E1128DE0E4F07BB9
:058B4300017A1479B471
:108B480022E0FFA3E0FD12F9A39014B0EEF0A3EF2A
:058B5800F012F7742289
:06A38B00901DA1122A2A18
:10A39100E4901DA4F0A3F0900D94E014FC128D85BF
:10A3A10013540330E018901DA1128CC8B4300FED86
:10A3B100D394014009901DA2128D6F1D80E8E49095
:10A3C1001DA4F0901DA4E0C39D5063128D85540718
:10A3D10030E005900D94E0FC900D73E06C703090CE
:10A3E1001DA5F0901DA5E0FF2475F582E4340CF560
:10A3F10083E0FE600D128CE7EEF0901DA5E004F005
:10A4010080E1128D7674732CF582E4340C80121283
:10A411008D76900D73E0FE04F074742EF582E434B1
:10A421000CF583EFF0901DA4E004F002A3C4900D9D
:10A4310073E02474128CEAE4F0FDFF12A183E4902E
:10A441001DA4F0A3F0901DA4E02474128CEAE06036
:10A451001A901DA4128CE3E0FF12A486901DA51290
:10A461008D8C70E17F0A12A48680DA128D855407E3
:10A4710020E00B7F5F12A486E4900C6BF022900C1D
:04A481006B7401F007
:01A4850022B4
:10D88A00E4901DEAF0A3F0900D94E0FE14901DECD4
:10D89A00F0900C6BE0B40105901DECEEF0E4FDFF96
:10D8AA0012A183901DECE0FF900D73E0FED39F4020
:10D8BA0006EE9F901DEAF0901DEAE02474128CEAAD
:10D8CA00E0601A901DEA128CE3E0FF12A486901D14
:10D8DA00EB128D8C70E17F0A12A48680DA900C6BB1
:0BD8EA00E07008900C55E0FF12A486CF
:01D8F5002210
:10F9A300EFFE7C00E42DFFEC3EFE900D98E02FFF70
:06F9B300900D97E03EFEFE
:01F9B900222B
:03C57B00901D7997
:10C57E00128DF21229A500000000128D4B128DB5FE
:10C58E00E4FCFD7BA07A8CF9F8122805901D7B1235
:10C59E002999128D4BA3128DB57C0E7D1012270298
:10C5AE00E4FCFD901D7B12298D128DA0901D79E06B
:10C5BE00FEA3E0FF2404128D43128DCEFD128D409A
:10C5CE0024D02D75F03CA4FFAEF0E4FCFD128DA03E
:10C5DE00901D79E0FCA3E0FD2407128CDC128DCDBA
:10C5EE00FFED2408128CDCE024D0FDE434FFCD2FC7
:10C5FE00FFED35F0FEE4FCFD1227EA901D7B1229BB
:07C60E0099901D7B122981A8
:01C615002202
:06B5F000901BD212299904
:10B5F600901BD81229A500000000901BDC1229A57B
:10B6060000000000128D57901BD8122999128D57F1
:10B61600128DBFE47B3CFA901BE0128D5F901BDC21
:10B62600122999901BE0122981E47B3CFAF9F81261
:10B636002890128DBF901BD7E02406FF901BD6E002
:10B646003400FEC006C007901BE0128DACD007D0B8
:10B656000612B6AEE0FEA3E0FF2406F582E43EF550
:10B6660083743AF0EF2403FFE43EFEC006C0079061
:10B676001BDC128DACD007D00612B6AEE0FEA3E0FE
:10B68600FFF5828E83A3A3A3743AF0C006C0079089
:10B696001BD8128DACD007D0067D0312B12D901B9E
:07B6A600D6128D4E742CF04A
:0AB6AD00227D0312B12D901BD6225E
:0EFC5100EFC3941A5005EF2461FF227F632257
:0AFD1400900C387414F0900C40229B
:10A77100900D7FE0FEA3E0F5828E83E024526034E9
:10A7810024E26062146061244C600302A846900CCC
:10A7910061E0FF125BE4900D7B74FF75F0FE122700
:10A7A1009F85F082F583E0FFA3E0900D7FCF12A893
:10A7B1005C02A84C900D7FE0FEA3E0FD901BAAEE89
:10A7C100F0A3EDF0F5828E83A3E0FF900D7FE0FC16
:10A7D100A3E0F5828C83A312A851E475F007122738
:10A7E1009F12AA4280658038900D7BE0FEA3E0C3F2
:10A7F10094FEEE94FF5046900C61E0FF125BE490F2
:10A801000D80E02403FF900D7FE03400FE900D7B6E
:10A81100E475F0021227B585F082F583EE12A85C8B
:10A82100900D7FE0FCA3E0FDF5828C83A3E0FF8D1A
:10A83100828C8312A851EEF0A3EFF0800E12FD146A
:10A841007402F0800612FD147401F07F0602DCF33D
:10A85100A3A3E0FD12F9A3900D7F22F0A3EFF07FF7
:05A8610005125BE4227A
:10AA4200901E10EEF0A3EFF0127A1A901E10E0FCA6
:10AA5200A3E0F5828C83E0FEA3E07C002400FFECFF
:10AA62003E901BBCF0A3EFF0901BACE0122AC8AAE8
:10AA7200CC01AAD502AAD803AADB04AADE05AAE160
:10AA820006AAE907AAEC08AAEF09AAF20AAAF50B94
:10AA9200AAF80CAB2B0DAAFB0EAAFE0FAB0110AB52
:10AAA2000411AB0712AB0A13AB0D14AB1015AB13A9
:10AAB20016AB1617AB1918AB1C1AAB1F1BAACF1C6F
:10AAC200AAD21DAB221E0000AB2502F3BB02946486
:10AAD200029D5D02667E026AB802B1FE02DED2907B
:10AAE2001BADE0FF02A288027BCA02EFCF026CBE5E
:10AAF20002F8A702EE9602CE9402C6B002DFE80286
:10AB020063E402B39702E23F02FDF9026EC002FD66
:10AB12000A02D7AD02F001023C080290A7025E953C
:0AAB220002B9BB12FD147467F022A3
:10EECB005750005743005752002C000D00563F0D72
:10EEDB0000545400313000313200313100323100F6
:10EEEB003330003430003031003032003033004CDE
:05EEFB00490052440033
:10A581007AEE79D67BFF901D07122A2A7B017A0683
:10A59100799122901A54E0FF3395E0FEEF24D0FF29
:10A5A100EE34FFFE22540F2430FF901D821229F356
:10A5B100EF1226CE901D821229F30226337B017AF7
:10A5C1001C79EDE0FEA3E0FFEE3395E0FDFC901C6D
:10A5D1001EE4F0A32278917C067D017BFF022D927F
:10A5E1007A1C79ED7B01901D07122A2A7A0679914E
:10A5F10022901D83E475F00102279F901A9AE0FFD3
:10A60100E4FBFA7D492278917C067D017BFF22EFF4
:10A61100F0A3ECF0A3EDF0A3022A2A7B64901A9A2E
:10A62100E0FF7A007D5222901A99E06401227B01B9
:10A631007A1A7913022A2AE0FFA3E0FCA3E0FD22A3
:10A64100901C05E0FEA3E0FF22FE901D881229F375
:10A65100EE0226CE901C171229F3901C20E02290C6
:10A661001CE30229F3901A54E0D3648094B9229038
:09A671001C1A122999901C2222E6
:06BC8E00901C9112A610AB
:10BC940012E330EF4E7005FE7F0180047E007F00CA
:10BCA400901C9AEEF0A3EFF04E605312A61C12BA49
:10BCB40073901C9112A638901C971229F3901CE6DD
:10BCC400122A2A901C941229F312EAE2901C9AEE8A
:10BCD400F0A3EFF064024E60D8901C9AE0FEA3E05B
:10BCE400FF64034E60CBEF64044E60C5EF64054E01
:10BCF40060BFEF64064E60B912A5FC12BA73901CC3
:10BD04009AE07004A3E064097008901C9AF0A3748C
:10BD140005F0901C91E0FF64696009EF646A6004B7
:10BD2400EFB46B057F3212EC5712F90F901C9AE0B6
:04BD3400FEA3E0FF8B
:01BD380022E8
:06EAE200901CE012A610DA
:10EAE800901CE0E0FF12BBE2EF4E60012212A6602C
:10EAF800E94A4B600B12A66012E0F2EF4E60012269
:10EB0800901CE012A638901CE61229F3901A0B12FA
:08EB18002A2A12A66012B2CDF8
:01EB200022D2
:06B2CD00901A0512A61004
:10B2D30012F83C901A06E0F47003A3E0F4701F7AAE
:10B2E300EE79CB12A5D6901D8212A62F901A0B12BF
:10B2F30029F312E8C1901D0712A62F02B367901A13
:10B3030005E0FF64696005EF646A701A901A081219
:10B3130029F3E94A4B12A60760067AEE79CE800D2F
:10B323007AEE79D1800712A6077AEE79D1122D929F
:10B333007B017A1A790E901A0612A5C47404F012CE
:10B34300B4607A1A790E12A5E512D8F67AEE79D49A
:10B3530012A58512D8F6901A0B1229F3901D071225
:10B363002A2A7B017A06799112D8F612A58112D87E
:10B37300F612F92812A628600EA3E0FF12F0C7BF49
:10B3830045F27E007F092212A6664004E024C9F03C
:03B3930012A5946C
:01B396002294
:0B96BB00901BF6EFF0A3EDF0A3EBF026
:1096C600E4901C03F0A3F012E330EF4E7005FE7F2A
:1096D6000180047E007F00901C05EEF0A3EFF04EA3
:1096E60070030297A212A61C12BA73C3901C04E060
:1096F6009403901C03E064809480500512A5F580C5
:1097060008901C03E4F0A304F0901C03E0FEA3E021
:10971600FFEE7053EF24FE601214601D24027047A2
:10972600901BF6E0FF6430603E8009901BF7E0FF77
:1097360064306033901BF9800A901BF8E0FF6430B8
:109746006025A3E0FCA3E0FD901BFD1229F3901D0C
:1097560012122A2A901BFBE0FAA3E0FB12ECD1902E
:109766001C05EEF0A3EFF012A64164024E70030250
:1097760096F1EF64034E70030296F1EF64044E70A7
:10978600030296F1EF64054E70030296F1EF64064C
:109796004E70030296F112A5FC12BA7312A641EEA0
:1097A6007033EF24F7601B2409702A901C001229DD
:1097B600F3A801AC02AD037B017A1A7956122D92F9
:1097C6008013901C05E4F0A37405F0901C00122988
:0B97D600F3E41226CE12F90F12A64198
:0197E1002265
:0EECD100901D0EECF0A3EDF0A3EAF0A3EBF023
:10ECDF0012BBE2EF4E600122901D121229F3E94A96
:10ECEF004B600E901D121229F312E0F2EF4E6001ED
:0DECFF0022901D0EE0FEA312A63812D129AE
:01ED0C0022E4
:10E330009004017401F0901A98F012F83C7FFF12DB
:10E340005D517F5012EC577B0612A61E12BA737AEB
:10E35000EE79D812A5D612F92812A6286017A3E0E4
:10E36000FF12F0C7BF45F212F90F12A5FC12BA73E3
:0FE370007E007F092212A5FC12BA73E4FEFF2281
:10F90F00E4FF125D5112FB9912FBB9E4900401F070
:09F91F00901A98F07F0A02EC57DF
:10F83C00E4901A97F012FA5A9007AE1229F3E412D8
:0BF84C0026CE7BFF7AF6797602F3935C
:10F92800E4901A99F012A58D9007AE122A2A12F6C1
:09F93800769008DFE0F460F9228A
:10BBE200901E2FEFF012F83C12A6077AEE79DC12C3
:10BBF2002D92901E2FE0122AC8BC1A62BC2263BC8E
:10BC02002A64BC3265BC3A67BC4268BC4A69BC5211
:10BC12006ABC5A6B0000BC227BFF7AEE79DF804659
:10BC22007BFF7AEE79E2803E7BFF7AEE79E5803621
:10BC32007BFF7AEE79E8802E7BFF7AEE79EB802625
:10BC42007BFF7AEE79EE801E7BFF7AEE79F1801629
:10BC52007BFF7AEE79F4800E7BFF7AEE79F780062D
:10BC62007BFF7AEE79E212A58712D8F612A581122D
:10BC7200D8F612F92812A628600EA3E0FF12F0C728
:0CBC8200BF45F27E007F092212A594222B
:10E8C100901D7F122A2A901D7F12A5B8602FC412B5
:10E8D100A5A6D394394005740712267912A5F290A2
:10E8E1001D7F12A5B812A5A6D3943940057407124D
:10E8F100267912A5F2901D8012A5F580C9901D827E
:07E901001229F3E40226CE07
:06D6CB00901D85122A2AC1
:10D6D100901D8512A5B8FE6059D394394005EE24FA
:10D6E100C98008901D8512A5B824D012A64A901DA4
:10D6F10085E475F0011229FC122633C454F012A6F8
:10D701004A901D8512A5B8FED394394006EE24C96E
:10D71100FF800612263324D0FF901D8812A5B84F32
:10D721001226CE901D8912A5F5901D8612A5F5022F
:0CD73100D6D1901D881229F3E40226CE08
:06E0F200901BBE122A2A59
:10E0F80012F83C12A6077AEE79FA122D927B017A71
:10E108001B79C1901D82122A2A901BBE1229F31274
:10E11800E8C17B017A1B79C112A5E712D8F612A5CE
:10E128008112D8F612F92812A628600EA3E0FF1271
:0DE13800F0C7BF45F27E007F092212A594BA
:01E1450022B7
:0ED12900901CE9EEF0A3EFF0A3ECF0A3EDF004
:10D1370012F83C12A6077AEE79FD122D92901CE99F
:10D14700E0F47003A3E0F46030901CE912A5BE740C
:10D1570004F012B46012A5E112D8F67BFF7AEE79DB
:10D16700D412A58712D8F6901CEB12A5BE7402F054
:10D1770012B46012A5E112D8F612A58112D8F612E0
:10D18700F92812A628600EA3E0FF12F0C7BF45F2E8
:10D197007E007F092212A6664004E024C9F012A58A
:01D1A70094F3
:01D1A8002264
:06B46000901C17122A2ABD
:10B4660012A6701229A500000001901C2212298143
:10B47600901C1FE01425E025E0F9F8122954901CD1
:10B4860022122999E4901C20F0A3F0901C1EE0FEE5
:10B49600A3E0FFC3901C21E09FEE6480F8901C207F
:10B4A600E06480985069901C2212298D901C1A1213
:10B4B6002981122890901C26EFF0901C1A122981DF
:10B4C600901C2212298D122890AC00AD01AE02AF5D
:10B4D6000312A6701229817804122941901C2212A7
:10B4E6002999901C26E0FFD394094005EF24378064
:10B4F60006901C26E02430FF12A655FCA3E0F58238
:10B506008C83EF1226E0901C2012A5F502B491124E
:10B51600A655FEA3E0F5828E83E41226E07E007F28
:01B526000123
:01B527002201
:10D412002558000A002563002000253273002532BA
:10D422006275002531627500253478003030303065
:10D43200003532003139004158494F4D4500547290
:10D44200616E736D697474696E67004163636570C0
:10D4520074206D7367203F004D73672072656365AA
:10D4620069766564004C6F636B696E67203F00509C
:10D47200617373776F7264203F002A2A2A2A2A2A4C
:06D48200003230000C0036
:10E201004107B1014104010042040300004408C573
:0CE21100807F02004507A85C0D0D0D0089
:107F13007A0579107B01901CC7122A2A901CCAE4A7
:107F2300F0A32274C62FF582E43407F583E0FD8DB8
:107F3300F03395E090079812279F0F22E49007985B
:107F4300F0A3F07A0879C57B019007AE022A2A7A5A
:107F5300D4791C7BFF901B03122A2A7B01229005F4
:107F630008E0FE04F074092EF582E43405F583225B
:107F7300EFFD3395E0FC74712DF58274073CF583B6
:107F830022901B06022A2A7B017A0779C622901EB9
:107F930032E0FE04F074C62EF582E43407F5832242
:107FA300A3F07B017A0879CF227D017BFF022D921A
:107FB300E0FF901CC0E4F0A3EFF0901DB80229F39A
:107FC3007407F07A0779C6229004FA1229F312266D
:107FD30033FF22900797E02409F9E43405FA7B0183
:107FE300901CBD022A2A7D017BFF022D92E490079B
:107FF300CDF0FFFE227BFF7AD47920229008DDE0CA
:108003009007CDF0E4A3F0FFFE22901E30E0FF9036
:108013000408E09008CE229004FB75F00102279F2C
:108023007B017A0779B29004FA022A2AE0FFA3E0DF
:10803300900403CFF0A3EFF022540F2430900408F0
:10804300F0D3943922C3EF9DEC6480F8EE648098FA
:10805300227D017BFF022D929006747401F0E4905F
:10806300040922F583E0FDAC070F74C62C22901D92
:10807300A61229F3901DA92290050BE024CE227BA2
:10808300017A067908229008DB7430F0229008D038
:108093007433F0227B017A067980229008D07434FD
:0C80A300F0227402F07B017A0879D822E8
:109B3500901E30EFF0900401E0B40108901E30E073
:109B4500FF02DF8C901E30E0B4020312FBF8900890
:109B5500CEE024FE602B1460441460791470030277
:109B65009BF4147003029C0D24056003029C4B902A
:109B75001E30E064026003029C4B9008CE7402F034
:109B850022901E30E0FFB44211127F61EFF0900881
:109B9500CE7403F0900402EFF022029C15901E3063
:109BA500E0FF645C6017900402E02FF0900508E088
:109BB500C394FF5006127F61EFF022805390050891
:109BC500E02409127F6BE4F09008CE7404F0900451
:109BD50002E0F4F022900402E0C412803C4004E06C
:109BE5002407F012800DB507047405F02280249037
:109BF5000402E012803C4004E02407F012800DB519
:109C050007047406F022800B901E30E0640D600797
:109C15009008CE7401F0229008CE7407F090050AE2
:109C2500E0B43722A3E024CD60101460162403703D
:109C35001512F1E2EF4E600E80099008DAE0B431BA
:079C450005800012F79222D6
:10F676009008DF74FFF09007AE127FCE600D128700
:10F68600BC9007AFE475F00102279FE49008DFF015
:01F696002251
:10EAA100900798E0FEA3E0F4FFEEF4FE900798F0E3
:10EAB100A3EFF07BFF7AD47912901AD3122A2A900D
:10EAC1001AD6EEF0A3EFF07B017A0879C91237DC90
:10EAD1009008CBE09007A9F09008CCE09007AAF04D
:01EAE1002212
:10F7B00012EAA19008DFE0F460F97A0779A8127FD5
:0CF7C0004A12F6769008DFE0F460F922AF
:08E41D00901E12EFF0A3EDF0D8
:10E42500127F3F12F676901E12E09008D0F0901EF3
:10E4350013E09008D1F07A0879CF127F17127FC3C5
:10E4450012DA9B127FF0127F26BF00010EEF6407E0
:10E455004E70F39008DFE0F460F9127F8A127F4C6A
:06E4650012F67602F7B08A
:10F1E2007F037E0074CF2FF582E43408F583E0FDBF
:10F1F20074092F127F6BE06D6004E4FEFF220FBFE3
:0DF2020000010EEF64074E70DB7E007FFF01
:01F20F0022DC
:06CF1900901DA6122A2A59
:10CF1F00E4901DA9F0A3F0FDFF12A183128071E030
:10CF2F00FEA3E0FFF5828E8312264C602AEF641079
:10CF3F004E700312CF94128071E475F0011227B571
:10CF4F0085F082F58312264C901AD3F07BFF7AD4AA
:10CF5F0079171237E280C5901DA9E0FEA3E0FFC349
:10CF6F009410EE64809480501BEF64104E70031287
:10CF7F00CF947BFF7AD4791A1237E2901DA9E4126D
:04CF8F00801D80D3AE
:0BCF9300227BFF7AD479151237E222CE
:10F697007B017A06791912CF199008DB7431F09043
:10F6A70007B1E060057F01125CA07D317F3102E484
:01F6B7001D35
:0FFBE9009008DBE0B431077D347F3512E41D2234
:10F9410012807B60062402700C800712F1E2EF4EF8
:09F95100600602F69712FBE922A0
:10F633007D017F0F12A1839008DAE07BFF7AD479F2
:10F6430017901AD3B43004745F80027423F0123716
:02F65300E222B1
:10F0330012808212CF1912F633E4FF125CA09008FB
:10F04300DBE0B4311C90050BE024CF600D04700E9F
:10F053001280897D317F3102E41D1280892212FBE7
:02F06300E922A0
:10CC6900127F527A07799A127F847A1A79AE124C16
:10CC7900F3127F527A07799C127F847A1A79AB1260
:10CC89004CF3127F527A07799E127F847A1A79A817
:10CC9900124CF3127F527A0779A1127F847A1A799A
:10CCA900B2124CF3127F527A0779A3127F847A1A4F
:10CCB90079B5124CF3127F527A0779A5127F847ADB
:10CCC9001A79B8124CF37B017A1A799C12AF8390C6
:10CCD9001A9FE0FF70089007A07436F08007EF24D0
:0BCCE9002F9007A0F0E49007A7F022B6
:10BDE200127F3F12F676128090A314F012E55112E0
:10BDF2007FA5127F19740B12BE819007D1F0FFFE4E
:10BE0200127F26BF00010EEF640B4E70F39008DF25
:10BE1200E0F460F9127F8A127F4C12F67612CC6936
:10BE2200E4FEFF749A2FF582E43407127F2EBF00DE
:10BE3200010EEF640D4E70EB9008DFE0F460F97BC9
:10BE4200017A07799A127F4C12F6767B017A087989
:10BE5200DA127F19740412BE819007CAF0FEFF1233
:10BE62007F26BF00010EEF64044E70F39008DFE0FE
:0FBE7200F460F9127F8A127F4C12F67602F7B055
:0ABE8100F07A0779C612DA9BE4227A
:10D32100127F3F12F676128090127FA3127F19129C
:10D331007FC312DA9B127FF0127F26BF00010EEF2E
:10D3410064074E70F39008DFE0F460F9127F8A12EF
:10D351007F4C12F6767B017A0879DA127F19740410
:10D36100F07A07799A12DA9BE490079EF0FEFF7437
:10D371009A2FF582E43407127F2EBF00010EEF646D
:10D38100044E70EB9008DFE0F460F97B017A0779D5
:0AD391009A127F4C12F67602F7B0F4
:10D5E600127F3F12F6761280907437127FA3127F55
:10D5F60019127FC312DA9B127FF0127F26BF000139
:10D606000EEF64074E70F39008DFE0F460F9127FC6
:10D616008A127F4C12F67612809712FADBAD07ACAF
:10D6260006E4FEFF128048501774802FF582E4341A
:10D6360006F583E0FB8BF0127F34BF00010E80E419
:10D646009008DFE0F460F9128097127F4C12F676AC
:03D6560002F7B028
:10E8320090050BE024CF601324FD601114601F14B7
:10E8420060261460252407702B801A800712F1E2DB
:10E85200EF4E602312D3219008DC7431F02212F1C2
:10E86200E2EF4E601202BDE2800712F1E2EF4E606B
:08E872000602D5E612FBE922C3
:10D2280012F67612809E7432127FA3127F19127F33
:10D23800C312DA9B127FFF127F26BF00010EEF6434
:10D24800084E70F39008DFE0F460F9127F8A127FCD
:10D258004C12F6767B017A06799112FADBAD07ACAF
:10D2680006E4FEFF128048501E74912FF582E434C4
:10D2780006F583E0FB3395E09007988BF012279F23
:10D288000FBF00010E80DD9008DFE0F460F97B013C
:0DD298007A067991127F4C12F67602F7B0FB
:10EB210012F67612809EA304127FA4127F19127F1F
:10EB3100C312DA9B127FF0127F26BF00010EEF6431
:10EB4100074E70F39008DFE0F460F9127F8A127FBC
:0DEB51004C12F67612F7B09008DA7430F02E
:01EB5E002294
:10F5A700127F3F12C1C8EF4E60159008DDE0B437F7
:10F5B700057430F080069008DDE004F002D22812CE
:03F5C700EB212213
:101FCF00127F3F12FB40EF4E600302D22812EB212B
:011FDF0022DF
:10ED0D00127F3F12F67612809EA37431127FA412E9
:10ED1D007F19127FC312DA9B127FFF127F26BF006D
:10ED2D00010EEF64084E70F39008DFE0F460F91205
:0BED3D007F8A127F4C12F67602F7B0BE
:10F6B8009008DBE0B4311812807B600A14600A24D9
:10F6C80002700902F5A7021FCF02ED0D12FBE92215
:108E17007AD47920127F567A1D7915127F847A05C4
:108E2700790E124CF3EF4E7003FEFF22127FF812F9
:108E37007F587A1D7916127F847A057910124CF3C0
:108E4700EF4E7003FEFF22901D16E0D3940C4003F3
:108E5700028F2D127FF8127F587A1D7917127F849F
:108E67007A057912124CF3EF4E7003FEFF22901D24
:108E770017E0D3941F4003028F2D7BFF7AD4792507
:108E8700127F587A1D7918127F847A057914124C4B
:108E9700F3EF4E7003FEFF22901D18E0FDD39406FA
:108EA7004003028F2DEDB40607E4901D18F08006ED
:108EB700901D18E004F0127FF8127F587A1D791977
:108EC700127F847A057915124CF3EF4E7003FEFF7B
:108ED70022901D19E0D394174002804A127FF8129E
:108EE7007F587A1D791A127F847A057917124CF305
:108EF700EF4E7003FEFF22901D1AE0D3943B400211
:108F07008024127FF8127F587A1D791B127F847A8A
:108F1700057919124CF3EF4E7003FEFF22901D1BCB
:108F2700E0D3943B4004E4FEFF227B017A05790CF1
:108F3700127F197402F07A0879D812DA9B781D7CAF
:108F47001D7D017B017A1D79157E007F0812260D94
:078F57001288827E007F01F9
:018F5E0022F0
:10F5600012F1E2EF4E60199008DAE0B43012127F27
:10F57000137404F07A0879D212DA9B7E007F01229C
:04F58000E4FEFF2284
:10DC920012FB9912FBB990050CE024CD602C1460A4
:10DCA2002114601614600B147028901E317402F057
:10DCB2008025901E317403F0801D901E317404F093
:10DCC2008015901E317405F0800D901E317406F09F
:10DCD2008005E4901E31F0901E31E0FF6007E4FB06
:10DCE2007D0112872E12FA5A7BFF7AF6797602F3B9
:01DCF200939E
:10CCF4007F417E07127F68E06422701E0EEEC394AB
:10CD0400E6500B127F68E0642260030E80EFEEC3EE
:10CD140094E6400302CD690E80DA127F73E4F012C8
:10CD24007F68E0B5070F127F73E004F00EEEC39442
:10CD3400E640EC8030127F68E0FD6440602B0FEF2A
:10CD4400B50507C3648094D440028019127F73E44C
:10CD5400F0127F68E0B507DD127F73E004F00EEE99
:10CD6400C394E640ECE4FEFF220F127F7374FFF0DD
:0ACD74000E900797EEF07E007F019D
:01CD7E002292
:06C07F00901DB8122A2AF0
:10C08500127FCB700512801A80F6EFB4FF0612807E
:10C09500237F03229007ADE07007127FBDE41226CF
:10C0A500CE127FCB9007ADE0FEC3EF9EFF901DBB88
:10C0B500F0900400E0FEEFD39E503F127FD6901D16
:10C0C500BB127FB312003A127FCB127FBD8F8275F0
:10C0D5008300E41226E0901DBBE0FF900797E02F58
:10C0E500F0900400E0C39FFFF0E49007ADF01280EC
:10C0F5001AEF70037F01227F0222127FD69004007F
:10C10500127FB312003A127FBD900400E0FFF58262
:0EC11500758300E41226E09007ADEFF07F0086
:01C1230022F9
:1074B6007BFF7AD4792A127F587A1D79BC127F8491
:1074C6007A05790C124CF3901DBCE0FEA3E0FFC3D5
:1074D60094FFEE94004038EF94FEEE94FF50309007
:1074E6000403E0FEA3E0FF901DBCE0FCA3E0FDB5B5
:1074F6000707ECB5060302766FEDF44C6011901D9C
:10750600BEECF0A3EDF0901DBC74FFF0A314F09058
:107516001DBCE0FEA3E08EF0122AEE756500007534
:10752600720010757F0020758C00307599004075CB
:10753600A6005075B2006675B7006775D900687504
:10754600DF006975E2006A75EE007075F1009376EA
:107556000100FF763FFFFE765DFFFF0000767412A6
:107566007F137410F07A0679080275FB127F137484
:1075760010F07A0679190275FB127F137410F07AEF
:1075860006792A0275FB127F137410F07A06793B8E
:107596000275FB127F137410F07A06794C0275FBA4
:1075A600127F137410F07A06795D804912805B8031
:1075B6001A900674E0B4011878097C047D017B01F9
:1075C6007A057910122D92E4900674F0FE7F01225E
:1075D60002767412DC3012F09602FD3C127F1374B0
:1075E60006F07A067978800D02766F127F13741092
:1075F600F07A06798012DA9B02766F12CCF4EF4E9F
:107606007003FEFF229008E074FFF0128023E490DE
:1076160007ADF01276789004FA1229F312A866EFF5
:107626004E7003FEFF2212AEAEEF64014E60028082
:107636003D901DBC12802F80309007977407F07B19
:107646000112767812AEAEEF64014E6002801F9092
:107656001DBE12802F80129008E0E0B4FF0BE4F00C
:10766600900403F0A3F002D6597E007F0122E4FEC7
:01767600FF14
:10767700227A05790912FADB900797E0FEC3EF9E9D
:05768700900400F02258
:10DBCE009008DBE06431704F12807B601914602383
:10DBDE001460332403703D128E17EF4E6002800DD9
:10DBEE007D357F35802B12F560EF4E60347D317FB1
:10DBFE0031801E7B017A05790C1252EBEF4E6021BB
:10DC0E007D317F31800B1274B6EF4E60147D317F03
:10DC1E003102E41D02FBE990050BE0B4390312DC7E
:02DC2E00922240
:09FD4500E4FB7D017F0502872E1D
:10F7920012FB9912FBB9C2B17F0512EC57D2B1121A
:0EF7A200FD4512FA5A7BFF7AF6797602F39350
:10F2100090050AE024CE601114601124FB601014E4
:10F2200060102408701602F94102F03302E832023D
:0DF23000F6B89008DAE0B4300312DBCE220D
:10E37F009008CF7450F07BFF7AD4792E127F1974E6
:10E38F0004F07B017A0879D212DA9B7BFF7AD47979
:10E39F0033127F197402F07B017A0879D612DA9B57
:10E3AF007BFF7AD47936127F191280A512DA9B90EF
:0FE3BF0008DA7430F0A3F0A3F0A3F0E4A3F02287
:10DE140078087C067AD47939127FAC78197C067A32
:10DE2400D47940127FAC782A7C067AD4794D127F5B
:10DE3400E9783B7C067AD4795A127FE9784C7C06DF
:10DE44007AD47967128054785D7C067AD479711219
:10DE5400805412805BF078787C067D017BFF7AD455
:0FDE6400797C122D9290067F7430F0E4A3F022A7
:10E55100901A9CE0700F7BFF7AD47983127F191295
:10E5610080A512DA9B7B017A1A79A8127F197406A9
:10E57100F07A0479FD12DA9B9008D8E0900503F057
:10E581009008D9E0900504F0901AAEE0900505F0EE
:0CE59100901AAFE0900506F0E4A3F02221
:0FFBF800E49008DFF0900508F09008CE04F022AA
:10F9BA007F0512DD549008CEE0B4070612F2101249
:07F9CA00FBF87F0502DCF3EE
:10E46B0012F7E812FD287B017D147F0912E6337B3E
:10E47B00FF7AD479861237E2E4FF125DC5128082EF
:10E48B0012CF1912F633E4FF125CA09008DC743043
:10E49B00F09007AE1229F3E41226CE12FD4512FAC4
:0DE4AB005A7BFF7AF6797612F39302FBF8A4
:0DFC7A0012FB9912FBB912F7E812808922E3
:10F9730012E37F12DE1412F7CC900790E0600612B8
:08F98300E59D12E99602FD4525
:0FFC0700EF9008DAB4FF047431F0227430F02269
:10C44300901DABEEF0A3EFF0A3122A2A901DAD12BC
:10C4530029F312FADBD3EF9410EE64809480400248
:10C463008071901DABE0FEA3E0FFEE7066EF122A31
:10C47300C8C49300C49910C49F20C4A530C4AB4062
:10C48300C4B150C4B766C4BF6AC4C5930000C4D660
:10C4930078087C06803078197C06802A782A7C0606
:10C4A3008024783B7C06801E784C7C068018785D5F
:10C4B3007C0680129006747401F0801B78787C06E9
:10C4C300800478807C067D01901DAD1229F3122D26
:0CC4D300928004E4FEFF227E007F012224
:10D57200EE706AEF122AC8D59B00D59F10D5A6205F
:10D58200D5AD30D5AF40D5B650D5BD66D5CD67D572
:10D59200D46AD5DB930000D5DF128082227B017A28
:10D5A200067919227B017A06792A2280177B017A71
:10D5B20006794C227B017A06795D22900674E0B4EA
:10D5C200010280197B017A06793B227B017A047978
:10D5D20009227B017A06797822128097227B007ACF
:04D5E20000790022AA
:04000E00127FA52296
:10F7CC007E007F807D00127F8A122F59127F8A90D3
:0CF7DC000791122A2A7A0779900297E21E
:10E59D00E4901E32F012F7CCE4FF127F91E0FE748E
:10E5AD00D22FF582E43408F583EEF00FEFB404EAD0
:10E5BD00901E32E0FF04F074C62F127F9BE090088E
:10E5CD00DDF0E4FF127F91E0FE74082FF582E43454
:0AE5DD0006F583EEF00FEFB478EAC4
:01E5E7002211
:10DC3000E4FFFE74D22EF582E43408128066127F6F
:10DC40009BEDF00EEEB404EB9008DDE0FEAD070FA7
:10DC500074C62D127F9BEEF0E4FE74082EF582E46C
:10DC60003406128066127F9BEDF00EEEB478EB1254
:10DC70007F8A900791122A2A900790747DF0785E2F
:10DC80007C1D7D017A0779907E007F0412260D02AB
:02DC9000BE8B49
:10FA5A00128721901DC3E04401F054F9F012871B6C
:06FA6A00128718D29C2255
:10FB9900901DC3E04402F054FEF0C269128713229B
:10FBA900901DC0E0A3E0FAA3E0F9122B1BC2992231
:10F39300901DED122A2A128721901DED1229F39058
:10F3A3001DC0122A2A901DC3E04408F054EFF0D286
:08F3B3006A12871812FBA9225F
:10FBB900901DC3E04410F054F7F0C26A1287132273
:08FD8400901DC3E04404F022CD
:0BFCE900901DC3E0FE54FBF0AF0622AC
:10FB5300C269C26AE4901DC3F0FB7D017F05128771
:02FB63002E2250
:0CFCBA001F1C1F1E1F1E1F1F1E1F1E1FD1
:04E21D00411A9B0007
:10B8420090000612264C0475F03C84900006E5F048
:10B852001226E090000612264C600302B900900006
:10B862000512264C0475F03C84900005E5F0122682
:10B87200E090000512264C600302B9009000041209
:10B88200264C0475F01884900004E5F01226E0902E
:10B89200000412264C706790000312264C0475F0C7
:10B8A2000784900003E5F01226E090000112264C76
:10B8B200FF90FCB993FEEFB40208122633540370D2
:10B8C200010E90000212264CC39E50099000027491
:10B8D2000112269B2290000274011226E0900001C0
:10B8E20012264C75F00C84E5F0049000011226E05B
:0FB8F20090000112264CB4010574011226792230
:10C26800901AA6E0FF7B067A007D5212BA73E4901A
:10C278001AA7F0901ABC7442F0C2AF1283927FA240
:10C288001282C175351A7536BF787FE618F60536FD
:10C29800E536AE357002053514F5828E83E0FF125F
:10C2A80082D7901ABCE064456040901AA6E0FF125D
:10C2B800F0C7BF4511128392901AA7E0FD7B067A5A
:10C2C800007F6312B901787E16E67008901ABC7474
:10C2D80045F080CE0536E536AE357002053514F5E5
:10C2E800828E83E0FF1282D780B81282AB128392CB
:10C2F800D2AF901AA6E0FFE4FBFA7D4912BA732286
:10F26A00901E14EFF0A3EDF01283927FA21282C1D6
:10F27A00901E14E0FF1282D7901E15E0FF1282D76B
:0CF28A001282AB1283927F0512EC572217
:10FB77007D04E4FF12F26A7D807F0812F26AC26F89
:01FB8700225B
:1083DF00C26F901CA4E0FF64546018EF64446013F4
:1083EF00EF6457600EEF644E6009E4FBFAFD7F44C3
:1083FF0012B901901CA4E024BC601424F660202460
:10840F00F760142403701E901CA57490F0801690D2
:10841F001CA574B0F0800E901CA574A0F08006907F
:10842F001CA57480F0901C9DE014D3940B40047F26
:10843F000180027F00901C9CE0D3946340047E0176
:10844F0080027E00EE4FFF901C9EE014D3941E40DE
:10845F00047E0180027E00EE4FFF901C9FE0D394BC
:10846F000640047E0180027E00EE4FFF901CA0E0CC
:10847F00D3941740047E0180027E00EE4FFF901CC4
:10848F00A1E0D3943B40047E0180027E00EE4FFFBB
:10849F00901CA2E0D3943B40047E0180027E00EE4C
:1084AF004F600AE4FBFA7D017F3312B901901ABFC6
:1084BF007408F0901CA5E0901AC0F0E4A3F0901C93
:1084CF00A2E0FF75F00A84FEC454F0FEEF75F00AC7
:1084DF0084E5F04E901AC2F0901CA1E0FF75F00AEF
:1084EF0084FEC454F0FEEF75F00A84E5F04E901A46
:1084FF00C3F0901CA0E0FF75F00A84FEC454F0FE98
:10850F00EF75F00A84E5F04E901AC4F0901C9EE0CF
:10851F00FF75F00A84FEC454F0FE901C9CE05403D7
:10852F00FDC4333354C04EFEEF75F00A84E5F04EB0
:10853F00901AC5F0901C9DE0FF75F00A84FEC4549C
:10854F00F0FE901C9FE0FDC43354E04EFEEF75F03B
:10855F000A84E5F04E901AC6F0787E760808760801
:04856F0012C26822AA
:0BFCF400306F05C26F7F01227F0022ED
:10EF6900901E16EFF01283927FA21282C1901E1694
:10EF7900E0FF1282D77FA21282CC128344901E171F
:10EF8900EFF01282AB1283927F0512EC57901E1795
:03EF9900E0FF2274
:10FA7000E4FF12EF69EF5406FFBF0609D26F7D0461
:06FA8000E4FF12F26A220D
:10F8C100EF75F00A8424301226CEEF75F00A84E534
:0AF8D100F024309000011226E0221E
:10D96100901AA0E0FF7B017A1A79B212F8C1901ADD
:10D97100A1E0FF7A1A79B512F8C1901AA2E0FF7AF4
:10D981001A79B812F8C1901AB4743AF0901AB7F033
:10D99100E4901ABAF0901A9EE0FF7A1A79A812F868
:10D9A100C1901A9DE0FF7A1A79AB12F8C1901A9CC6
:10D9B100E0FF7A1A79AE12F8C1901AAA742FF0908A
:09D9C1001AADF0E4901AB0F02256
:10F2C100901ABFEFF01283927FA21282C175351A94
:10F2D1007536BF0536E536AE357002053514F58253
:0BF2E1008E83E0FF1282D7128392227E
:10CD7F00EFD39410400302CE09787EEFF608F61237
:10CD8F008392901ABC7442F07FA21282CC75331A30
:10CD9F007534BF1282EE0534E534AC3370020533BF
:10CDAF0014F5828C83EFF0901ABCE06445604578EF
:10CDBF007E16E670057445F080ED787EE6D394011B
:10CDCF0040161282EE0534E534AC3370020533148D
:10CDDF00F5828C83EFF080CF1283970534E534AC66
:10CDEF00337002053314F5828C83EFF0901ABC7404
:0BCDFF0045F080B31282AB1283922239
:07FDBC00901ABBE024FF22B6
:06FDFF007F0412DCF32278
:10F23D00901AC2E0FFC4131354037020901ACFE04C
:10F24D00B40319901AB1E0C394605006E02404F0A1
:0DF25D008005E4901AB1F0E4901ACFF02281
:10888200901D1EE014D3940B40047F0180027F00F0
:10889200901D1DE0D3946340047E0180027E00EEB1
:1088A2004FFF901D1FE014D3941E40047E018002EE
:1088B2007E00EE4FFF901D20E0D3940640047E011F
:1088C20080027E00EE4FFF901D21E0D394174004FA
:1088D2007E0180027E00EE4FFF901D22E0D3943B8A
:1088E20040047E0180027E00EE4FFF901D23E0D304
:1088F200943B40047E0180027E00EE4F600AE4FB5E
:10890200FA7D027F3312B901E4901ABFF0A3740416
:10891200F0E4A3F0901D23E0FF75F00A84FEC45436
:10892200F0FEEF75F00A84E5F04E901AC2F0901D49
:1089320022E0FF75F00A84FEC454F0FEEF75F00ADF
:1089420084E5F04E901AC3F0901D21E0FF75F00A05
:1089520084FEC454F0FEEF75F00A84E5F04E901ADE
:10896200C4F0901D1FE0FF75F00A84FEC454F0FEAF
:10897200901D1DE0FD5403FCC4333354C04EFEEF82
:1089820075F00A84E5F04E901AC5F0901D1EE0FFC6
:1089920075F00A84FEC454F0FE901D20E0FBC4333F
:1089A20054E04EFEEF75F00A84E5F04E901AC6F0E0
:1089B200ED1313543F25E025E0901AB1F0901ACF41
:1089C200ECF0787E760808760812C268789C7C1AE9
:1089D2007D017B017A1D791D7E007F0812260D1212
:1089E200D96112FDFF901ABB74FFF0E4901ABDF03A
:0189F2002262
:10AF8300901DF0122A2AC2AF7F0212F2C17F05126E
:10AF9300CD7FD2AF12F23D901ABFE0FFC4540F75BC
:10AFA300F00AA4FEEF540F2EFF901DF01229F39028
:10AFB3000006EF1226E0901AC0E0FFC4540F75F0AC
:10AFC3000AA4FEEF540F2E9000051226E0901AC13A
:10AFD300E0FF5430FEC4540F75F00AA4FEEF540F83
:10AFE3002E9000041226E0EF5440FFC413135403C1
:10AFF3009000071226E0901AC2E0FF5430FEC454BA
:10B003000F75F00AA4FEEF540F2E9000021226E0F3
:10B01300EFC413135403FF901AB1E02F1226CE90FE
:10B023001AC3E0FF5410FEC4540F75F00AA4FEEFD8
:10B03300540F2EFE901DF01229F3900001EE1226FC
:10B04300E0EFC41354079000031226E012FDFFE45F
:05B05300901ABDF0227F
:10A07C00901ABFE0FF540FFE4430901AB9F0EFC4B1
:10A08C00540FFD4430901AB8F0ED75F00AA42E90E0
:10A09C001AA2F0901AC0E0FF540FFE4430901AB68A
:10A0AC00F0EFC4540FFD4430901AB5F0ED75F00A82
:10A0BC00A42E901AA1F0901AC1E0FF540FFE443068
:10A0CC00901AB3F0EF5430FFC4540FFD4430901A83
:10A0DC00B2F0ED75F00AA42E901AA0F0901AC2E01E
:10A0EC00FF540FFE4430901AA9F0EF5430FFC454C3
:10A0FC000FFD4430901AA8F0ED75F00AA42E901ABA
:10A10C009EF0901AC3E0FF540FFE4430901AACF04E
:10A11C00EF5410FFC4540FFD4430901AABF0ED75A2
:10A12C00F00AA42E901A9DF012F23D901AC2E0FF94
:10A13C00C413135403FF901AB1E02FFD901A9CF036
:10A14C0075F00A84E5F04430901AAFF0AF05EF7566
:10A15C00F00A844430901AAEF0901AC1E05440FFDB
:10A16C00C413135403901AA3F0901AC3E0FFC41342
:07A17C005407901A9FF02226
:1080AF00901A9BE07006206903306A5DC2AF901A88
:1080BF00A4E0FEA3E0FF7880E6FC08E6FDC39FFF87
:1080CF00EC9EFED2AFC3EF9414EE94004031C2AFDA
:1080DF00901AA4ECF0A3EDF0D2AF7B017A1A799C41
:1080EF0012B84212D961901ABEE00475F03C84E5D3
:1080FF00F0F012F5847D117C007F0412CF9E227D5B
:10810F00017C007F0412CF9E22901ABF7402F09060
:10811F001ABDE0FFD39405400BEFFB7A007D017F82
:10812F005812B901C2AF1283927FA21282C15009B5
:10813F00901ABDE004F0D2AF2275351A7536BF051F
:10814F0036E536AE357002053514F5828E83E0FFC5
:10815F001282D75009901ABDE004F0D2AF221282DA
:10816F00AB787E7605087605128392E4901AA7F015
:10817F00901ABC7442F07FA21282CC5009901ABDA3
:10818F00E004F0D2AF22E4901ABDF075331A7534C3
:10819F00BF787FE618F61282EE0534E534AC337003
:1081AF0002053314F5828C83EFF0901ABCE064451E
:1081BF006045787E16E670057445F080ED787EE6B2
:1081CF00D3940140161282EE0534E534AC337002BD
:1081DF00053314F5828C83EFF080CF12839705342B
:1081EF00E534AC337002053314F5828C83EFF090D5
:1081FF001ABC7445F080B31282AB128392901ABEF0
:10820F00E0FFA3E06F60277D117C007F0412CF9EFB
:10821F00901ABFE0901ABEF012A07C7880E6FF089B
:10822F00E6901AA4CFF0A3EFF012F58480097D0138
:0A823F007C007F0412CF9ED2AF2214
:10FAF000E4901ABBF0128392E4FFFE12DB6A901AC4
:04FB0000A6EFF0225A
:10F8DB007B017A1A799C12AF8312D961901ABFE01F
:0AF8EB00901ABEF0E4901ABDF0225E
:10F9D100781D7C1D7D017BFF7AFD79AC7E007F085F
:07F9E10012260D128882229C
:10933000901D8B122A2AED644D600AE4FBFA7D022F
:109340007F4312B901901D8B1229F3E41226CEFE41
:109350007F80FD7B017A187952122F59C2AF7FA40A
:109360001282C1E4FF1282E67FA41282CCE4901D37
:109370008EF01282EE901D8EE02452F582E43418B5
:10938000F583EFF0901D8EE004F0E0C3947F40E29F
:10939000128344901D8EE02452F582E43418F58344
:1093A000EFF01282ABD2AF7FFFE4901D8EF0901DE4
:1093B0008EE0FEC39480501974522EF582E4341866
:1093C000F583E06004E4FF8008901D8EE004F080E7
:1093D000DDEF60030294619018D0E0901D90F09052
:1093E00018D1E0901D8FF0E49018D0F0A3F07E1813
:1093F0007F527D7EFC12D81CAC06EC9018D0F0EFAA
:10940000A3F0901D90E0FF9018D0E06F7038901D91
:109410008FE0FF9018D1E0B5072C901D8B1229F337
:10942000900001122A3FA801AC02AD037B017A181B
:1094300079527E007F7E12260D901D8B1229F374C7
:109440007E1226CE801B7B007A007900C003C0020A
:10945000C001901D8B1229F3900001122A6F7F002A
:04946000227FFF2246
:10B058009018D2122A2A7E007F807D007B017A1800
:10B0680079D9122F597B017A1879D99018D6122AD2
:10B078002A7A1879D57D4D129330EF700302B12AE0
:10B088009018D5E0700302B12AA31229F390004466
:10B09800E41226E09018D61229F3E92430F9E43AAC
:10B0A800FA901CC7122A2A901CCAE4F0A3740CF068
:10B0B8009018D21229F312DA9B9018D21229F39021
:10B0C800000C74201226E07D2012F8209018D2126D
:10B0D80029F38F828E83E41226E09018D61229F382
:10B0E80090004312264CFF901959F012FC16500993
:10B0F800901959E02450F08023901959E0FF12F874
:10B10800725016901959E0FFC39441400CEFD39444
:10B11800465006EF2449F080037F0022901959E039
:05B12800FF227F002260
:10BE8B00901D5EE0D3947E4009E4FBFAFD7F4112E6
:10BE9B00B9017E007F807D007B017A187952122FC9
:10BEAB0059901D5EE0FF7E0078527C187D01A31235
:10BEBB0029F312260D7E187F527D7E7C0012D81C32
:10BECB00AD07EFEEFF9018D0F0A3EDF0E4901D64FA
:10BEDB00F0C2AF901D62F07FA41282C1901D62E090
:10BEEB0075F008A4FF1282DBE4901D63F0901D64D3
:10BEFB00E02452F582E43418F583E0FF1282D790E8
:10BF0B001D64E004F0901D63E004F0E0D39407405F
:10BF1B00DC1282AB7F0A12EC57901D62E004F0E05A
:08BF2B00D3940F40B2D2AF2203
:10E99600C2AFE4901E18F07FA41282C1901E18E048
:10E9A60075F008A4FF1282DBE4901E19F0E4FF1252
:10E9B60082D7901E19E004F0E0D3940740EF12824C
:10E9C600AB7F0A12EC57901E18E004F0E0D3940FC8
:05E9D60040C5D2AF2294
:1097E200901D91122A2AE41226CEFE7F80FD7B0173
:1097F2007A187952122F59C2AF7FA41282C1E4FFA4
:109802001282DB7FA41282CCE4901D94F01282EECD
:10981200901D94E02452F582E43418F583EFF09021
:109822001D94E004F0E0C3947F40E2128344901D53
:1098320094E02452F582E43418F583EFF01282ABFF
:10984200D2AF7FFFE4901D94F0901D94E0FEC3948C
:1098520080501974522EF582E43418F583E06004C6
:10986200E4FF8008901D94E004F080DDEF600302C5
:1098720098FE9018D0E0901D96F09018D1E0901DBF
:1098820095F0E49018D0F0A3F07E187F527D7EFC14
:1098920012D81CAC06EC9018D0F0EFA3F0901D96F5
:1098A200E0FF9018D0E06F7038901D95E0FF90189F
:1098B200D1E0B5072C901D911229F3900001122AD4
:1098C2003FA801AC02AD037B017A1879527E007F7A
:1098D2007E12260D901D911229F3747E1226CE80DF
:1098E2001B7B007A007900C003C002C001901D9169
:0F98F2001229F3900001122A6F7F00227FFF22BC
:10F95A007B017A18794512B0588F6CE56C70037583
:09F96A006C85901D01E56CF02292
:07FDC3007B017A187945224B
:1070C1000000102120423063408450A560C670E763
:1070D10081089129A14AB16BC18CD1ADE1CEF1EF0B
:1070E100123102103273225252B5429472F762D6B3
:1070F10093398318B37BA35AD3BDC39CF3FFE3DE5B
:10710100246234430420140164E674C744A4548502
:10711100A56AB54B85289509E5EEF5CFC5ACD58DAA
:10712100365326721611063076D766F6569546B452
:10713100B75BA77A97198738F7DFE7FED79DC7BCFA
:1071410048C458E5688678A70840186128023823A2
:10715100C9CCD9EDE98EF9AF89489969A90AB92B4A
:107161005AF54AD47AB76A961A710A503A332A12F2
:10717100DBFDCBDCFBBFEB9E9B798B58BB3BAB1A9A
:107181006CA67C874CE45CC52C223C030C601C4142
:10719100EDAEFD8FCDECDDCDAD2ABD0B8D689D49EA
:1071A1007E976EB65ED54EF43E132E321E510E7092
:1071B100FF9FEFBEDFDDCFFCBF1BAF3A9F598F783A
:1071C100918881A9B1CAA1EBD10CC12DF14EE16F1A
:1071D100108000A130C220E3500440257046606752
:1071E10083B99398A3FBB3DAC33DD31CE37FF35E6A
:1071F10002B1129022F332D24235521462777256A2
:10720100B5EAA5CB95A88589F56EE54FD52CC50DB9
:1072110034E224C314A004817466644754244405F1
:10722100A7DBB7FA879997B8E75FF77EC71DD73C09
:1072310026D336F2069116B0665776764615563441
:10724100D94CC96DF90EE92F99C889E9B98AA9AB59
:10725100584448657806682718C008E1388228A391
:10726100CB7DDB5CEB3FFB1E8BF99BD8ABBBBB9AA9
:107271004A755A546A377A160AF11AD02AB33A92E1
:10728100FD2EED0FDD6CCD4DBDAAAD8B9DE88DC9F9
:107291007C266C075C644C453CA22C831CE00CC131
:1072A100EF1FFF3ECF5DDF7CAF9BBFBA8FD99FF849
:1072B1006E177E364E555E742E933EB20ED11EF081
:10EB5F00AB07AA068B828A83E0FFECFEEF6D25E000
:10EB6F00FFEE33FE74C12FF58274703EF583E4938C
:10EB7F00FC740193FD8B828A83A3E0FEEC6EFFEDA4
:0EEB8F00AC02AD038D828C83CFF0A3EFF02299
:10D81C00901CA6EEF0A3EFF0A3ECF0A3EDF0E490D7
:10D82C001CAEF0A3F0901CAAF0A3F0901CA8E0FE94
:10D83C00A3E0FFA3E0FCA3E0FDC39FEC9E502F9060
:10D84C001CA6E0FEA3E02DF582EE3CF583E0FF7E06
:10D85C0000901CACEEF0FCA3EFF0FD7E1C7FAE1232
:10D86C00EB5F901CAAE475F00112279F80BD901C01
:0ED87C00AEE0FCA3E0FAEC2400FFE43AFE224A
:109F7400EF122AC89FD6019FDC029FE1039FE604EB
:109F84009FEB059FEE069FF8079FFB089FFE09A025
:109F9400010AA0040BA0070CA00A0DA00D0EA0102E
:109FA4000FA01310A01E11A02912A03413A03F1457
:109FB400A04615A04D16A05217A05718A06A199FC5
:109FC400D91AA06D1BA05E1CA0651D9FF31E000086
:109FD400A070D20822D20722D210D20822D20DD2E7
:109FE4000822D241D20822D20922D20ED20922D288
:109FF40046D20922D21A22D21922D20B22D20B2201
:10A00400D21D22D21E22D20C22D21122D20A22D254
:10A0140012D20AC217C216C21522D217D20AC21607
:10A02400C215C21222D216D20AC217C215C21222F5
:10A03400D215D20AC217C216C21222D213D20AC22F
:10A044001422D214D20AC21322D243D20A22D244F4
:10A05400D20A22D21CD20AC21B22D21CD20AD21B7E
:10A0640022D20FD20A22D21822D23122EFFB7A0056
:08A074007D017F3812B90122C1
:10ACF500EF122AC8AD5701AD6102AD6403AD67041B
:10AD0500AD6A05AD7106AD7707AD7A08AD7D09ADC4
:10AD1500800AAD830BAD860CAD890DAD8C0EAD8F64
:10AD25000FADA410ADA711ADAA12ADAD13ADB01402
:10AD3500ADB315ADB616ADB917ADBC18ADC519ADEA
:10AD45005E1AADC81BADBF1CADC21DAD741E0000A3
:10AD5500ADCBC210C20DC24122C20722C21022C20F
:10AD65000D22C24122C209C20EC24622C20E22C211
:10AD75004622C21A22C21922C20B22C20B22C21DAE
:10AD850022C21E22C20C22C21122C20AC212C2173C
:10AD9500C216C215C213C214C243C244C21C22C287
:10ADA5001222C21722C21622C21522C21322C214AF
:10ADB50022C24322C24422C21C22C21C22C20F222A
:10ADC500C21822C23122EFFB7A007D017F3912B908
:02ADD500012259
:10EB9D00EF122AC8EBBA01EBBD05EBC008EBCC09AF
:10EBAD00EBC30BEBC60CEBC90F0000EBCFD2002271
:10EBBD00D20122D20222D20322D20422D20522D2A3
:0EEBCD000622EFFB7A007D017F3A12B9012289
:10EBDB00EF122AC8EBF801EBFB05EBFE08EC0A0978
:10EBEB00EC010BEC040CEC070F0000EC0DC2002247
:10EBFB00C20122C20222C20322C20422C20522C2C5
:0EEC0B000622EFFB7A007D017F3B12B9012249
:10FA9C00307009901E33E0FF129F7422901E33E0E9
:05FAAC00FF12ACF52281
:10FAB100307109901E34E0FF12EB9D22901E34E05C
:05FAC100FF12EBDB2247
:10E90800C207C206C205C204C203C202C201C200D3
:10E91800C20FC20EC20DC20CC20BC20AC209C20883
:10E92800C217C216C215C214C213C212C211C21033
:10E93800C21EC21DC21CC21BC21AC219C218C244BE
:07E94800C243C241C23122AB
:10B52800901D65122A2AE4901D69F0901D6BF07435
:10B53800002531F582E43403F583E0901D6AF0902C
:10B548001D68E549F0901D6AE0FF20E749901D65F8
:10B558001229F3E92404F9E43AFA901D6BE07C001F
:10B5680029F9EC3AFAEF1226CE901D68E0FF901DFB
:10B578006AE0FEEF6E901D68F0A3E02EF0901D6B60
:10B58800E004F0E025312400F582E43403F583E09B
:10B59800901D6AF080AF901D651229F3E92404F923
:10B5A800E43AFA901D6BE0FF7C0029F9EC3AFAE4E2
:10B5B8001226CE901D651229F3900003EF1226E0A3
:10B5C800901D68E01226CE901D6BE0FF901D69E08B
:10B5D8002FFF901D651229F3900001EF1226E090CD
:08B5E8000002E5491226E022F1
:10F06500901E1CEFF07FFF12F8F5901E1CE0600A61
:10F07500901E1A7400F0A37400F07E1E7F1A1249C8
:10F0850004E433901E1DF012FD72901E1DE024FF56
:01F095002258
:0100220022BB
:104904008E838F82C083C082E0F513A3E0F5148503
:104914001383851482A3E0601FAC13AD147F1112BE
:10492400494950148E138F148C118D128A158B16CD
:10493400124A314004024913C3D082D083E513F0F4
:10494400A3E514F0228C838D82E58230E001A3E09C
:10495400A3AC83AD82605604600E3072F11249C07C
:10496400604B8C838D8250E6ECB55504EDB5540054
:1049740092287A007B00E06034047007E58230E01E
:104984001280083072051249CB4008A30BBB00010A
:104994000A80E3BA0006EBB5070040ADE555B583E0
:1049A40005E554B582008228409FD3800A124C68E2
:1049B400E07003124C68C3AE83AF8222B46400403B
:1049C400041249FA22C322B464004028F9E5822083
:1049D400E022BA0012BB0600500DC083C082E91267
:1049E40049FAD082D083229406F58250021583E9D5
:1049F4001249FE22C322C2D5800478FFD2D575F0B5
:104A04000A84FE75F00679FFE0A36020B50100502A
:104A140001F930D50A15F0E0A3B500005001F8D52E
:104A2400F0E6E930D50328C313B5060022C22012EC
:104A34000101202052C223120CC820234AC2211291
:104A440005E7202142C22512087E20253AC21F1202
:104A54000A39201F32C22612613D20262AC227129B
:104A64006140202722C224122FC120241AC23212EC
:104A74003451203212C2221210F120220AC24512ED
:104A84004A8D204502C322D322C24522EE8003EE82
:104A9400C3132E4005B507005006EF2E1304800201
:104AA40074FF22AA42AB45124BBF4011AA41AB444A
:104AB400124BBF4008854144854245C322D322128C
:104AC4004B0D4014AF4AAE4B124BA8400BF542AF0E
:104AD4004CAE4D124BA850028014F54110340DE534
:104AE4004C254C4007954A50037541FFC322D322FD
:104AF400C083C082758303853182F0302904053177
:104B040080021531D082D08322853883853982AEE4
:104B140007E4FAFBF54AF54CF4F54BF54DE0A3FC3C
:104B24002AFA50010BEC302C10B54A004002F54A29
:104B3400B54B005002F54B800EB54C004002F54CCD
:104B4400B54D005002F54DB22CDFD2EE124C10EAF6
:104B5400500104C53C600DFAAB3CAC5053040F1239
:104B64004BBF402CE550C4540FFAE53C8AF084B5A1
:104B74004B00501CB54D005017E53C8AF0A4C5F01D
:104B8400700CC5F0B54A004007B54C004002C32282
:104B9400D322F5F0C31325F04009C5F003030354F1
:104BA4001F25F022EE124B96400FB5070040047407
:104BB400FF8004EF2E1304C322D322EAC39B5002C6
:104BC400F404F5F0EA2B500713C5F0C313C5F0C580
:104BD400F06008C5F084B504004002C322D322204B
:104BE4002A0B855383855282E551F0801E858353B9
:034BF40085825265
:104BF7007AFFA3A3E0B502005001FADBF5855383E2
:104C0700855282E0F551EAF0227006F4FAFBD2D21F
:104C170022BB0008CAFD7C007E008018AC02FAE4C3
:104C2700CBFD7E08ED20E70CC3EB33FBEC33FCED4B
:104C370033FDDEF18AF0846017ADF02BFBBE00E494
:104C47008011D3EB33FBEC33FCED33C39AFDDED598
:104C5700BE00EFEAC313B50500AA03AB04EDC2D249
:0B4C6700220582D582021583158222EF
:102FC100A20C72315012851183851282AB15AA169B
:102FD100BB0006BA0D00500122851282851183853E
:102FE10012398511387406124C10B40137EAB44312
:102FF100005031F549D229753101D23A12306D5064
:103001001CC2290539E5397002053875315F74FF35
:10301100124AF412306D4051B46A4E800FB4670009
:103021004047800802306A12306D403D124AF4D5A3
:10303100491E30290DB46A3174FF124AF475310109
:10304100801AB467004022B46A00501D0531800C1B
:10305100E5392406F5395002053880CB1234024097
:10306100081233014003D22422022FD912308040AA
:103071000D1230D01231434005123168400022C296
:1030810047853883853982D236E0794BF775F0056B
:10309100A3800F853883853982E0F46030F4C3134F
:1030A10080E8E0203602C31309F719274008F70921
:1030B100A3D5F0EE80051036DA8012303A0DC23A0F
:1030C100E54C204704C313254CF54BC322D322758D
:1030D100F00B1230F67807ED7FFF801074FFF6E5F4
:1030E10046C395F0F546E5479400F5477002A646BC
:1030F10018B800E8227B00E54B254D50010B254F08
:1031010050010BFA8B478A46E5F0124C1050010A28
:10311100E547C313FDE54613FCEAF5F0232CFC500B
:10312100010D8C468D4722C000B50100400E78028A
:10313100F5F0E6B5F000500608B808F67800E8D0DA
:103141000022784BE6123128601BF608B850F5785A
:103151004B7903E6F70809B850F9202906EBCFFBB4
:10316100ECCEFCC322D322EB2D2FB40B212C2EB499
:103171000F00401AB415005015A2E09235EBC39C24
:10318100C39D2E240975F0038485F0488003023223
:10319100FFED141475F01FA4FAEE141475F009A4D0
:1031A1002A246FFAEC141475F01DA4F4042AFAEB26
:1031B100141475F006A4F4042AB4F10050D02403C9
:1031C100830232B64EFFFFFFFFFFFFFFC9FFFFFF84
:1031D100FFFFFFC3FFFFFFFFFFFFFFBEFFFFFFFF7B
:1031E100FFFFFF3BFFFFFFA8FFFF38EACBFFFF25F3
:1031F100FFFFA04F4AFF22FFFFB22F44FFFF57FFFF
:10320100FF2CFFFFFFFF9CFF5EFF4CFFFF99160B9A
:10321100FFFFC7FFFF01D488FFC1FFFF139085FFA8
:10322100FFE1FFFF8DCDD8FFFF39FFD1DB3C1DFF53
:1032310036B389E6301A92A99E5F0617DA825526BF
:103241002D0365B59411232AFF56D9640EFF5CFF47
:10325100FF9B6352FF68FFFF98150AFFFFC5FFFF41
:1032610000D387FFBFFFFF698F84FFFFFFFFFF8C44
:10327100FFE2FFFFFFFFD0FFFF3AFFFFFFA7FFFFC6
:1032810037B4BDFFFF24FFFF9F6048FF21FFFFB15F
:103291002E42FFFFFFFFFF2BFFFFFFFFFFFF5DFF41
:1032A100FFFFFFFFFF67FFFFFFFFFFFFFFC6FFFFFE
:1032B100FFFFFFFFC0F46046F4A23530E701B340E1
:1032C1003DC2E7FA75F00484240283801B40555502
:1032D1000000800000545505000208004655555570
:1032E100190000A800806A01C5F06008C5F0030359
:1032F10015F080F4E5F05403B54803EAC322D32264
:10330100C2347559007583038531827531647548FE
:1033110064C237C238C239E00582B46704D237804B
:103321000AB46804D2388003B4692DE00582B46719
:0E333100005062303725B440005005242002C1
:10333F0033C2B46000500424C08078B46202804964
:10334F00B46302804CB4645B804D0233F3303818A1
:10335F00B4600050042420805AB46202802BB463FE
:10336F0002802EB4653D8035B464005010FA75F0BC
:10337F000A8424301233F5E5F024308036B4640229
:10338F008015B4651E80168039D239B237B23880B5
:10339F008CC237C238801FC237D2388019C238D298
:1033AF00378013B46610203408E5597009D2348081
:1033BF0005741D1233F5303906C239B237B23802EF
:1033CF00332CB46A1FE559B44100501874BC123342
:1033DF00F7200C0530340D800675498030340375A5
:1033EF004981C322D3220559C082854882F00548FE
:1033FF00D08222758303853182754701E00582FAF9
:10340F000582E01582B46A028020E08547F0A4AB04
:10341F00F02A50010BFABB00028009C39467FA50DF
:10342F00011B80F20547058280D6EA75F06784E0BC
:10343F00B5F00D746AF005820582E0F47002C322C4
:10344F00D322301112851183851282AB15AA16BBB8
:10345F000006BA1F00500122851282851183851242
:10346F00398511387406124C10B401EBEAB44300DD
:10347F0050E5B4050040E0F549D229753101D23A43
:10348F001234F75017C2290539E53970020538751E
:10349F00314874FF124AF41234F74049B42F468072
:1034AF00080234F41234F7403C124AF4D54914B4EC
:1034BF002F3330290A74FF124AF475310180100539
:1034CF0031800CE5392406F5395002053880D512C4
:1034DF0036DF4011123626400CD232754990303407
:1034EF00037549912202346612350A400D12350FC9
:1034FF001235504005123575400022D247023082F6
:10350F0075F0091230F67806ED7EFF801074FFF625
:10351F00E546C395F0F546E5479400F5477002A6DA
:10352F004618B800E822C000B50100400E7802F539
:10353F00F0E6B5F000500608B807F67800E8D000BE
:10354F0022784BE6123535601BF608B850F5784BEC
:10355F007903E6F70809B850F9202906EBCFFBEC01
:10356F00CEFCC322D322EB2D2FB4090C2C2EB40D7D
:10357F00004005B411004003023624EE1414FAED96
:10358F00141475F004A42AFAEC141475F010A42A7C
:10359F00FAEB141475F040A42AF5487F00EF2412BB
:1035AF0083B54807EF240C830236220F0FBF60ED5F
:1035BF00023624032FA00005010A020F0350045501
:1035CF00055A060007A508F009400A450B4A0C905A
:1035DF000D950EE00F141019111E126413B414017F
:1035EF001506160B175118A119541A591B411C46D1
:1035FF001D911EA41F15201A2165227823522480A5
:10360F00258526D02716282929422A562B942C8126
:10361F002D692EC322D322755900758303853182FC
:10362F00753164754864E00582B42F56E00582B4A5
:10363F002F0774BC1236ABC322B42B005018B40A38
:10364F0000400C1236A050051236B6800424072411
:10365F00301236A980D6D234F8E00582C8B42B09CF
:10366F0012369F401D940980E8B42C0A12369F40F1
:10367F00111236C180DBB42D0B12369F4004241774
:10368F0080CFD322B42EFB12369F40F6245780C131
:10369F00C8B4240050ECB40A00220559C0828548F2
:0E36AF0082F00548D0822224DD83222D2E20B9
:1036BD00242F2B2524F783221B1C1D1E1F3B3C3D55
:1036CD003E3F5B5C5D5E5F7B7C7D7E7F0040607F0F
:1036DD007F7F7583038531827FFEE020E7040582BD
:1036ED0080F81582158275470175480279007A00B8
:1036FD00E0FE1582E0FDFAAF821582AC018547F040
:10370D0012375FA9040547E547B415004003754717
:10371D0001AC028548F012375FAA040548E548B4AC
:10372D00100040037548011582E0B42FCEE975F005
:10373D002F84EDB5F01AEA75F02F84EEB5F0117403
:10374D002F8F82F0058205820582E0F47002C3227C
:10375D00D322E0A4ABF02C50010BFCBB000280097E
:0A376D00C3942FFC50011B80F222D0
:10010100A208720D72417207400122851183851286
:1001110082AB15AA16BB0006BA1300500122851244
:10012100398511380ABA00010B740A124C106005A6
:1001310012057C40E8EAB44200505CB40300405729
:1001410014F54914F559755063307203755034D262
:1001510029D22A753101753C0075572A300703757C
:10016100572412021040301202BBB42A04F5578002
:100171003FB55702803A1210C1E54703F547120215
:10018100BBB42A04F5578003B5570CC22975315FFA
:1001910074BC124AF48019808412021040F91202D0
:1001A100BB60F4D549028014124AF4B5570280E7C6
:1001B100E539240AF5395002053880DDB557D830C4
:1001C100290A74BC124AF475310180020531E557E0
:1001D100B42A0280097549E9A207402E802D75498C
:1001E100101205CE5024D220300D0E1204172047D4
:1001F1001A304105120530501212033C400D120312
:100201009C754910303403754911C3B392202230D3
:100211002A0F7B03124BE3307207C333B551004001
:10022100737F09D22C124B0D406AE0FAE54DC313DE
:10023100B50200505F853982853883AF4AAE4B12D3
:100241004BA84050F542AF4CAE4D124BA84045F57E
:100251004112029F403E853883853982D22CE4FACF
:10026100FBF5437F09E0202C09B54100B3EA33FADD
:10027100800BB54200B350020543EB33FBA3B22C14
:10028100DFE38A478B462029081210C1E54703F5B1
:1002910047C38001D3302A05C22A124BE322AA4A5E
:1002A100AB4B75F0051210DE400CAA4CAB4D75F04E
:1002B100051210DE4002C322D322AB47EB30D079C6
:1002C100E5437007EBF4540FFB8021B4026B801CF3
:1002D100E54AB54C004006AC4CAD4A8004AC4AAD91
:1002E1004CECC3132C4005B50500404D7A00EBC31F
:1002F100134006CA240DCA80F6703EE546C2E42AC0
:100301002402838035244B52514F4E547E4D4C5321
:100311007E502F41484745444A7E4342497E462B01
:100321003138373534307E3332397E3625552E2DEE
:1003310059582A7E5756207E5AE4227A0075830343
:10034100853182E020E728800DE01203782A75F0DC
:100351002B84AAF005820582E0158230E7EBE012DA
:100361000378B5020AD23430000374BCF08002C2B3
:1003710034A234A000B322B441004003943722B424
:100381003000400394302224E1832226000000271C
:0D0391002A00000000002900242528C234A5
:10039E00301075758303754801853149854982E0B2
:1003AE00FA854882F020E75D0549854982E0FBB475
:1003BE004100404DB45B005048EAB42405EB24C024
:1003CE008033B42F05EB24E0802BB42B05EB2420D7
:1003DE008023B4252CEB24C183801A1B1C1D1E1FE9
:1003EE003B3C3D3E3F5B5C5D5E5F7B7C7D7E7F008C
:1003FE0040607F7F7F854882F005480549D2348072
:10040E009B0548809775310122C0A075A0037860C6
:10041E007A05E4F208DAFC758303853182E020E781
:10042E000505820A80F7BA06437F001582E0C39461
:10043E00304033240283802B00010203040506079B
:10044E000809FFFFFFFFFFFFFFFF0A0B0CFF0D0E5A
:10045E000FFF1011121314FF15161718191A1B1C63
:10046E001D1E1FB4FF0BD3D247D0A022C3C247809C
:10047E00F8604AFE7870E4F2087A047B07EF2B836B
:10048E00F2080BDAF88018000000010000003200BC
:10049E000010240003276801048576335544327D0D
:1004AE0005EE13FE500778647974120522DD028082
:1004BE000C7874797412052280E7020439EF240453
:1004CE00FFB418F67B057F0078607970E2FA54F07D
:1004DE0060178092E2FAC4540FFC2375F00A84254B
:1004EE00F02FD4FFEC4430F309EA540FBB0103FEA6
:1004FE008005FC2FD4FFEC4430F30908DBD6EF5413
:10050E000F6E600302047A7480F3C37531707549FF
:10051E00120204757A05C3E2FBE33BD4F21819DA32
:10052E00F6227A007B00758303853182E020E70F87
:10053E00B43A005037B43000403205820A80EDBA2A
:10054E00072A1582E0540FFC8531827A02E0540F9F
:10055E008AF0A42BFB05820ABA08F275F00B84E52B
:10056E00F0B5040874BCF0C375491322D322FF12F0
:10057E0005B0502AE004700DA3A31F1F8582398594
:10058E008338EF6019C083C082E514142582F5828A
:10059E00E5833400F583E0D082D083047002C32259
:1005AE00D322C083C082851383851482124C68E0E7
:1005BE00D082D083B4FF071F1FBF0002C322D322F5
:1005CE00758303853182E0B4240D7800A308E030F2
:1005DE00E7FAB80302C322D32230091285118385AC
:1005EE001282AB15AA16BB0006BA11005001228565
:1005FE001282851183740A124C10B407F1EA23F5A6
:10060E0049B441005061F55975506430720375500C
:10061E0046D22AC22F2072077B04124BE380057B41
:10062E000D1210ABC22AA3A3A3A3858239858338EA
:10063E00753C00D234D22C12077540288541448572
:10064E004245851239851138D22C7F0412074C850C
:10065E008239858338124BE3BC000FD229753101E4
:10066E00D22C8020124BE30205FC53040EBC02F781
:10067E00C22975315F74BC124AF4C22CE53970027E
:10068E001538153912077B40DE858239858338157A
:10069E0049D549F0D234753C00D22C7F0320290471
:1006AE007F04C22C124AC340BE853982853883D25C
:1006BE002C7F0375F004202907C22C7F0475F000EF
:1006CE0012074CE5F0B5049F30290A74BC124AF4A7
:1006DE0075310180020531302F0A20011FE559B412
:1006EE0002158018300105120817400812070D3048
:1006FE0047055006020675754920D221C22F22E504
:0E070E0059B40E31300E10A83175A003E275FB
:10071C00A000B43004C23C8005D23C304619200104
:10072C0005120817400EECF0754922203C050531E6
:10073C00754921C3D24722C247227C08124AA722FC
:10074C00853982853883E4FAFBFCE0A3302C09B5AB
:10075C004200B3EA33FA8007B54100B3EB33FBA296
:10076C00E0EC33FCB22CDFE2227F0A124AC32212E5
:10077C000775407430721F20290FE559B549028066
:10078C000D1414654960078008E549B402038541DE
:10079C004412074640528539828538837F0A1207F6
:1007AC004C8A468B472029071210C1AA47AB46EA50
:1007BC001207F65013202F3020292DBA002AE559A4
:1007CC0065497024D22F8003124AF4EB1207F650BD
:1007DC0012202F14302911BB000EA849B80209D2DF
:1007EC002F8003124AF4C322D32220D01C541E03A0
:1007FC0024028380100037343032393600313835DA
:10080C0000330000006002C322D3227A007B007503
:10081C008303853182E020E7570582E030E7FA1543
:10082C0082AD82E0FC1582E0C394302BFBE531B540
:10083C008202800D1582E0C394302AFAE531B5822C
:10084C00E4EB75F003A42AFAE435F0600BFBEA2420
:10085C0006FA40011BEB70F6EA75F00A84E5F060CD
:10086C0003F4240B2430B504078D8274BCF0C3222E
:10087C00D322301A12851183851282AB15AA16BBAE
:10088C000006BA1500500122C236851282851183EA
:10089C00740A124C10B40704D2368004B401E81A5E
:1008AC00EAF549B441005077F5597550643072033C
:1008BC00755046303611D22A2072077B04124BE356
:1008CC0080057B0D1210ABC22A8582398583387561
:1008DC003C00D22C3036051209CB80031209CF40D4
:1008EC0038854144854245851239851138D22C7F93
:1008FC00063036027F0412074C85823985833830E6
:10090C003608BC001D124BE3800653043EBC281A6B
:10091C00D229753101D22C802B303603124BE302D5
:10092C00089353040EBC02F7800653043FBC22EF1D
:10093C00C22975315F74BC124AF4C22CE5397002BD
:10094C00153815391209FB40D6858239858338D57F
:10095C0049F2D22C30360C753C007F0320290D7FD8
:10096C000480077F052029047F06C22C124AC3404D
:10097C00AE853982853883D22C30360F7F0375F0E3
:10098C00042029167F0475F000800D7F0575F01189
:0D099C002029077F0675F005C22C12074CBC
:1009A900E5F053041FB50402800302089330290AB5
:1009B90074BC124AF475310180020531D22575499A
:1009C90030227F0C80027F0A124B0D4061AF4AAE84
:1009D9004B124BA84058F542AF4CAE4D124A93F515
:1009E90041B4FF0CE54CB54A005043E54C04F541D0
:1009F900C3221209CF403730720885414412074695
:100A0900402C8539828538837F0A12074C8A468BA8
:100A1900472029071210C1AA46AB47BB0002800331
:100A2900BB010BEA1207F64005124AF4C322D3228E
:100A3900301912851183851282AB15AA16BB0006DF
:100A4900BA1100500122C2360ABA00010B7406120B
:100A59004C1070F1EA1414F549B44100504EF5599F
:100A6900755064307203755046C22A851239851152
:100A790038753C00D22C120B5640318541448542D1
:100A890045851239851138D22C7F0612074CD22C94
:100A990085823985833853043EBC20028005BC0C0D
:100AA9000ED236D229753101D22C801C020A4EBCD5
:100AB90002028005BC18F5D236C22975315F74BCB3
:100AC900124AF4753C00D22C120BAA40DF858239F8
:100AD900858338D549F2D22C753C007F05120B5815
:100AE90040CA3072077C02124AA740C0D22C7F0547
:100AF90075F01030360375F006202910120B4DC21F
:100B09002C7F0675F00130360375F00C12074CE5A1
:100B1900F053041FB5049530290A74BC124AF475C0
:100B290031018002053130020F20360712081740C3
:100B3900128005120C3E400BD21F75494030360316
:100B490075494122E539700215381539227F051298
:100B59004B0D4038AF4AAE4B124A93F542AF4CAEFB
:100B69004D124A93F541E5425541B4FF1AE54CB59A
:100B79004A005007E54B04F542801FE54D14F54145
:020B8900E54A3B
:100B8B0004F5428018E542B4FF02804BE541B4FF07
:100B9B000CE54CB54A00503FE54C04F541C322D25D
:100BAB002C120B5640313072077C02124AA7402799
:100BBB00202910120B4D7F06C22C12074C120C323F
:100BCB00A380077F06D22C12074CEC543E120BE489
:100BDB004005124AF4C322D322543F03B4190050E8
:100BEB0044241583603F20360810E63730E7348005
:100BFB003410E71E30E62C802C00B00037AD34707B
:100C0B00000032790036000000B9313800350000A1
:100C1B000033F8E54B75F003A4B54A005007E5F037
:100C2B007003E8C322D3227F06EC7C0013CC33CCB9
:100C3B00DFFA22D2477B032047027B0275A003A871
:100C4B00317A00E220E704080A80F8EAB503004095
:100C5B005D304705120CBEF582120CBEF583AE005B
:100C6B007A007B007C017D0120471A120CBEFF8DA0
:100C7B00F0A42B75F00B84ABF0BD0A0040027D0095
:100C8B000D304713EF8CF0A42A75F00B84AAF0BC3F
:100C9B00090040027C000CE8B531D0304704EAB5BE
:100CAB00820CEBB58308A80674BCF2C38001D37524
:100CBB00A0002218E2540FB40D02740A22300B125A
:100CCB00851183851282AB15AA16BB000ABA1700D1
:100CDB005005C223C22F228512828511830ABA00C6
:100CEB00010B7408124C1070E9EAB4030040E3B432
:100CFB00410050DEF549F559C22375505630720349
:100D0B00755047851138851239D22A753C00D22986
:100D1B00120F5C40BDFAA23792297531014008755C
:100D2B00315F74BC124AF4EA1549753C0080051218
:100D3B000FC54059124AF4E5392408F5395002051C
:100D4B0038D549EBC03C753C00C22FC223120F5C57
:100D5B00D03C4005120DF8800ED223C22F155975C9
:100D6B004901120DDC4026303723124AF430290A90
:100D7B0074BC124AF475310180020531300605123C
:100D8B00105F4009754950D223C22FC322020CDDDC
:100D9B00E549335402F549E5392408F53950020584
:100DAB0038E5392407F582E5383400F583E0B4FFE4
:100DBB0017C03C434901120F5CD03C4007A849B80F
:100DCB0003278021D2238009302306753C00120EA5
:100DDB0009120FC5400F124AF40559302FB2C22F1A
:100DEB00124BE680ABD3C22322D22F0559FF853895
:100DFB0013E5392407F51450020513EFC322C22360
:0A0E0B00D22F2072077B02124BF178
:100E150080057B0D1210AB22EE75F003842E0422A3
:100E2500EE203607120E1D40498035124B96404282
:100E3500EE75F003842EB507005037EE2557B5073C
:100E450000500CE55703547FB506004025800CE59E
:100E55005703547F2557B507004017EE8011401200
:100E6500FCB50700400474FF8006EE2F80001304D4
:100E7500C322D322EE120E1D40F8B50700400474BC
:100E8500FF80ED207204EE2F80E4C083C082853898
:100E950083853982D2D2D2477E047801E0A3A3B5F7
:100EA5004A0510D20A8006B54B03104702F608DE44
:100EB500EBE9B502005004EAAA01F9E92A13354B1A
:100EC500133400254A133400FBC3202A23E54B03C2
:100ED500547F254BC3954AB34016EA03547F2AFD38
:100EE500C3954A500BAB05E903547F29C3954AB313
:100EF500EBD082D08322853883853982AF4AAE4BC9
:100F05007D04A2369234D236120E794048A234922C
:100F150036F542853883853982A3AF4CAE4D7D03C6
:100F2500120E254030F541853883853982D22C7AD9
:100F3500007B07E0B54200202C03B54100B3EA2051
:100F4500290313800133FAA3B22CDBE7202902EA37
:100F550003F548C322D3227F07D22C202A05120F7E
:100F6500E98003124B0D401B120F91D236120EFB76
:100F7500C236400F12100F400AC247B44100400567
:100F8500C38003D247D3302A02C22A2285388385FB
:100F95003982755700A37E03E0A3A3B54D0EE5572F
:100FA5006005B54D028018854D57800FB54C0EE58F
:100FB500576005B54C028007854C57DEDBF5572297
:100FC5007F07D22C202F05120FE98003124B0D400D
:100FD50011120EFB400C12100F4007B441005002D5
:100FE500C322D322C04A124B0DD0024007AB4A7C24
:100FF50005124BBF2275830305318531820582E0D9
:1010050030E7FA158274BCF0C3227B00EB2416830B
:10101500B5480CEB241083A2E79237C2E780370B63
:101025000BBB30E8803203300631093260331234AD
:10103500423521362437303848390C2D1824453AA5
:10104500512F542E152B1AC129C20BC30EC42C4186
:101055004A4268433844C322D32279007583038505
:101065003182E020E70CC3942424198329F90582F1
:1010750080F0E9540FD3700C1582E01582F00582DB
:1010850074BCF0C3220B8080808080800F800A0EA4
:101095000D000102030405060708090C8080808005
:1010A500808010111213858353858252E0F5518B90
:1010B500F0A4C4540FC5F0C445F0F022E5467F0501
:1010C5007A0013CA33CADFFA8A46E5477F057A00F4
:1010D50013CA33CADFFA8A4722EA2B1384FDEAC30F
:0C10E5009B5002F404C313FCB50500226C
:1010F100300A12851282851183AB15AA16BB000630
:10110100BA210050012285128285118385124785FB
:10111100114812116920D2ED7B02D22A124BE3C28F
:101121002A1211C912129220D2394037C23AC23B57
:10113100C23C12152620D22B203C141215AF20D20E
:1011410022203B0B12162120D219203A0280D21202
:1011510019A020D20E40CA1211D720D206D22212D3
:101161004BE322124BE3809DC238C237C239EB7088
:101171002D85823AE53A2A14F53BEAB42B00500753
:10118100D2387559008017B43B005009D237D23894
:1011910075592B8009D238D237D23975593BA215EE
:1011A100721672175012A23882159238A23782161F
:1011B1009237A23982179239A237B0129237A238E8
:1011C10072377239B392D2227583037582017A1311
:1011D100E4F0A3DAFC22E4A23E92E0A23F92E1FF16
:1011E1007582027583037A12E0C2E42430F005822D
:1011F100DAF67A05203F077A02203E027A00303B78
:101201000A7549D07B0D758205804E303A287549A3
:10121100A0302C06300F777549A8201C0C7B0F7568
:101221008202204334058280307B1B758215301B7E
:101231002815820B80237B0F7582027549E0E0B48B
:1012410030177549B82043117549B00582304409FA
:10125100E0B4340505827549C085823175820FEA93
:10126100600E1AE0C0828B82F0D0820B058280EF83
:10127100853182E0B430004015B43A005010A3EB40
:10128100B582F074BCF0E5492FF549C2D222D2D221
:1012910022121338500302133012146430D20302A5
:1012A1001334754A00754B06854739854838E53949
:1012B1007A0614B53A02802ADAF8E539C39404F5BE
:1012C1003950021538121B0420D2684015740225CA
:1012D1004BF582758303EAF0E54AC404C4F54AD5A7
:1012E1004BCCE53BC39547B40B00403FE5478548F0
:1012F100382405F53950020538754B06E5397A056C
:1013010004B53B028025DAF8121B0420D225401BCC
:10131100740FC3954BF582758303EAF0054AE539ED
:101321002404F53950020538D54BD1C2D2C322C2AB
:10133100D2D322D2D2D322755004800375500580B6
:0613410025854883854765
:1013470082E58220E01A1215115015A312151150CB
:101357000FA312151150091213B94004C3C2342246
:101367000547E4B547020548E53B24FCB547CCE50E
:1013770015703DE5596039B516361394012512F5F8
:1013870047E5113400F5487559008548838547823C
:10139700C236E58220E0191215115004D2368006B4
:1013A700A3121511500AA31215115004D234C322E7
:1013B700D322C247303907741B1213DF5016303758
:1013C7000774131213DF500C30380BD247741B12FB
:1013D70013DF4002C322D322FFC083C0822582F5D8
:1013E70082E5833400F583121429D082D083400527
:1013F70030472DC247C083C0820F0FC3E5829FF5D8
:1014070082E58394005009D082D083304712800E42
:10141700F583121429D082D0834003304702C322B8
:10142700D322C083C082E0FAA3E0F9A3E0FBD08215
:10143700D083EA2B138550F084FDEAC39B5002F456
:1014470004C313B505005014E92A138550F084FD31
:10145700E9C39A5002F404C313B5050022854883F3
:10146700854782E4FAFBFCFD7F0530341DC083C04D
:101477008230360CE0A3A3A3A3F0D082D0838010E0
:10148700A3A3E0D082D083F08006E58220E008E0C5
:101497002AFA50010B8006E02CFC50010DA3DFEA6D
:1014A700EDC313FFEC132CFCED3FFDEA2CFEEB3DE7
:1014B700FF404EEAC39CFAEB9DFB9235500AEAF4D3
:1014C7002401FAEBF43400FBEE75F007A4FDAEF04F
:1014D700EF75F007A42EFEEB600FEE13FEED13FD84
:1014E700EBC313FBEA13FA80EEEAAB06AA05124C2C
:1014F7001020D210EB700DEA34004008F549C2D233
:1015070022D2D2227549FFC2D2228550F0C083C0B1
:1015170082E0FAA3A3E0FBD082D0831210DE223050
:101527003940E54AB4663B74E51217E6754E121268
:1015370018A720D272402B74191217E6754E0312A2
:1015470018A720D2624060C247121805E54DB43F84
:1015570013D22912188BC24712180574E51217E621
:10156700800E8041C229E54CB43F3A741F1217E63A
:10157700E54DD247C2D612183B402AC36001D38239
:10158700124022C24712179A3005157583037582D8
:1015970002E0B400080582E0B404028003203405A9
:1015A700D23CC2D222C2D22230374DE54A30130A8A
:1015B70030140754F0B440408003B4443B74ED1238
:1015C70017E6754E121218A720D24E404A74111210
:1015D70017E6754E031218A720D23E403CD2471299
:1015E7001805E54DB40F13D22912188BD2471218DC
:1015F7000574ED1217E6800E801DC229E54CB40F65
:101607001674171217E6E54DB4000CD24712179A55
:101617004005D23BC2D222C2D22230384BAA4A74EA
:10162700061216F250035302F0BA603FC229E5478B
:101637002404B53B028031854883E5472403F582BE
:1016470050020583755005121511501C74E51217C9
:10165700E6C3953AB40700500F754E121218A7400B
:101667000774051217E6804D0216EFAA4A74FE1298
:1016770016F2500353020FBA066ED229E547B53A60
:0C168700028065854883854782124C680C
:10169300755005121511505474191217E62406FAE1
:1016A300E53BC39AB407005043754E031218A74095
:1016B3003B74FF1217E612188BC247121805E54D4B
:1016C300D247D2D6D22812183D40211216FF302C11
:1016D3000F7583037582037401F07582147431F0FE
:1016E300C24712179A4005D23AC2D222C2D222125C
:1016F30017E6853883853982E02402227583037ACD
:1017030006758209E4F00582DAFB758202E0FAE4E9
:10171300F075820EEAF075821BEAC2E42430F0759C
:1017230082147430F075820378017F15E0C2E4F609
:10173300C0828F822430F0D082E4F005820F08B893
:1017430007EA758203E4F00582E9F00582EAF00511
:1017530082EEB403005010EEF075820BEBF00582BD
:10176300ECF00582EDF022B4030EEBF005827582F6
:101773000CECF00582EDF022B4040CEBF00582ECE6
:10178300F075820DEDF022EBF00582ECF00582EDB1
:10179300F075820DEEF0227583037A027B037F06D8
:1017A3003047027F05E4FCFD8A82E0C2E42CFC8B17
:1017B30082E0C2E42DFD0A0A0B0BDFECED75F003AA
:1017C300A42C75F00A84E5F06005740AC395F0FB58
:1017D3008A82E0C2E4B50304C234C322D2343005A2
:1017E300F9D32285483830E710F404F539E547C3C7
:1017F3009539F53950021538222547F53950020538
:101803003822758203758303E4F54DF54C7A06E0BF
:10181300A2E4E54D33F54D0582DAF47A06E0A2E45D
:10182300E54C33F54C0582DAF430470B534D0FE5A5
:101833004C0303540FF54C22C228C22C30D615306A
:101843002809C22820E504D22C8001F4543F6036D5
:10185300B40701E46021B40B00402BB41D005026F3
:1018630024F7838012018002038080808004800734
:101873000880800509800620E70C3047077583033D
:10188300758202F0C322D3227409FBFA1A7583030B
:101893007D068A82E0FC8B82E0CCF08A82ECF01A2F
:1018A3000BDDEF22853883853982E54E20E0202049
:1018B300E00C124C68E0F544A3E54E20E028E0F587
:1018C30041A3E0F542A3E0F543A3E54E20E0E6E4BF
:1018D300FEFF7A04E02EFE50010FA3DAF78F468E47
:1018E30045E54E20E0C9AB46AA4530E510E5442462
:1018F30002400ABB0046E544B50200403FE54912F9
:101903004C1050010A8A4F740EAB46AA45124C1074
:1019130050010AEAFB75F003A4FCAD03AE04AF0467
:10192300EB75F005A4C5F0600375F0FFE54E30E4F8
:1019330002AFF030E208AD04AEF080028057AA4F48
:10194300E54EA2E1203501B39236E541303604C3BA
:101953009A80012A4043B50300403AB50700503549
:10196300E542203604C39A80012A402DB503004086
:1019730024B50400501FE54E20E316E5433036043A
:10198300C39A80012A4012B505004009B5060050EC
:1019930004C2D2C322D3C2D222D2D2D322C23EC2E3
:1019A3003FA21372145006302906021A61021A78F4
:1019B300E53BC39539FA7022AC13AD147F0D124980
:1019C300498C838D82EB8A03FA40068E138F148031
:1019D300D9E5392402B582D28005B40E0040CBE5A7
:1019E300392402F53950020538754E061218A7201E
:1019F300D251406AE5392403F53950020538755749
:0E1A03000F754A00E53BC39539B40300403827
:101A1100121B044033758303855782F00557054A2D
:101A2100E54AB405028021E53BC39539B40600407F
:101A310017754E091218A7400FE5392406F53950DC
:101A410002053880C1021A80E54AB40209121A84DB
:101A5100400ED23E800AB40507121AB04002D23FAE
:101A6100A213B014B03E4013A214B013B03F400B08
:101A7100A23EB3B03F4004C2D2C322C2D2D322D2CB
:101A8100D2D32275830375820F7B00E0A2E4CB33AE
:101A9100CBC2E475F00AA4FA0582E0A2E4CB33CB11
:101AA100C2E42A75F00484EBB5F002C322D3227597
:101AB10083037A0F7B107E05E4FCFD7F018A82E0BF
:101AC100A2E4CF33CFC2E42CFC0A0ADE0280118BE0
:101AD10082E0A2E4CF33CFC2E42DFD0B0B1E80DDEB
:101AE100ED75F009A4FAEC75F003A42A75F00A84E7
:101AF100AAF0EFD2D6C24712183B4005B50202C385
:101B010022D322853982853883E582A2E0923D2065
:101B11003501B39236E4FFFE75F0047902C240E06C
:101B2100F7B4FE02D2402EFE50010F09A3D5F0EF0B
:101B31008F468E45EF601975F0047902E7C313F7FC
:101B410009D5F0F8EFC313FFEE13FE80E7021C1076
:101B5100EE8549F084FFE549C313B5F00050010F4C
:101B610075F0047902E7303604C39F80012F40DD10
:101B7100F709B236D5F0EE8A418B428C438D44EEA3
:101B810075F00E84FAE5F0B4080040010A78047F8C
:101B9100037903EF8AF0A4F7090F0FD8F6121C1886
:101BA10020D26CE541254225432544B40702801625
:101BB100B4065C30405979417A04E7B403030780E5
:101BC100E209DAF68049AA41E542232AFAE54323EC
:101BD10023232AFAE54475F00CA42A24E883802201
:101BE10016001403FFFFFF180115FF09120717055F
:101BF100FFFF0211FF131908FF04FFFFFF10FFFF92
:101C0100FF06A2E4303D01B392E4FAC2D2C322D36B
:101C1100C2D222D2D2D3227941E7B502004029B5FE
:101C21000300500477018019B50400500477028045
:101C310010B50500500477038007B50600500977F9
:0B1C41000409B945D4C2D222D2D2223D
:10613D00C22622301E12851183851282AB15AA1636
:10614D00BB0006BA0D0050012285128285118374A1
:10615D0008124C10B405F1EAF549B421005048F588
:10616D0059755064307203755046C22A858239853F
:10617D008338753C00D22CD23412628340298512AB
:10618D0039851138D22C8539828538837F03126287
:10619D0022C2E0B40414D229753101D22CE58270EB
:1061AD0002158315828019026155B40202800270B6
:1061BD00F6C22975315F74BC124AF4753C00C22CCD
:1061CD008582398583381262E440DC858239858386
:1061DD0038D549F2202917C22CE582700215831596
:1061ED00827F03126222ECC2E2B401BB800AD22C80
:1061FD007F03126222BC02AF30290A74BC124AF42A
:10620D00753101800205313004051263684098D262
:10621D0027754970227C007BFFE0FDB5030050011E
:10622D00FBA3E0B4FF01EBFEED75F00484F5F02D5A
:10623D00500274FFB506004007EDC395F0B506009A
:10624D00B3EC33FCDFD3228539828538837A007B2A
:10625D00007C00E0A3302C0BB542028001B3EA3381
:10626D00FA8009B541028001B3EB33FBA2E0EC33B8
:10627D00FCB22CDFDE227F08124B0D403EAF4AAE42
:10628D004B124A93F542AF4CAE4D124A93F5411065
:10629D00342BE542B4FF22E541B4FF1FE54D254CFB
:1062AD001304F5F0E54B254A1304B5F000500CE549
:1062BD004A04F542E54D14F541C322D322E541B41C
:1062CD00FF05E54D254C13F544E542B4FF05E54BBF
:1062DD00254A13F545C322126283402D3072077C87
:1062ED0002124AA740238539828538837F081262BE
:1062FD00548A468B47202907126349AA46AB471299
:10630D0063184005124AF4C322D322EA7006EB60EB
:10631D0009F480026BF4540F701CEA540F240283AD
:10632D0080103031323334353637383900000000C3
:10633D0000006002C322D3227F0780027F04C007C2
:10634D00E5467A0013CA33CADFFA8A46E547D00715
:10635D007A0013CA33CADFFA8A4722C2367A007B23
:10636D0000758303853182E020E70505820A80F7F9
:10637D00BA020040607A001582AD82E0FC1582E021
:10638D00C3943023A236340075F00A84A2E092360D
:10639D00E5F02BFBE531B58202800D1582E0C3944B
:1063AD00302AFAE531B582D5EBA23634002AFA50FF
:1063BD000C7B01EA2406FA40011BEB70F6EA75F03E
:1063CD000A84E5F06003F4240B2430B504078D82B4
:0763DD0074BCF0C322D322BF
:1055FE000000000000000000009E000000000E00F1
:10560E000E000028FE28FE28004854FE54240046B2
:10561E002610C8C4006C92AA44A000000A0600001E
:10562E000000384482000000824438000028107CBC
:10563E0010280010107C10100000C0600000001038
:10564E00101010100000C0C0000000402010080410
:10565E00007CA2928A7C000084FE80000084C2A29C
:10566E00928C0062828A966200302824FE20004EC0
:10567E008A8A8A720078949292600002E2120A0676
:10568E00006C9292926C000C9292523C00006C6CE8
:10569E0000000000AC6C00000010284482000028BE
:1056AE0028282828008244281000000402A2120C88
:1056BE00006492F2827C00FC222222FC00FE929276
:1056CE00926C007C8282824400FE8282443800FE0C
:1056DE009292929200FE12121212007C829292F418
:1056EE0000FE101010FE000082FE8200004080823C
:1056FE007E0200FE1028448200FE8080808000FE24
:10570E00041804FE00FE081020FE007C8282827CBB
:10571E0000FE1212120C007C82A242BC00FE12325B
:10572E00528C008C92929262000202FE0202007E65
:10573E008080807E003E4080403E007E8070807E75
:10574E0000C6281028C6000E10E0100E00C2A2924D
:10575E008A860000FE8282000004081020400000AD
:10576E008282FE000008040204080080808080808F
:10577E000000020408000040A8A8A8F800FE9088C7
:10578E0088700070888888400070888890FE00704D
:10579E00A8A8A8300010FC1202040018A4A4A47C2F
:1057AE0000FE100808F0000088FA80000040808893
:1057BE007A0000FE20508800000082FE800000F873
:1057CE00083008F000F8100808F00070888888701B
:1057DE0000F8282828100010282830F800F81008A3
:1057EE0008100090A8A8A84000087E888040007885
:1057FE00808040F8003840804038007880608078A3
:10580E000088502050880018A0A0A0780088C8A852
:10581E0098880000106C8200000000FE000000005E
:10582E00826C10000008082A1C0800081C2A0808B0
:10583E00001CA2E222240078828042F80070A8ACFC
:10584E00AA300040ACAAACF00040AAA8AAF00040D2
:10585E00AAACA8F00040AEAAAEF00018A4E4241042
:10586E000070ACAAAC300070AAA8AA300070AAAC26
:10587E00A83000008AF8820000008CFA8400000034
:10588E008AFC800000F02A282AF000F02E2A2EF042
:10589E0000F8A8ACAAA800E8A8F0A8B000FC12FE78
:1058AE00A2A200708C8A8C7000708A888A70007038
:1058BE008A8C88700078848244F80078828440F85C
:1058CE000018A2A0A278007886848678007882805C
:1058DE008278003048FC48200010FC9294800052E0
:1058EE0054F85452007E0A2EF0A00090907C1212B2
:109C4C007828790030B3170000D9F9D8F7800D784F
:109C5C0028790020B3080000D9F9D8F7D322C32201
:109C6C0074E2D5E0FD22C2AB7F0012F8F5D272C2CD
:109C7C002C5389F0438902A2B392287F02900000F2
:109C8C00302810129C5B4008129C6C129C4C501398
:109C9C00029D4C129C4C4008129C6C129C5B500315
:109CAC00029D4C758A00758CFFC28DD28C202C25A0
:109CBC0020281130B252308D03758CFF30B2492000
:109CCC00B3F1803430B241308D03758CFF30B23833
:109CDC0030B3F1802320281120B22D308D03758CE8
:109CEC00FF20B22420B3F1800F20B21C308D0375FD
:109CFC008CFF20B21330B3F1C28CDF02802AB22861
:109D0C00858355858254809BE58A758A00758C0005
:109D1C00A28DC28D13F0A3E583B40307129D53C229
:109D2C008C8005B22C029CB9E58AA28D13F0A3E5B8
:109D3C0083B40303129D53E4F0D2AB12FD72D32211
:109D4C00D2AB12FD72C3220582D582021583158215
:019D5C0022E4
:0CFCC6002573002D24252B0025627500FD
:10F9E8007E007F287D007B017A117917122F59E458
:07F9F800787DF6787BF62212
:10F34100901116E0FFE4FBFA7D4912BA73E4FF1253
:10F351005E05900100E493FF641B6004EFB43A087A
:09F361009010A2E0FF125CA02252
:0AFD1E0012F34112F98B12F9E822EA
:10FB88009010A2E564F0E4FF12DCF3D26612F9E803
:01FB9800224A
:0DFC8700D26812F341E4FF12DD54C2662280
:10F5CA0030671F9010AE1229F312FADB9010B3EFD6
:10F5DA00F078B57C107D019010AE1229F3122D92AD
:03F5EA00C26722D3
:10EF9C00129C72502D901E1E74FFF0E4A3F0901E74
:10EFAC001EE0FF12F065501AE4901E1EF07B017AF1
:10EFBC0011793F12B528129E6AE433901E1FF0E0BF
:03EFCC0060DC22E4
:108B5D00787CE624FB7003028C5E147003028CA8F3
:108B6D00147003028C3324066003028CB612F2ECEF
:108B7D00901298EFF07003028CBA787C760512F99A
:108B8D008B901116E0FF7B6E7A007D5212BA7390B6
:108B9D0010B1E06401600DE49010A3F0901115F098
:108BAD00901299F0900100E493FF641B6005EF644F
:108BBD003A706D9010A4E0547024E0601824F060B9
:108BCD001C24F0602024F06024244070289010A113
:108BDD007405F080259010A1740AF0801D9010A1ED
:108BED007414F080159010A1741EF0800D9010A1DA
:108BFD007428F08005E49010A1F09010A2E564F0C7
:108C0D009010A1E0601A7F01125CA0901116E0FF98
:108C1D009010A1E0FB7A007D5212BA73787C760732
:108C2D007FFF125E0522901116E0FF12F0C7BF45BF
:108C3D0012787C7605901116E0FF7B6E7A007D52DE
:108C4D0012BA7312F2ECEF706412FD1E787C76018D
:108C5D0022900100E493FF641B6004EFB43A05E435
:108C6D00FF125CA012EF9C901116E0FF12F0C7BF2F
:108C7D004507787C760612FD1E12F2ECEF7008782F
:108C8D007C760112FD1E229010B1E06401601E90F1
:108C9D0010A3E06018E4F012FB882212F2ECEF70E2
:0E8CAD000C787C760112F98B22787C760122FD
:10857300901C27E0D394DD5045901C29E0FF9440E4
:10858300503C901C28E09F5035901C2AE0940950E1
:108593002DA3E0FF149403400BEF94664020EFD328
:1085A3009469501A901C2E1229F3122633601990E5
:1085B3001C2CE0D3940F5006A3E09403400AE4FB81
:1085C300FA7D017F3512B90178A47C107D017B010E
:1085D3007A1C79277E007F0D12260D9010A8E0FFEC
:1085E300D3940450089010B17401F0800DEF249CD3
:1085F3009010B1F09010A87401F09010A8E0FF144F
:10860300603C146028146014147046901253744232
:10861300F0E4A3F0901256F0901297F090120E74BB
:1086230042F0E4A3F0901211F0901252F09011C9AD
:108633007442F0E4A3F09011CCF090120DF090107E
:10864300B27442F0E4A3F09010B5F09010F6F0800D
:108653000BEFFB7A007D027F3512B9019010AB124C
:1086630029F312263360209010A9E0FFA3E0FD1246
:10867300A1839010AB1229F3901AD3122A2A7BFFFD
:108683007AFC79C61237E2C2679010AE1229F31250
:108693002633606B9010A8E06401706312FADB90DC
:1086A3001C34EFF09010A6E0FEEFD39E400E901C1A
:1086B30034E0FB7A007D037F3512B901E4901C3569
:1086C300F0901C34E0FFA3E0FEC39F50309010AE47
:1086D3001229F38E8275830012264CFF9010A7E0B7
:1086E300FD12B6B7EF700E901C35E0FB7A007D04E7
:1086F3007F3512B901901C35E004F080C4D26712B3
:03870300FB8822CE
:10F7E8009010B27444F09011C9F090120EF090127B
:0CF7F80053F09010A2E564F012FC872290
:10F85700EF24BFFFC3940A5011EF75F003A424F7F8
:0BF86700F582E43410F583122A2A22F7
:1040700012FCDE12F98B901142E0FF7876F66006B2
:10408000E6D39440400D7876E6FB7A007D017F37D9
:1040900012B9017876E6B4041978437C117D017B6E
:1040A000FF7AFC79C9122CA9EF7007FF125E051286
:1040B000F317E47879F6901143E064246003024139
:1040C000BE9010A4E030E21C7876E6B4031690119E
:1040D00044E0B42B0FA3E0FF12FC1650077879766A
:1040E000040241BE9010A8E0640160030241BE904A
:1040F00010A4E0FF20E00620E1030241BE7876E64E
:10410000FFB40313901144E0B42B0CA3E0B42D07CB
:10411000787976020241BEEFB40313901144E0B403
:10412000250CA3E0B42507787976030241BEEFB4ED
:10413000031A901144E0FF12FC165010901145E054
:10414000FF12FC1650067879760180729010A4E078
:1041500030E1167876E6B40210901144E0FF12FCCC
:104160001650067879760180559010A4E030E14E23
:104170007876E664047047901144E0FF643160058E
:10418000EF64327039901145E0FF12FC16502F9009
:104190001144E0B43207A3E0D39435502190114686
:1041A000E0FF12FC165017901144E0B4320CA3E06B
:1041B000B43507A3E0D39435500478797601787943
:1041C000E61470030243C0147003024445147003E4
:1041D00002447A14700302449A240460030244BB2C
:1041E0009010A4E030E3030244BBE47878F690102A
:1041F000A5E0FF7876E6FEC39F400CA3E0FFEED378
:104200009F5004787876FFE47877F67877E6FFC3F6
:10421000189650257878E6B4FF1F74432FF582E492
:104220003411F583E0FF9010A7E0FD12B6B7EF70F0
:10423000037878F678770680D29010B1E064016058
:104240000D901115E0C3940A4004E47878F678786C
:10425000E670569010A8E0FF1460301460201460DF
:1042600010147036901253744EF0E4A3F09012566E
:10427000F090120E744EF0E4A3F0901211F0901131
:10428000C9744EF0E4A3F09011CCF09010B2744ECB
:10429000F0E4A3F09010B5F0800BEFFB7A007D0204
:1042A0007F3712B90112FC8722787BE6702A787674
:1042B000E69010B3F02401FFE433FE78B57C107D66
:1042C000017B017A11794312260D901141E0901083
:1042D000F6F0787B06024365787BE6640170297806
:1042E00076E69011CAF02401FFE433FE78CC7C110D
:1042F0007D017B017A11794312260D901141E090E6
:10430000120DF0787B06805D787BE6640270297878
:1043100076E690120FF02401FFE433FE78117C1250
:104320007D017B017A11794312260D901141E090B5
:104330001252F0787B06802D787BE6B403277876DE
:10434000E6901254F02401FFE433FE78567C127D8F
:10435000017B017A11794312260D901141E09012F0
:1043600097F0787B069010A8E0FF787BE6C39F501B
:10437000030244BB901298E06409600678787645A1
:1043800080047878764CEF14601E14601414600A70
:0943900014701E7878E6901253B7
:10439900F07878E690120EF07878E69011C9F07806
:1043A90078E69010B2F0800BEFFB7A007D037F373F
:1043B90012B90112FC8722E4FF125E05C2677BFF76
:1043C9007AFC79CE901B03122A2A7B007A00797A2B
:1043D900901B06122A2A0B7A117944124CF3BEFF5C
:1043E90012BFFF0F787AE6FB3395E0FA7D047F3739
:1043F90012B901787AE6FF9010A7E0FD12B6B7EF7F
:1044090070030244BB9010A6E0FF9010B3E0C39F75
:1044190040030244BB787AE6FF9010B3E0FE04F053
:1044290074B52EF582E43410F583EFF09010B3E003
:1044390024B5F582E43410F583E4F022E4FF125E3A
:104449000512F5CA9010A5E0FF9010B3E0C39F4094
:104459006112FC87901298E0640960089010B274A8
:1044690045F080069010B2744CF09010F674F0F09C
:1044790022E4FF125E059010B3E0D39400400EE0F1
:1044890014F024B5F582E43410F583E4F012F5CA8A
:1044990022E4FF125E05901145E0540F787AF67513
:1044A900F003A424F7F582E43410F5831229F312FA
:0344B9002B1B2298
:109E6A00C268901142E07003029F719010B1E064E1
:109E7A00017057FF787DE6FEEFC39E5022EF25E082
:109E8A002417F582E43411F583E0FCA3E0FD901178
:109E9A003FE0B50407A3E0B50502C3220F80D5EE63
:109EAA00C394144003029F7190113FE0FCA3E0FDAC
:109EBA00EF25E02417F582E43411F583ECF0A3EDE5
:109ECA00F0124070787D06029F719010A374FFF023
:109EDA00901115E06046901142E0FF901187E0FE74
:109EEA006F7034901141E0FF901186E0B507287B2E
:109EFA00017A117943901D28122A2AEEFF901D2B10
:109F0A00E4F0A3EFF07A11798812DB03EF7008907E
:109F1A001299E004F08005E4901299F0901299E009
:109F2A00702704F0901142E0901187F02401FFE4B9
:109F3A0033FE78887C117D017B017A1179431226E0
:109F4A000D901141E0901186F0901115E004F09007
:109F5A0010B1E0FF901299E06F6009901115E0C30B
:0A9F6A00940A4003124070A268221E
:10BF33009010B27444F0E4A3F09010F6F0FE7F4149
:10BF4300FD7B017A1079B5122F599011C97444F011
:10BF5300E4A3F090120DF0FE7F41FD7B017A11798D
:10BF6300CC122F5990120E7444F0E4A3F0901252A5
:10BF7300F0FE7F41FD7B017A127911122F59901245
:10BF8300537444F0E4A3F0901297F0FE7F41FD7BDD
:10BF9300017A127956122F59E4FF7BFF7A00792A2E
:10BFA300EF75F003A424F7F582E43410F583122A25
:10BFB3002A0FEFB40AE412E908D270901E33740119
:10BFC300F012FA9CE4FFFE12DB6A901116EFF012F6
:07BFD300F9E8787C760122F9
:10CABE0025730000030300000605000000060700B2
:10CACE000000013741424301344A4B4C013153546B
:10CADE0055012E2C3B3F0400000000000404000012
:10CAEE000606000000060800000001384445460115
:10CAFE00354D4E4F0132565758013024253A0120FC
:10CB0E002B2D2F0002020000000909000002000078
:10CB1E000000013947484901365051520133595AE4
:10CB2E002A03000000000001010000FFEC19FF7253
:10CB3E00C1FFE94FFFED48FFE6C7FFFBC9FFFAC68D
:0CE22100C164C16541196A0041195B012C
:10F9FF00125D7592732064083073057FFA12EC570D
:07FA0F00A2739264A27322AE
:10F2EC0090196AE0701D12F9FF501420650A125D26
:10F2FC00C150057F0A12EC57125DC192658006C29F
:0BF30C00658002D265A265E433FF2299
:10EA1E007F03125BE4EFF4600AE4FBFA7D017F40B2
:10EA2E0012B901E4FEE42EF582E43480F583E0FDB4
:10EA3E0020E003AF0622ED20E105EE2408FF22AF11
:10EA4E0005ED20E205EE2410FF220EEEB408D67F6F
:02EA5E00FF2295
:08FD8C007F0212DD54C2622265
:08FD94007F0212DCF3D26222AF
:10FB65009019B3E0FFE4FBFA7D4912BA73E47870AB
:02FB7500F62276
:09FD4E0012FB657F0A12B77E2248
:09FD57007870E6600312FD4E22F3
:10F47E003063229019671229F312FADB786FEFF6D8
:10F48E0090196CF0786E7C197D019019671229F332
:06F49E00122D92C2632250
:10990100901C36E0D3940F5038901C38E0FF9440FF
:10991100502F901C37E09F5028901C39E09409503B
:1099210020A3E0941F501A901C3D1229F3122633F4
:109931006019901C3BE0D3940F5006A3E0940340C0
:109941000AE4FBFA7D017F3F12B901785D7C197D44
:10995100017B017A1C79367E007F0D12260D90194C
:109961006B7442F0E4A3F012FB65E4786FF6FE7FBE
:1099710041FD7B017A19796E122F599019641229D0
:10998100F31226336020901962E0FFA3E0FD12A1DB
:10999100839019641229F3901AD3122A2A7BFF7A31
:1099A100CA79BE1237E2C2639019671229F31226EF
:1099B10033606312FADB901C43EFF090195FE0FE15
:1099C100EFD39E400E901C43E0FB7A007D027F3F67
:1099D10012B901E4901C44F0901C43E0FFA3E0FEA7
:1099E100C39F50309019671229F38E82758300123C
:1099F100264CFF901960E0FD12B6B7EF700E901C77
:109A010044E0FB7A007D037F3F12B901901C44E0E2
:0A9A110004F080C4D26312FD942219
:0AFD280090196B7444F012FD8C2258
:10F5160090195DE030E01D90195CE070177D10FCDD
:10F526007F0A12CF9E90195C74FFF09019AFE4F039
:05F53600A37408F0229F
:10EC19007870E66401601212FD57901961E030E1E5
:10EC29002C7872E6FF12BFDA2212FD577873E6FFDD
:10EC39006409600B901961E030E11212FDED229038
:0EEC49001961E030E3077873E6FF12FDED225B
:1072C1007870E6FF600E9019B2E07872666072EF36
:1072D1006401606D12FD57901961E020E0030274B2
:1072E100B5C26390195FE0FF786FE6C39F504C7899
:1072F10072E6FFA3E0FD12B6B7EF603F7872E6FFDA
:10730100786FE606246EF582E43419F583EFF0E632
:10731100FF246EF582E43419F583E4F090196CEFE3
:10732100F07F0112B77E12F51690195FE0786F6653
:1073310060030274B57F0A12DD54227F0B12B77EFF
:10734100227870E6640160030273D6901961E0202F
:10735100E00412FD4E22C26390195BE0700F787356
:10736100E6FF12FC3450067873742026F690195FFC
:10737100E0FF786FE6C39F50537873E6FFA3E0FD0B
:1073810012B6B7EF60467872E69019B2F008E6FFE0
:10739100786FE606246EF582E43419F583EFF0E6A2
:1073A100FF246EF582E43419F583E4F090196CEF53
:1073B100F07F0212B77E12F5169019B3E0FF7B3C05
:1073C1007A007D5212BA73787076022212FD4E7FD6
:1073D1000B12B77E227870E6640270679019B2E0F2
:1073E100787266705E90195BE0700F7874E6FF1238
:1073F100FC3450067874742026F67874E6FF9019F0
:1074010060E0FD12B6B7EF601C7874E6FF786FE6B6
:10741100246DF582E43419F583EFF07F0312B77E12
:1074210012F5168019786F16E6246EF582E4341988
:10743100F583E4F0E690196CF07F0B12B77E78705B
:107441007603227870E66403706A9019B2E078726C
:1074510066706190195BE0700F7875E6FF12FC347D
:1074610050067875742026F67875E6FF901960E06D
:10747100FD12B6B7EF601C7875E6FF786FE6246DF4
:10748100F582E43419F583EFF07F0412B77E12F52B
:10749100168019786F16E6246EF582E43419F583A7
:1074A100E4F0E690196CF07F0B12B77E12FD4E7F6F
:0574B1000A12DD542267
:10E94F00901961E0FF20E00620E10330E3387F07F4
:10E95F0012B77E7870E6700876017F0912B77E22B3
:10E96F007870E6B4011990195DE030E21990195BE7
:10E97F00E070047F0180027F0090195BEFF022129C
:07E98F00FB657870760122A0
:10ED480012FD57901961E030E02F12F47E90195EA1
:10ED5800E0FF90196CE0FEC39F401990195FE0FF37
:10ED6800EED39F500F7F0512B77E12FD8C90196B62
:0AED78007445F0227F0B12B77E22D3
:10E6C70012FD57901961E030E03E30630912F47E85
:10E6D7007F0612B77E22786FE6D39400402516E6B0
:10E6E700246EF582E43419F583E4F0E690196CF0B2
:10E6F7007F0612B77E12F516786FE6700B7F0A1247
:09E70700DD54227F0B12B77E22C3
:10FBC90012FD57901961E030E0057F0812B77E22D7
:10FAC60012FD57901961E030E20A7872E6FF12E5FE
:05FAD6000512F51622E7
:10F6D80012FC433062197871E675F003A42439F5F9
:10F6E80082E434CBF583122A33122B1B12F98B22B6
:10EE600030622D9019B0E02404FD9019AFE0340019
:10EE7000FC7F0A12CF9E12F6D8D39019B0E094000E
:10EE80009019AFE09400400D74FFF5F012279F2217
:06EE90007F0A12DD54228E
:09FD60007F0A12DD5412F98B2216
:10E1460090195AE024FE603604704212F2ECEF6039
:10E156004212F98B901961E030E40612FC4312FA80
:10E166004490195DE030E10612FC4312ED487D0152
:10E176007C007F0212CF9E90195A7402F02212F28E
:10E18600ECEF700F90195A04F012F98B2290195A7D
:04E196007401F022FE
:10D73D0012E14612F80412EA1E901E35EFF012F8AF
:10D74D00109019B1E024FE603F04704D901E35E03D
:10D75D00FFF4604BE490195CF0EF75F005A424C163
:10D76D00F974CA35F0FA7BFF78717C007D007E007C
:10D77D007F0512260D12F6D87D017C007F0212CF97
:10D78D009E9019B17402F022901E35E0B4FF101274
:10D79D00FD609019B17401F0229019B17401F0225D
:10F3E20090196B7444F0E4A3F07EFB7FC912DB6AD0
:10F3F2009019B3EFF0E4786FF6FE7F41FD7B017A5E
:07F4020019796E122F592247
:10CB4E00901DF3EFF0A3ECF0A3EDF09019B4E0FF1D
:10CB5E00C39414400BEFFB7A007D017F2712B901BD
:10CB6E00901DF3E0FFC39414400BEFFB7A007D029F
:10CB7E007F2712B901901DF3E0FF25E025E024B5D3
:10CB8E00F582E43419F583E06449600BEFFB7A001B
:10CB9E007D037F2712B901901DF3E0FF25E025E00C
:10CBAE0024B5F582E43419F5837453F0901DF4E046
:10CBBE00FCA3E0FDEF25E025E024B7F582E434196F
:0FCBCE00F583ECF0A3EDF09019B4E004FFF02232
:10DCF300901E36EFF09019B4E0FF901E36E0FEC39D
:10DD03009F400BEEFB7A007D017F2812B901901E24
:10DD130036E0FF25E025E024B5F582E43419F583E8
:10DD2300E0B44418EF25E025E024B6F582E4341985
:10DD3300F583E0FFE4FBFA7D4912BA73901E36E0E7
:10DD430025E025E024B5F582E43419F5837452F017
:01DD530022AD
:10DD5400901E37EFF09019B4E0FF901E37E0FEC339
:10DD64009F400BEEFB7A007D017F2912B901901EC2
:10DD740037E0FF25E025E024B5F582E43419F58386
:10DD8400E0B44418EF25E025E024B6F582E4341924
:10DD9400F583E0FFE4FBFA7D4912BA73901E37E085
:10DDA40025E025E024B5F582E43419F5837453F0B5
:01DDB400224C
:10CF9E00901DF6EFF0A3ECF0A3EDF09019B4E0FFC6
:10CFAE00901DF6E0FEC39F400BEEFB7A007D017FE5
:10CFBE002B12B901901DF6E025E025E024B6F5828E
:10CFCE00E43419F583E0B4FF19E4FFFE12DB6A9036
:10CFDE001DF6E025E025E024B6F582E43419F5834C
:10CFEE00EFF0901DF6E0FF25E025E024B5F582E494
:10CFFE003419F5837444F0EF25E025E024B6F5826C
:10D00E00E43419F583E0FF901DF7E0FAA3E0FB7D11
:05D01E005212BA73225A
:10F36A00AE079019B4E0FFEEC39F5011EE25E025D9
:10F37A00E024B5F582E43419F583E0FF22EEFB7A46
:09F38A00007D017F2A12B9012265
:10AC1200901E2174FFF0E4901E20F09019B4E0FF22
:10AC2200901E20E0FEC39F400302ACEFEE25E0251C
:10AC3200E024B5F582E43419F583E064447045EE0E
:10AC420025E025E024B6F582E43419F583E0FF120D
:10AC5200F0C7BF452F901E20E025E025E024B6F581
:10AC620082E43419F583E0FFE4FBFA7D4912BA73FA
:10AC7200901E20E025E025E024B5F582E43419F5A4
:10AC8200837452F0901E20E025E025E024B5F58281
:10AC9200E43419F583E06452704A901E20E0FF25E7
:10ACA200E025E024B5F582E43419F5837445F0EF2C
:10ACB20025E025E024B7F582E43419F583E0FEA30C
:10ACC200E0AA06F9122B1B901E20E025E025E024C5
:10ACD200B5F582E43419F583E0B445087452F0E422
:10ACE200901E21F0901E20E004F002AC1D901E2167
:03ACF200E0FF225E
:10F53B00E4FF9019B4E0FEEFC39E5018EF25E025D1
:10F54B00E024B5F582E43419F583E0B44503745235
:05F55B00F00F80DE222C
:07FDCA0012AC12EF60FA22F7
:10E9DB00E49019B4F0FFEF25E025E024B5F582E4CF
:10E9EB003419F5837449F0EF25E025E024B6F58260
:10E9FB00E43419F58374FFF0EF25E025E024B7F537
:10EA0B0082E43419F5837400F0A3742AF00FEFB489
:03EA1B0014C422FE
:10D1A900306D033066089017AD74FFF08013901747
:10D1B900ADE070047F0180027F009017ADEFF07041
:10D1C9005D788106E670021806E4FF9017AEE0FE6E
:10D1D900EFC39E5049EF75F003A424EBF582E434C4
:10D1E90017AD82FCF583E064527030A374FFF5F04B
:10D1F90012279F8D828C83A3E0FAA3E04A701C8DCD
:10D20900828C837445F0EF25E024AFF582E434176E
:0FD21900F583E0FCA3E04C6002D2750F80AD22DC
:10DA33007D017C007F0312CF9E30755BC275E4903D
:10DA43001E38F09017AEE0FF901E38E0FEC39F50E3
:10DA530046EE75F003A424EBF582E43417AD82FCA3
:10DA6300F583E0B44529EE25E024AFF582E43417CD
:10DA7300F583E0FCA3E04C6016EE25E024AFF582CD
:10DA8300E43417F583E0FEA3E0AA06F9122B1B90FA
:08DA93001E38E004F080AC2213
:10DB6A00901E22EEF0A3EFF09017AEE0FFC3941ED2
:10DB7A00400BEFFB7A007D017F2C12B9019017AEA2
:10DB8A00E0FF75F003A424EBF582E43417F58374FF
:10DB9A0049F0EF75F003A424ECF582E43417F58319
:10DBAA00E4F0A3F0901E22E0FCA3E0FDEF25E024C0
:10DBBA00AFF582E43417F583ECF0A3EDF09017AEDD
:04DBCA00E004F02261
:10BA7300901DC4EFF0A3EDF0A3EAF0A3EBF0901751
:10BA8300AEE0FF901DC4E0FEC39F400BEEFB7A00C7
:10BA93007D017F2D12B901901DC5E0FFB44932A28B
:10BAA300AF9274C2AF901DC4E0FE75F003A424EB03
:10BAB300F582E43417F5837449F0EE75F003A4249A
:10BAC300ECF582E43417F583E4F0A3F0A27492AFAB
:10BAD30022EF64527043901DC6E0FEA3E0FFD394AF
:10BAE30000EE94004033A2AF9274C2AF901DC4E045
:10BAF300FD75F003A424EBF582E43417F583745247
:10BB0300F0ED75F003A424ECF582E43417F583EE2D
:10BB1300F0A3EFF0A27492AF22901DC4E0FB7A0071
:08BB23007D027F2D12B9012201
:10F0C700901E39EFF09017AEE0FD901E39E0FFC3B8
:10F0D7009D4009EFFB7A007F2F12B901901E39E09E
:10F0E70075F003A424EBF582E43417F583E0FF22DF
:10E5E800901E3AEFF09017AEE0FDFF901E3AE0FC67
:10E5F800FB3395E0FAC3EB9F7480F86A98400AEC05
:10E608003395E0FA7F2E12B901901E3AE0FF339558
:10E61800E0FE9017EC75F003EF1229E7EE75F003B2
:0BE62800A42583F583E0FEA3E0FF22A1
:10EF0000E49017AEF0FFEF75F003A424EBF582E474
:10EF10003417AD82FCF5837449F0A3E4F0A3F0EF5D
:10EF200025E024AFF582E43417F583E4F0A3F00F75
:05EF3000EFB41ED22227
:0DFC9400426174746572794C6F7720200016
:04E22D00411CB4FFDD
:10F4A40012F9FF50207F0512DD5412FDF390FE1B6C
:10F4B400E493600312FE1A12F53B12E09A7F3212B3
:06F4C400EC5712E3CE221A
:10F5ED00125D7F501D7D02E4FF12A1837BFF7AFC2B
:10F5FD0079941237E27F6412EC5712F9FF5003121F
:03F60D00F4A42240
:10F61000125D7F501D7D02E4FF12A1837BFF7AFC07
:10F6200079941237E27F6412EC5712F9FF500312FB
:03F63000E3CE2204
:10FA860090FE1BE493600312FE1AE4FF125DF2126D
:06FA9600FC5F12D488227F
:07FDD10012F98B12C90A228E
:10FA1600C2ABC28EC28F53890F438910758D4CE4D9
:07FA2600F58BD28ED2AB225A
:08FD9C007D327F0C125CD422C1
:08FDA4007D147F05125CD422DE
:10E63300901E24EFF0A3EDF0901E24E0FFC394019D
:10E643004037EFD394105031EBD394014020901C0A
:10E65300B9EFF0901E25E0FF901CB2F0EB14901C74
:10E66300B5F0EF2402FDE433FC7F0512CF9E901E2C
:0AE6730024E0FFA3E0FD125CD422B6
:10F15600901CB9E0FF901CB2E0FD125CD4901CB587
:10F16600E014F0E0D394004010901CB2E02402FDBD
:0FF17600E433FC7F0512CF9E227F0512DD542269
:0EFC5F00901CB6E0FFE4FBFA7D4912BA732256
:07FDD80012FC5F12F4A422EB
:10F98B0012F9FF5012901CB6E0FF901CB0E0FAA3E6
:08F99B00E0FB7D5212BA732259
:09FD6900901CB0EEF0A3EFF022B3
:10FB04007EFD7FD812DB6A901CB6EFF07F8C7E00FE
:04FB140012FD692253
:10D2A500901CB3E024FE601604702312F5ED12F90C
:10D2B500FF402112FA86901CB37402F0801612F911
:10D2C500FF501112FDD1901CB37401F08006901C23
:10D2D500B37401F0901CB8E0146022147037125D2D
:10D2E50089901CB7EFF0600E901CB474FFF0901C91
:10D2F500B7E0FF12F296901CB87401F022125D8916
:10D30500EF700B901CB4E06005E4F012F717901C69
:0CD31500B87402F022901CB87402F022E0
:10F4090012F9FF5008901CB37401F08006901CB3E8
:10F419007402F0125D89EF6007901CB87402F02243
:07F42900901CB87401F022F1
:10B6B700901E26EFF0A3EDF0E0122AC8B6E500B71A
:10B6C7000C01B71802B70003B74304B72405B73016
:10B6D70006B75A07B76908B6F1090000B76C901E9C
:10B6E70026E0FF12FC25E433FF22901E26E0C394D8
:10B6F7002040037FFF227F0022901E26E0FF12FCDE
:10B7070016E433FF22901E26E0FF12F872E433FF9F
:10B7170022901E26E0FF12F4CAE433FF22901E2671
:10B72700E0FF12F4F0E433FF22901E26E0FF6430BE
:10B737006004EFB431037FFF227F0022901E26E0D2
:10B74700FF12FC164007901E26E0B42E037FFF224F
:10B757007F0022901E26E0C3948050037FFF227F44
:10B7670000227FFF22901E27E0FD901E26E0FB7A35
:07B77700007F3012B901222E
:01002A0022B3
:10C308005245534554000C004641554C5420434F68
:10C318004445005052474D204641554C5400502545
:10C328003032627500432530326275004D25303356
:10C33800750043686B52616D436F6E6669670025CF
:10C34800754B6220666F756E64000C546573746972
:10C358006E672020202020002052616D42616E6BA4
:10C3680020202020002530326275002025754B6280
:10C37800206F6B2100436C656172696E673A2020FB
:10C3880020002020202020202020202020200055B0
:0FC39800AA006618E7817E7E81E7186600AA5525
:06FE0500E51724FCFF22BA
:10E3CE0012D9E9E4FF125CA0E4FF125DC5E4FF126E
:10E3DE005DF2E4FF125E057F01125DAEE4F5A8FF6B
:10E3EE00EFB410027F1874082FF8E6FE74B52FF5FF
:10E3FE0082E43416F583EEF00FEFC394F840E17526
:0FE40E00B0FF75A0FF7590FF7580FF7587022224
:0CFCD200E4F588F5C8F589F5A8F5B8221E
:0BFCFF00E51964AA6003D38001C32252
:040016007519AA228C
:04001E0075195522D9
:10F755007BFF7AC37908901CC7122A2A901CCAE439
:0FF76500F0A37405F07B007A00791812DA9B226A
:07FDDF0012FCD21200002209
:10F317007BFF7AC3790E1237E2E4FF125CA0E4FFA9
:10F32700125DF2E4FF125E0512001E12FDDF7B0084
:0AF337007A807D017F3112B90122B6
:10F096007BFF7AC3790E1237E2E4FF125CA0E4FF2D
:10F0A600125DF2E4FF125E0512F7557F01125DAEA6
:10F0B600D29312FFFF7B007A80E4FD7F3112B90103
:01F0C6002227
:10EF3500901DC8EEF0A3EFF0E4A3F0A3F0901DC878
:10EF4500E0FEA3E0FFC3901DCBE09F901DCAE09EAD
:10EF550050117F3212EC57901DCAE475F00112274B
:04EF65009F80DA228D
:10B90100901DCCEFF0A3EDF0A3EAF0A3EBF0E4FF80
:10B91100125E0512FDA412FDA47BFF7AC3790E12FB
:10B9210037E2901DCEE0FEA3E0FFEE30E714547F36
:10B93100901DCEF0EFA3F07BFF7AC379101237E2AE
:10B9410080097BFF7AC3791B1237E27D02E4FF1283
:10B95100A1837BFF7AC37926901DCCE0901AD3F0A6
:10B961001237E27D027F0412A1837BFF7AC3792D16
:10B97100901DCDE0901AD3F01237E27D027F0812BC
:10B98100A1837BFF7AC37934901DCEE0FFA3E090C1
:10B991001AD3CFF0A3EFF01237E27FA07E0012EFAF
:10B9A1003512FDA4901DCCE0B4200312F09612F9DB
:0AB9B100FF500312E3CE12FDDF2267
:10EDBC00901E3BEDF0125BE4EFF4600B7B007A806D
:10EDCC007D3A7F2512B901901E3BE075F008A42412
:10EDDC0097F974C335F0FA7BFF78F87CFF7D017EE0
:07EDEC00007F0812260D2232
:10ED8200901E3CEDF0125BE4EFF4600B7B007A80A6
:10ED92007D3A7F2512B901901E3CE075F008A4244B
:10EDA20097F974C335F0FA7BFF78F87CFF7D017E1A
:0AEDB200007F08122F35EF24FF2226
:101C4C0012F6107D01E4FF12A1837BFF7AC3793A6F
:101C5C001237E212F804206E0575174480037517CD
:101C6C0014206E0EE4FD7F4312EDBCE4FD7F2312C5
:101C7C00EDBC7D017F1312EDBCE4FD7F0712EDBCC2
:101C8C00206E2CE4FD7F4312ED825003751724E483
:101C9C00FD7F2312ED825017E517C39444400D7B52
:101CAC001F7A007D3A7F2512B90180037517147DC8
:101CBC00017F1312ED825017E517C39424400D7B5E
:101CCC000F7A007D3A7F2512B9018003751708E45D
:101CDC00FD7F0712ED82500B7B007A807D017F2205
:101CEC0012B90112F81012FD9C7D02E4FF12A183BF
:101CFC0012FE05EF75F020A4901AD4F0E5F0901ABE
:101D0C00D3F07BFF7AC379471237E27FFA12EC5794
:101D1C007FFA12EC577BFF7AC379521237E27D01BE
:101D2C00E4FF12A1837BFF7AC379601237E212F8C9
:101D3C00047882760112FE057882E6FEC39F502C51
:101D4C00EE2404FF125BE4EFF4600B7B007A807DE1
:101D5C003A7F2412B9017E087F007882E6FD7B0170
:101D6C007A807900122F5978820680C978827601A0
:101D7C0012FE057882E6FEC39F5066EE2404FF1225
:101D8C005BE4EFF4600B7B007A807D3A7F2412B920
:101D9C0001E4901DD2F0A3F0901DD07480F0A3E468
:101DAC00F0901DD0E475F0011227B585F082F58313
:101DBC00E0FF7882E6FEEF6E600BEEFB7A007D0EA4
:101DCC007F2212B901901DD3E004F07006901DD251
:101DDC00E004F0C3901DD2E0940840C578820680E0
:101DEC008F12F81012F61012F8047882760112FE97
:101DFC00057882E6C39F4003021F2E7D017F0812E7
:101E0C00A1837BFF7AC3796D7882E6901AD3F012A6
:101E1C0037E27D02E4FF12A1837882E62404FF12EC
:101E2C005BE4EFF4600B7B007A807D3A7F2412B97F
:101E3C00017E087F0090C398E493FD7B017A807942
:101E4C0000122F59E4901DD2F0A3F0901DD0748095
:101E5C00F0A3E4F0901DD0E475F0011227B585F0E5
:101E6C0082F583E0FF90C398E493FEEF6E600B7BEA
:101E7C00007A807D0F7F2212B901901DD3E004F00F
:101E8C007006901DD2E004F0C3901DD2E09408407F
:101E9C00C37E087F0090C397E493FD7B017A807921
:101EAC0000122F59E4901DD2F0A3F0901DD0748035
:101EBC00F0A3E4F0901DD0E475F0011227B585F085
:101ECC0082F583E0FF90C397E493FEEF6E600B7B8B
:101EDC00007A807D107F2212B901901DD3E004F0AE
:101EEC007006901DD2E004F0C3901DD2E09408401F
:101EFC00C37BFF7AC379737882E62401FFE433FE57
:101F0C00EF7805C333CE33CED8F9901AD4F0EE90D7
:101F1C001AD3F01237E212FD9C12F61078820602E8
:101F2C001DFA12F8107FFA12EC577FFA12EC5712C6
:101F3C00F610E4FDFF12A1837BFF7AC3797D123783
:101F4C00E27D01E4FF12A1837BFF7AC37960123733
:101F5C00E27D02E4FF12A1837BFF7AC3798A1237F8
:101F6C00E27882760112FE057882E6C39F50491210
:101F7C00FD9C7D017F0812A1837BFF7AC3796D786C
:051F8C0082E6901AD36B
:101F9100F01237E27882E62404FF125BE4EFF4608A
:101FA1000B7B007A807D3A7F2412B9017E807F000D
:101FB1007D007B017A807900122F5912F610788208
:0E1FC1000680AD7FFA12EC577FFA12EC572221
:05000600A26D926C22C6
:03FE0F00A26C22C0
:10F8F500EF6005438F018003538FFEE58F30E003F2
:0AF90500D38001C3926D1287242203
:0DFCA100EF6003D38001C3926B12F8F522CF
:09FD7200A26BE433FF12F8F52244
:10D9CA007F2F12DA1B7FA312DA1BAF6C12DA1B7FCE
:10D9DA00A012DA1B7FC812DA1B7FAF12DA1B227F72
:10D9EA00AE12DA1B7FA512DA1B22E9C0E079009099
:10D9FA0080FAE030E702D9F7D0E0F92212F804EF12
:10DA0A00C0E07F03125BE4D0E09080F9F012F810D6
:10DA1A002212F804EFC0E07F03125BE412D9F490FB
:09DA2A0080F8D0E0F012F810229F
:10824900D292D2950000306D050000000000C29264
:108259000000306D050000000000C2952275F0088D
:10826900EF339292306D0100D295000000306D0617
:10827900000000000000C295306D020000D5F0E159
:10828900D29212828F22306D020000D29500003006
:108299006D050000000000A292306D03000000C2CD
:1082A9009522C292306D020000D2950000306D0512
:1082B9000000000000D29222EFC2E0FF12824912B0
:1082C900826622EFD2E0FF1282491282662212826E
:1082D9006622EF20E706D2E7FF12826622EF20E747
:1082E9000312826622D29275F008306D03000000F5
:1082F900D2950000306D050000000000A292000038
:10830900306D050000000000C2950033D5F0DBF99F
:1083190000306D080000000000000000C29200005B
:10832900306D050000000000D2950000306D050099
:1083390000000000C295D292E9FF22D29275F0089E
:10834900306D03000000D2950000306D050000007B
:108359000000A292306D0100C295306D010033D545
:10836900F0DEFF00306D0700000000000000D2922F
:108379000000306D050000000000D2950000306D4E
:10838900050000000000C29522D292D29522D29215
:1083990075F008306D03000000D2950000306D05BE
:1083A9000000000000A292306D0100C295306D01FD
:1083B9000033D5F0DEFF306D020000D292000030AC
:1083C9006D050000000000D2950000306D05000029
:0683D900000000C2952225
:0A00300031393935204D2E532E00D2
:071FE000C293FFFF020000A5
:105BE400EFB40500403AB5170040037F0022C39488
:105BF4000475F01084FF306E04B2F2B2F3E5F0C421
:105C0400A2E492E3A2E592E4C2E5F454D8C2AF530D
:105C14001F27421F759076908000E51FF0EF240443
:105C2400C2AF531EECC403905C2F73431E03851E46
:105C3400908036431E11851E90802E431E12851EB1
:105C4400908026431E13851E90801E431E10851EC1
:105C5400908016431E00851E90800E431E01851EF3
:105C6400908006431E02851E90D2AF7FFF22C08320
:105C7400C08212F804125BE4908000EDF012F81078
:105C8400D082D08322C083C08212F804125BE490D5
:105C94008000E0FF12F810D082D08322BF040050AD
:105CA4002E531FFCBF0108431F027564018019BFF6
:105CB4000208431F01756402800EBF0308431F03DB
:105CC40075640380037564007F02AD1F125C722249
:105CD400ED6069FEEF60657F0014905D4193F97C8F
:105CE40000FD1200260EE92323FCFD530403530593
:105CF400FC6304FF6305FFC2AF5389F04389018C41
:105D04008C8D8AC28DD28C308DFDC28C306D0D8C01
:105D14008C8D8AC28DD28C308DFDC28C306E0BB2CC
:105D240094DFDCDEDAD2AFD29422B2B5DFD1DECF9B
:105D3400D2AF7F003076027FFF125DC522EDD3BC67
:105D4400B19E8C7D75685D574E453D3A33BF000466
:105D5400D2B48007C2B47F0112EC5722306E09BF5F
:105D64000003D2B522C2B522BF0003D2B422C2B40A
:105D7400227F01125C89EFA2E3B3227F01125C89C6
:105D8400EFA2E0B3227F01125C89EF30E50920E441
:105D94000920E1097F03227F00227F01227F022262
:105DA4007F01125C89EFA2E2B322BF0005531FEF0B
:105DB4008003431F107F02AD1F125C7222A296B3B0
:105DC40022306E1DBF000D531FDF7F02AD1F125C1A
:105DD40072C27622431F207F02AD1F125C72D276FC
:105DE40022BF0005D2B5C27622C2B5D27622BF0048
:105DF40005431F048003531FFB7F02AD1F125C7217
:105E040022E56BB455028008B466028003306E0E3E
:105E1400BF0003D2B422C2B47F0112EC5722BF00E8
:105E24000B531FDF7F02AD1F125C7222431F207FC2
:105E340002AD1F125C7222306E03A2B3227F0012E5
:105E44005C89EFA2E7B322EFB4080050145363F85F
:105E54004263AD637F00306E027F01125C727FFF8C
:105E6400227F0022900000E4F0A3E58330E7F822CB
:105E74009000007A007B007900E0A36AFAE0A36B4B
:105E8400FBD9F6E58370F2EA4B60037F00227FFFC3
:015E940022EB
:10EC5700EF60167FE4DFFE7FE4DFFE306D087FE4C0
:10EC6700DFFE7FE4DFFE1470EA22EF6008DFFE308C
:06EC77006D03FFDFFE2229
:109A1B0012F8047F01125BE4EFF4600AE4FBFA7DB9
:109A2B00017F4212B901908000E030E603D3800140
:109A3B00C39251908000E030E703D38001C3925270
:109A4B007F03125BE4EFF4600AE4FBFA7D037F40D3
:109A5B0012B9019080FAE0540F7003D38001C392C6
:109A6B0053908004E020E203D38001C39254908092
:109A7B0000E020E003D38001C39255908000E020EA
:109A8B00E103D38001C3925612F8102051092052E2
:109A9B000620B3037F662220511520521230B30FDC
:109AAB0030530C2054092055062056037F1C2220CE
:109ABB00510F20520C30B3093053063054037F1A28
:109ACB002220511220520F30B30C3053093055065F
:109ADB003056037F1B2220511520521230B30F201A
:109AEB00530C2054092055062056037F3B2220514E
:109AFB001220520F30B30C20530930550630560349
:109B0B007F3A222051063052037F22223051062009
:109B1B0052037F4A223051092052063054037F4BA7
:0A9B2B00223051053052027F55220E
:10FBD900129A1B8F6BEFB42203D38001C3926E225A
:10FA2D00E56B6455600FE56B643A6009E56B643B0B
:07FA3D006003D38001C32226
:040026001227142267
:10CBDD00010001010101010000000001010000013F
:10CBED00010100010100010001010101010100002D
:10CBFD00010100010100010100010101010101001C
:10CC0D00010100000001010101010101010101010A
:10CC1D0001000101010101010101000101000000FC
:10CC2D0001000100000101000101010000010101ED
:10CC3D0001010100000101010001000101010001DC
:10CC4D0001010101010001010000010001010101CB
:0CCC5D00010101010101000101010101C0
:10F0F70012FA2D502A7D087F1012A183E4901E3D3D
:10F10700F0E4FF12DA06901E3DE004F0E0D39460CD
:10F1170040EF901CFFE0FF901D00E0FD12A183224D
:108F5F00901CF2122A2A12FA2D40030290A67D08C5
:108F6F007F5512A183901CF21229F3122633701829
:108F7F00901CF5F0E4FF12DA06901CF5E004F0E027
:108F8F00C3941C40EF029099901CF21229F3122601
:108F9F003324D0901CF7F090000112264C24D0906F
:108FAF001CF8F090000312264C24D0901CF9F0907E
:108FBF00000412264C24D0901CFAF0E4901CF5F01B
:108FCF00E4901CF6F0901CF6E0FFC39407400302F8
:108FDF00907E901CF5E0FE600464027053EE700901
:108FEF00EF7006901CF6E004F0EE700C901CF7E0AA
:108FFF007006FF12DA06806E901CF5E024F7F582FA
:10900F00E4341CF583E075F007A424DDF582E43425
:10901F00CBF583C083C082901CF6E0D082D083252D
:10902F0082F582E43583F583E493FF12DA06803606
:10903F00901CF5E024F7F582E4341CF583E075F01D
:10904F0007A42423F582E434CCF583C083C0829037
:10905F001CF6E0D082D0832582F582E43583F58338
:10906F00E493FF12DA06901CF6E004F0028FD4901E
:10907F001CF5E0B401057F0112DA06901CF5E0043F
:10908F00F0E0C394045003028FCF901CFFE0FF90D9
:08909F001D00E0FD12A1832277
:10F43000901E3EEFF012FA2D501C7D087F1012A195
:10F4400083901E3EE0FF12DA06901CFFE0FF901D45
:07F4500000E0FD12A1832280
:10E4B800901DF9122A2A12FA2D50417D087F201248
:10E4C800A183901DF91229F3122633FF12DA069060
:10E4D8001DF91229F390000112264CFF12DA06905A
:10E4E8001DF91229F390000212264CFF12DA069049
:0DE4F8001CFFE0FF901D00E0FD12A183223B
:10DF2F00901DFC122A2A12FA2D50517D087F2E12B5
:10DF3F00A183901DFC1229F3122633FF12DA0690EB
:10DF4F001DFC1229F390000112264CFF12DA0690E5
:10DF5F001DFC1229F390000212264CFF12DA0690D4
:10DF6F001DFC1229F390000312264CFF12DA0690C3
:0DDF7F001CFFE0FF901D00E0FD12A18322B9
:10F45700901E3FEFF012FA2D501C7D087F3D12A140
:10F4670083901E3FE0FF12DA06901CFFE0FF901D1D
:07F4770000E0FD12A1832259
:10DE7300901E28EFF012FA2D50547D087F5112A105
:10DE830083901E297403F0901E29E0FFD394004071
:10DE93001B901E28E09F50077F0112DA068005E4DD
:10DEA300FF12DA06901E29E014F080DB901E28E0B2
:10DEB300C3940450077F0112DA068005E4FF12DAE7
:0FDEC30006901CFFE0FF901D00E0FD12A18322DE
:1087060012871012871312872122C2AC22C29CC282
:108716009822D2AC22D29C22D27722C27722AF6094
:10872600AD61AB62128738228F608D618B621287D2
:108736003822BF0B005050BD0500504BBD040ABB8C
:108746000145755F08C2D5800EBB02005039ED2386
:108756002BF55FA2E092D5C2ACC2AD75980075C884
:1087660030EF23908790306D039087A693F5CBEF7B
:10877600230493F5CAEFC4425FD29EA2D55387BFA6
:10878600929FD2CA7FFF227F0022FB80FDC0FEE0BF
:10879600FF70FFB8FFDCFFEEFFF4FFF7FFFAFFFD07
:1087A600F700FB80FDC0FEE0FF70FFB8FFDCFFE8CE
:1087B600FFEEFFF4FFFAE55F540F239087C5738041
:1087C60010802F80178034801D8038801F8039806C
:1087D6003CEFC2E7A2D0B392E7F59922EFC2E7A237
:1087E600D092E7F59922EFD2E7F59922EFC2E7F5A5
:1087F6009922EFA2D0B3929BF59922EFA2D0929B39
:10880600F59922D29B8F9922C29B8F99228F99220A
:10881600AF99E55F540F23908821738010803080D4
:108826001580358019803A801E803C803FEFA2D0AB
:10883600B3547FFF803AEFA2D0C2E7FF8032EFA2A7
:10884600E7B3C2E7FF8029EFA2E7C2E7FF8021EF87
:10885600A29A20D01BB38018EFA29A30D012B38010
:108866000FEFA29AB38009EFA29A8004EFC38000AB
:0C887600D2694004129B352212FD8422BE
:10EC7D0030770412FE1522309805C298128816308E
:08EC8D009905C29912FBA922AE
:0DE23100421CFB0000411D0200411D0300C6
:10A18300901DD4EFF0A3EDF012FA2D400302A28745
:10A19300901DD5E0FF64086014901DD4E0C39410B3
:10A1A300400302A287EF6408700302A287901D0395
:10A1B300E070047E0180027E00EF640860047D018C
:10A1C30080027D00ED5E600B901DD4E0901CFFF0DB
:10A1D300A3EFF0EF6408600D901DD4E075F006A4C2
:10A1E300F0E02410F0901DD4E0FEC4540F4410900E
:10A1F3001DD6F0EE540FA3F0EF70167FB012DA1BEA
:10A20300901DD6E0FF12DA1B901DD7E0FF12DA1B78
:10A2130022901DD5E0B401167FB112DA1B901DD632
:10A22300E0FF12DA1B901DD7E0FF12DA1B22901D0C
:10A23300D5E0B402167FB212DA1B901DD6E0FF12EE
:10A24300DA1B901DD7E0FF12DA1B22901DD5E0B474
:10A2530003167FB312DA1B901DD6E0FF12DA1B90B0
:10A263001DD7E0FF12DA1B22901DD5E0B408157F3D
:10A27300B812DA1B901DD6E0FF12DA1B901DD7E04F
:05A28300FF12DA1B22AE
:10E67D008F6574E02565F565E4F566E565FD901C2F
:10E68D00FCE02DFD901CFBE034008D82F5837406BB
:10E69D001229D6E5822566F582E43583F583E58278
:10E6AD0024FEF582E5833455F583E493FF12DA06F3
:0AE6BD000566E566C3940640C2221C
:09FD7B00901CFBEEF0A3EFF02256
:07FDE6007BFF7AFE790B227E
:10E09A00E4F567E56724B0FF12DA1B7F1112DA1B79
:10E0AA00E4FF12DA1BE4F568E4FF12DA06E4FF1271
:10E0BA00DA06E4FF12DA06E4FF12DA06E4FF12DAFD
:10E0CA0006E4FF12DA06E4FF12DA06E4FF12DA06C1
:10E0DA000568E568C3940C40CFE4FF12DA060567C9
:08E0EA00E567C3940440AC2279
:10F18500901D02E0F47027901CFFE0C39410501E00
:10F1950012E67D901CFFE0FFA3E0FD12A183901C09
:0FF1A500FFE0901CFDF0901D00E0901CFEF0229A
:10EDF300901D02E0F4702F901CFFE0C39410502686
:10EE0300901D0374FFF0901CFDE0FFA3E0FD12A131
:10EE130083E4901D03F07F2012E67D901CFFE0FF4A
:07EE2300A3E0FD12A1832210
:10A48600901E40EFF012FA2D4006901E40E0FF228B
:10A49600901E40E0C394204027901CFFE09410508B
:10A4A6001C12EDF3901CFFE004F0901E40E0FF123A
:10A4B600E67D7F5F12F185901E40E0FF227F00223D
:10A4C600901E40E0B40C1112E09AE4FDFF12A18345
:10A4D6007F5F12F18502A57B901E40E0B40A1C90B6
:10A4E6001D00E0045403F012EDF3901D00E0FDE4BE
:10A4F600FF12A1837F5F12F185807A901E40E0B43F
:10A506000D1412EDF3901D00E0FDE4FF12A1837F10
:10A516005F12F185805F901E40E0B4070512FDA42E
:10A526008053901E40E0B4081D901CFFE0600214AA
:10A53600F012EDF3901CFFE0FFA3E0FD12A1837F74
:10A546005F12F185802F901E40E0B40113901D022A
:10A55600E0B4FF217F2012F185E4901D02F0801502
:10A56600901E40E0B4020E12EDF3901D0274FFF04F
:0BA576007F5F12F185901E40E0FF2285
:10E71000901E41EFF0E024806009147017E56C242E
:10E7200080FF22901D01E0F56CAF6C12DA1BE56CE6
:10E730002480FF22901E41E0FFC394004015EFD3D8
:10E74000940F500FEF2480F56CFF12DA1B901E41DE
:09E75000E0FF22901E41E0FF22CF
:08FDAC00030913030F152B00DE
:0300030002C4DF55
:03000B00C2A93255
:03001300C2AA324C
:03001B0002C4F923
:0300230002C543D0
:03002B00C2AD3231
:10C4DF00C28CC0E0C0F0C0D0C083C08212FE12D0A8
:10C4EF0082D083D0D0D0F0D0E032C000C001C002E3
:10C4FF00C003C004C005C006C007C0D0C0E0C082E2
:10C50F00C083C0F0C28EE58B2400F58BE58D344CD3
:10C51F00F58DD28E12D1A9D0F0D083D082D0E0D0B9
:10C52F00D0D007D006D005D004D003D002D001D090
:10C53F0000C28F32C000C001C002C003C004C005DA
:10C54F00C006C007C0D0C0E0C082C083C0F012ECEC
:10C55F007DD0F0D083D082D0E0D0D0D007D006D01D
:0CC56F0005D004D003D002D001D000326F
:10F80400D083D082E51E44ECC0E0E473D083D08280
:0CF81400D0E0431E13521E851E90E473CA
:0300000002BB2B15
:10BB2B0075A800C29375B0FF751E74851E9075D0F5
:10BB3B0000756E007808B81802782074AD28F5826D
:10BB4B00E43416F583E0F608B800EB758182756D69
:09BB5B000090768CC082C08322A8
:10BB640022E493A3F8E493A34003F68001F208DFF0
:10BB7400F48029E493A3F85407240CC8C333C454B1
:10BB84000F4420C8834004F456800146F6DFE48065
:10BB94000B010204081020408090E1EDE47E019343
:10BBA40060BEA3FF543F30E509541FFEE493A36035
:10BBB400010ECF54C025E060A840B8E493A3FAE492
:10BBC40093A3F8E493A3C8C582C8CAC583CAF0A3E3
:0EBBD400C8C582C8CAC583CADFE9DEE780BEE5
:01E23E0000DF
:01FE1B0000E6
:01FE150022CA
:01FE160022C9
:01FE170022C8
:01FE180022C7
:01FE190022C6
:01FE1A0022C5
:02002E00274D5C
:01FFFF000001
:0200FF00111CD2
:04FE0B003733340055
:03FE1200C2A82261
:10E041000C54657374696E67202020202000436C96
:10E051006F636B2020204265616D0042757A7A659D
:10E06100722020204B6579000C44617465202620C4
:10E0710054696D65200025303262753A253032626F
:10E08100753A2530326275000C257300202020205E
:09E0910020202020202020200086
:10A67A0012FD9C7BFF7AE079411237E27D01E4FF0B
:10A68A0012A1837BFF7AE0794F1237E27D02E4FF61
:10A69A0012A1837BFF7AE0795C1237E27FFA12EC2F
:10A6AA00577FFA12EC577FFA12EC5712FB7712FD1A
:10A6BA009C7BFF7AE079691237E27B017A1B79EE9B
:10A6CA0012AF8378E47C1B7D017B017A1B79EE7ED5
:10A6DA00007F0812260DE4901BEDF07D017F011228
:10A6EA00A1837BFF7AE07977901BF0E0901AD3F090
:10A6FA00901BEFE0901AD4F0901BEEE0901AD5F080
:10A70A001237E27D027F0312A1837BFF7AE0797719
:10A71A00901BF2E0901AD3F0901BF3E0901AD4F059
:10A72A00901BF4E0901AD5F01237E27B017A1B797C
:10A73A00EE12AF8312F610901BEDE004F0E0C39422
:10A74A00A4409812FD9C78E47C1B7D017B017A1B56
:10A75A0079EE7E007F08122F35EF700AFB7A807D32
:07A76A00377F1F12B9012225
:10768C00D2BC12870612FCFF400302780D12001EBA
:10769C007FFF12FCA1120006125E6812BB9D12FB4A
:1076AC00D9D2AF12F95A12D9CA7D087F1012A18310
:1076BC00E4901BEDF0E4FF12DA06901BEDE004F011
:1076CC00E0D3947040EFE4FF125DC5E4FF125CA0C0
:1076DC00900100E493656B600B7B007A807D047FE6
:1076EC002012B9017BFF7AFE790B901AD3122A2A49
:1076FC007AE079891237E2121C4CE4FDFF12A18367
:10770C007BFF7AE0798D1237E27D01E4FF12A183D1
:10771C007BFF7AE0798D1237E27D02E4FF12A183C0
:10772C007BFF7AE0798D1237E2E4FB7D017F051255
:10773C00872E12FE1612E9DB12EF0012FAF012FB82
:10774C005312BF3312FB0412F3E27C8B7D5DE4FF1A
:10775C0012CB4E7CD27DA57F0112CB4E7CD77D3DCA
:10776C007F0212CB4E7CDA7D337F0312CB4E7C80B2
:10777C007DAF7F0412CB4E7CF17D567F0512CB4E34
:10778C007C587DFE7F0612CB4E7CF17DB47F0712B8
:10779C00CB4E7C007D127F0812CB4E7C007D1A7F75
:1077AC000912CB4E7CEE7D607F0A12CB4E7CFE7DA7
:1077BC00177F0B12CB4E7F0112DCF37F0212DCF32E
:1077CC007F0312DCF37F0412DCF312F61012F9D1F2
:1077DC0012A67A12F8DBE4FF125DC5E4FF12FCA1DD
:1077EC0012C61612FA16901BEC74FFF01200161249
:1077FC00FCFF50367B007A807D387F1F12B90180E8
:10780C002912FA1612FA707F0212EC5712D9CA1208
:10781C00F8DB12FD72EF700AFB7A807D397F1F1244
:10782C00B90112F655E4901BECF012F40912F98B25
:10783C0012F88DD2AF901BECE0700812F9FF4003E8
:09784C0012FA8612FDCA80FB222B
:101FE700EC4D6011E8497017ED33EC3304600DE4F4
:101FF700FCFFFEFD22E933E8330470F802218F125B
:10200700215A58046009E4CC24815006285009025B
:102017002199284003022196C0E0EB4A7044B98019
:1020270006D0E0FB022185EF4E701CBD8008EBFF58
:10203700EAFEE9FD80EBE98DF0A4FEE5F00220D091
:10204700E9CDF9EAFEEBFFEF89F0A4FCE5F0CE89D4
:10205700F0A42EFFE435F0CD89F0A42DFEE435F091
:102067008067EF4E7005BD80D780C3EF8BF0A4ACBF
:10207700F0EE8BF0A42CFCE435F0F8EF8AF0A42CFA
:10208700E5F038FCE433CB8DF0A42CFCE5F03BF80D
:10209700EE8AF0A42CFCE5F038F8E433CF89F0A4FD
:1020A7002CFCE5F038CF3400CE89F0A42FFFE5F003
:1020B7003EFEE433C98DF0A42EFEE5F039CD8AF05B
:1020C700A42FFFE5F03EFEE43DFD33D0E0FB5007D3
:1020D7000BBB000F022199EC2CFCEF33FFEE33FE14
:0620E700ED33FD02217142
:1020ED0074F8CC6480CCC86480C8F582046043C3A6
:1020FD00EB9FF5F0EA9E42F0E99D42F0E89C45F039
:10210D0060305018E5825FFFE582F42B5582FB505D
:10211D00210ABA001D09B90019088016E5825BFB7A
:10212D00E582F42F5582FF50090EBE00050DBD004E
:10213D00010CC3EB9FF5F0EA9E42F0E99D42F0E8F9
:0D214D009C45F06007CC4820E701B3EC2270
:10377700E55A24D3F582E4341AF583E0055A2290FA
:103787001AD0304F03901AD3E475F0011229FC02C6
:1037970026332048E97F2ED2488018EF540F249013
:1037A700D43440D4FF304C0BEF24BFB41A0050037D
:1037B7002461FFE55B6002155B055EE55E7002054F
:1037C7005D304F0E901AD0E475F0011229FCEF021C
:1037D70026CE02A4867403D24F8003E4C24FF55A63
:1037E700901AD0122A2AE4F55BF55DF55EE55B6079
:1037F700077F201237BA80F5755CFFC249C248C2FD
:103807004AC24BC24DC24EC250123786FF700D30AE
:103817004F057F001237CBAF5EAE5D22B4255FC286
:10382700D5C24C123786FF24D0B40A00501A75F05F
:103837000A785B30D50508B6FF0106C6A426F62030
:10384700D5047002D24B80D924CFB41A00EF5004AC
:10385700C2E5D24C023ACBD24980C6D24880C0D208
:103867004A80BCD2D580BAD24D80B47F201237BAF5
:10387700204A077401B55B0040F1123777FF123712
:10388700BA0237F4D250D24E8095123777FB1237EF
:1038970077FA123777F94A4B700679C97A3B7BFF7B
:1038A700204A3BE55B60377E00E9C0E02EF9EAC0BD
:1038B700E03400FA122633F9D0E0FAD0E0C9600606
:1038C7000EEE655C70E3C2D5EBC0E0EAC0E0E9C08C
:1038D700E0EE123B2CD0E0F9D0E0FAD0E0FB122664
:1038E70033FF609DEBC0E0EAC0E0E9C0E01237BA01
:1038F700D0E02401F9D0E03400FAD0E0FBE55C0425
:1039070060DCD55CD9023888D24A8094123B0E60BD
:10391700F7E55C7001041221A4A95C600DE55C6009
:103927000914F55C123BB6EF60F3EA30E702F404E2
:10393700C3995079EAF4255C0430E701E404F55CA7
:10394700800D123B0E60C1EA055C255C1221A4EADA
:10395700901AFFF030E701E4255C04D55C04204DA4
:103967000114123B2CE4C0E0123BB6901AFFE06052
:103977001320E70714F01237A2802204F0D0E014D6
:10398700C0E07F001237A2E55C6007123799155C2B
:10399700800B304D03123799D0E00237F4D0E004A2
:1039A70080C4123B0E609EE55C041221A4901AFFAE
:0639B700EAF0E55C204D82
:1039BD00026001042404123B2C74FF04C0E0123B8E
:1039CD00B61237A2E55C204D026003123799D0E0A4
:1039DD00B55CE87F451237AC901AFFE07F2B30E7DE
:1039ED00047F2DF404C0E01237BAD0E075F00A84DC
:1039FD00C0F01237A3D0E01237A30237F47910804C
:103A0D00027908C24EC2508008D2D5790A80047955
:103A1D000AC2D5E55C047002F55CE4FAFDFEFF1206
:103A2D003777FC7B08204913123777FD7B10304820
:103A3D000A123777FE123777FF7B20EC3382D5924F
:103A4D00D55013C3E43048069FFFE49EFEE42049A1
:103A5D00039DFDE49CFCE4CBF8C249EC700CCFCE89
:103A6D00CDCCE824F8F870F38017C3EF33FFEE33B5
:103A7D00FEED33FDEC33FCEB33FB994002FB0FD82D
:103A8D00E9EB304905F8D0E0C448B249C0E00AEC92
:103A9D004D4E4F78207B0070C2EAB55C0040BCC033
:103AAD00E0123B2ED0F0D0E0204904C4C0E0C4B2F7
:103ABD0049C0F01237A3D0F0D5F0EB0237F4122A3B
:103ACD00C83891533A0A5838624C385E423A0E4F14
:103ADD003A16443A16493877433A1C55394946390E
:103AED00A9453913473BE95038662D386A2E388D74
:103AFD002B386E23388B203BD72A382648000038C8
:103B0D0085E55CB4FF03755C06123777FC123777D9
:103B1D00FD123777FE123777FF901AF80221E179FF
:103B2D000AA2D5204B14304D09B910020404B9086E
:103B3D000104A2D5204E02500104204A68924AB5D4
:103B4D005B005034C0E07F20304B197F30A24A72A9
:103B5D004E724D500F123B85C24AC24EC24DC250DD
:103B6D007F30800F304D03E9C0E01237BA304D037E
:103B7D00D0E0F9D0E0B55BCC304D177F30B9100CEB
:103B8D001237BA7F58304C077F788003B90803127B
:103B9D0037BA304A057F2D0237BA7F202050F87F83
:103BAD002B204EF322924A80CF7F00B40700500B9A
:103BBD0024F8F582E4341AF583E0FF22286E756C43
:103BCD006C29002D50434958D2491237773049F8A6
:103BDD00C249785B30D50108F602382612377724B2
:103BED0003B405004001E4903BD0931237AB743A17
:0B3BFD001237ABD24B755B04023A0A92
:104C7200E508305A0104F823282403F582E4341BA2
:104C8200F58322901B00305A03901B03E475F00158
:104C92001229FC02263360EAC50C7002150B14C5FA
:104CA2000C205A04FF02FDB4901B0074FFF5F002C1
:104CB2002A13FF02FB2CE5096006D509037F0022B7
:104CC200205A0F12FB18EF6008050CE50C70020564
:104CD2000B22901B00E475F0011229FC122633FF0F
:104CE20080E4124CC2EFC0E0124CB4D0E040F3803A
:104CF200A5D25A8002C25A901B00122A2AE4F50A4F
:104D0200F508F50BF50C750900C259C257C258C215
:104D12005B124C85FF7005AF0A7E0022B42530126B
:104D22004C85FF24D0B40A00500C75F00AC509A4C2
:104D32002509F50980E924CFB41A00EF5002C2E533
:104D4200024F90D25880D8D25780D4D25B80D0EF15
:104D5200124CB45008124CE4EF600E80A9EFC0E090
:104D6200124CC2D0E06F609EEF6074124C9880A724
:104D7200124CC2EF6069E509700705098003124C05
:104D8200C2EF6014205B0E124C72E475F00112291E
:104D9200FCEF1226CED509E6205B040508050A8041
:104DA200BA124CB8EFC0E0124CB4D0E05004124C2E
:104DB20098E4FF205B0E124C72E475F0011229FC9C
:104DC200EF1226CEEF70DA205B040508050A808B0D
:104DD200E50960020509124CE4124CB8EF70C630C6
:104DE2005A04E4124C98E50A6003024D197EFF7FD3
:104DF200FF22E50960020509124CE4D25DD25C1281
:104E02004CB8EF305D0260D7C0E0124C98D0E0ACF5
:104E12000DAD0EAE0FAF1012AB3F8C0D8D0E8E0F7F
:104E22008F105007124CC2C25C80D4205B10205CF1
:104E320002050A124C721229F30508122967024D63
:014E42000867
:104E4300D0E0809A7900800A791080067908800280
:104E5300790AD25CE50960020509E9C0E0124CE475
:104E6300EF60DD124CC2BF2D04D2598003BF2B0962
:104E7300124CE4EF60CA124CB8D0E0B40A0280339B
:104E8300B40802802EBF302770027408C25CC0E0F1
:104E9300124CB8D0E0BF78028003BF58160509D57D
:104EA30009028007D50904D25C800B741080197045
:104EB30002740ABF000AEFF8E4FCFDFEFF024F4351
:104EC300C0E0EF124C98D0E0F9E4FCFDFEFFE9C02E
:104ED300E0ECC0E0EDC0E0EEC0E0EFC0E0124CB8A3
:104EE300EFF8D0E0FFD0E0FED0E0FDD0E0FCD0F062
:104EF300E8604DB461004007B47B005002C2E52472
:104F0300D0503DFA24F6500724F95034240AFAEA23
:104F1300B5F000502BCFA9F0A42FFF92D5E9C5F02F
:104F2300CEA4A2D53EFE92D5E9C5F0CDA4A2D53D2F
:104F3300FD92D5E9C5F0CCA4A2D53CFCC25C808E21
:104F4300E8C0E0205B2A205C08050A3059031229D7
:104F530022124C721229F3050820570B20580DEE2C
:104F63008FF01227CB80091229678004EF1226CE17
:104F7300D0E0124C98024D08205B10124C7212299B
:104F8300F30508E50B850CF01227CB80E8122AC83D
:104F93004DD2534E4B584D494C4D45424D21484EF1
:104FA3004F4F4E53444D72434E47494E53554DF464
:104FB300464DF4454DF4474D4D2A4F7B4E00004D71
:014FC300519C
:10E75900D25D901DFF122A2A12E795C0E0FF12FB35
:10E769002CD0E040F312AB3F400122ECC0E0EDC0F9
:10E77900E0EEC0E0EFC0E012E795D0F0AFF0D0F0E6
:10E78900AEF0D0F0ADF0D0F0ACF080D9E475F00186
:09E79900901DFF1229FC02263339
:10215A00E9D2E7C933E833F892D5EDD2E7CD33ECCB
:07216A0033FC5002B2D52244
:10217100EC30E7100FBF000C0EBE00080DBD0004CF
:102181000BEB6014A2D5EB13FCED92E7FD2274FF7B
:10219100FCFDFEFF22E480F8A2D574FF13FC7D80D4
:0321A100E480EFE8
:1021A400F920E73624F950037907E4F42402FBE527
:1021B40082158270021583DBF6E024FB501BE96074
:1021C40014E4F0E582158270021583E004F0B40A89
:0D21D40008E4F0D9EE7401F00A22C2D52211
:1021E100ED33EC3392D5FA602AB4FF33EDC2E77BCD
:1021F100FF60067A227906E4227A22790F20D5043B
:102201007A22790A224E614E002B494E46002D4911
:102211004E4600E47A08F0A3DAFC7B00740722C082
:1022210083C082ECC0E0EDC0E0EEC0E0EFC0E0EAC8
:1022310075F010A4CAABF075F04DA42BFBE435F09A
:10224100FCEA2410FAEB34C5FBEC34D9FCEDC2E70F
:10225100FF75F056A4F42411C5F0F434C58FF0A431
:102261002AE5F03BE43CF020E7141224FDD0E0FF26
:10227100D0E0FED0E0FDD0E0FC1223E18014F404B4
:102281001224FDD0E0FFD0E0FED0E0FDD0E0FC1252
:102291001FE7D082D083E0FAEDD2E7CD33EC3324CF
:1022A10082FBE4C3CF33CFCE33CECD33CD33DBF39B
:1022B1007B0775F00A846004F0A31B0AE5F0F0A324
:1022C1008FF0740AA4FFACF08EF0740AA42CFEAC5B
:1022D100F050010C8DF0740AA42CFDE435F0F0A34C
:0522E100DBDE740722A2
:10AB2C00C25EC25FC260C261F9E4F569F56AFCFD00
:10AB3C00FEFFE9105DEA20600CB42D04D260D32234
:10AB4C00B42B02D32224D0504794095041240A300C
:10AB5C006115F8856AF0740AA42872E74051C5F0B3
:10AB6C00704D85F06AD322D25FC0E0E4FBFA792005
:10AB7C007841121FE7ECF8EDF9EEFAEFFBD0E0FCB0
:10AB8C00E41224991222ED305EB41569D322240A02
:10AB9C00206120B4FE07205E1AD25ED32224EB6023
:10ABAC000424E0700EA260925ED261C260D322C314
:10ABBC0002218FE430610BE56A306002F404A25E7E
:10ABCC009260305FEA256920D2E5A2E792615002DB
:10ABDC00F404B4260050D8CCC0E0EDC0E0EEC0E0E8
:10ABEC00EFC0E0EC1224FDD0E0FFD0E0FED0E0FDA1
:10ABFC00D0E0FC206105121FE780031223E13060D6
:06AC0C000312247EC322A6
:1022E60002218FE86480F8E933E83360110460F076
:1022F600ED33EC337009E8FCE9FDEAFEEBFF22045E
:1023060060DED3EB9FEA9EE99DE8C2E78CF0C2F758
:1023160095F0400CE8CCF8E9CDF9EACEFAEBCFFB24
:1023260012215A85D0F05804700320D5B3E8047002
:10233600075002B2D502219992D5EC0460F7E4CC9D
:10234600C0E0C398F8603B94186008400DD0E0FBED
:10235600022171E4FBFAC9FC8028E830E406E4C9EE
:10236600FBE4CAFCE830E305E4C9CACBFCE8540741
:102376006010F8C3E913F9EA13FAEB13FBEC13FC4C
:10238600D8F130F52FC3E49CFCEF9BFFEE9AFEEDEF
:1023960099FDD0E0FBEF4E4D4C701222DB0302217B
:1023A60096EC2CFCEF33FFEE33FEED33FDED30E71C
:1023B600EB022171EF2BFFEE3AFEED39FDD0E0FB8B
:1023C60050130BBB0003022199ED13FDEE13FEEF34
:0823D60013FFEC13FC0221715E
:1023DE00022199EC5D046005E85904700302218F17
:1023EE0012215A580460F6EC4860F2EC7004FDFEBF
:1023FE00FF22C860DB2481C85009C39860025006D2
:10240E000221969850CAF582E9294B4A7005AB8293
:10241E0002218575F0007C1A7880C3EF9BEE9AED51
:10242E0099400DC3EF9BFFEE9AFEED99FDE842F049
:10243E00DC23ACF0D0E0FFD0E0FED0E0FDAB82209C
:10244E00E7101BEB60BAEC2CFCEF33FFEE33FEED26
:10245E0033FD022171E803F830E705C0F075F00096
:10246E00EF2FFFEE33FEED33FD40B830E7C280AA0A
:10247E00ED33EC33600A047003BD8004ECB2E7FC6C
:01248E00222B
:10248F0075F020800E75F010800575F0087D007EC8
:10249F00007F003392D530D503122922EC33401040
:1024AF00EF33FFEE33FEED33FDEC33FCD5F0ED22D1
:0E24BF00E5F0247EA2D513CC92E7CDCEFF220D
:1024CD003F8000004120000042C80000447A000017
:1024DD00461C400047C35000497424004B18968099
:1024ED004CBEBC205A0E1BCA6753C21C749DC5AE90
:1024FD00FB60065407601C232312252BEB54386018
:10250D0009122517122526121FE7ECF8EDF9EEFA40
:10251D00EFCB22EB12252680F1543803241C902496
:10252D00CDFE93FC0EEE93FD0EEE930ECE93FF2299
:10253D00E709F608DFFA8046E709F208DFFA803E80
:10254D0088828C83E709F0A3DFFA8032E309F6086D
:10255D00DFFA8078E309F208DFFA807088828C83D5
:10256D00E309F0A3DFFA806489828A83E0A3F60889
:10257D00DFFA805889828A83E0A3F208DFFA804C63
:10258D0080D280FA80C680D4806980F2803380103A
:10259D0080A680EA809A80A880DA80E280CA8033A3
:1025AD0089828A83ECFAE493A3C8C582C8CCC5831B
:1025BD00CCF0A3C8C582C8CCC583CCDFE9DEE780EB
:1025CD000D89828A83E493A3F608DFF9ECFAA9F06A
:1025DD00EDFB2289828A83ECFAE0A3C8C582C8CCC0
:1025ED00C583CCF0A3C8C582C8CCC583CCDFEADED9
:1025FD00E880DB89828A83E493A3F208DFF980CC3B
:10260D0088F0EF60010E4E60C388F0ED2402B40433
:10261D000050B9F582EB2402B4040050AF232345DA
:06262D00822390258D734D
:10263300BB010689828A83E0225002E722BBFE02A5
:09264300E32289828A83E49322D8
:10264C00BB010CE58229F582E5833AF583E0225043
:10265C0006E92582F8E622BBFE06E92582F8E2228D
:0D266C00E58229F582E5833AF583E49322A7
:10267900BB010989828A83F8E028F022500327F7F1
:1026890022BBFE05F8E328F3228A838982F8E493C2
:022699002822F5
:10269B00BB010FF8E58229F582E5833AF583E02843
:1026AB00F0225009C58229F8E58226F622BBFE09E5
:1026BB00C58229F8E22582F222F8EA2583F583E91F
:0326CB009328222F
:1026CE00BB010689828A83F0225002F722BBFE01EB
:0226DE00F322E5
:1026E000F8BB010DE58229F582E5833AF583E8F030
:1026F000225006E92582C8F622BBFE05E92582C8DC
:02270000F222C3
:10270200EF8DF0A4A8F0CF8CF0A428CE8DF0A42EEB
:02271200FE22A5
:10271400BC000BBE0029EF8DF084FFADF022E4CCA9
:10272400F875F008EF2FFFEE33FEEC33FCEE9DEC72
:10273400984005FCEE9DFE0FD5F0E9E4CEFD22EDB8
:10274400F8F5F0EE8420D21CFEADF075F008EF2F02
:10275400FFED33FD4007985006D5F0F222C398FDF3
:052764000FD5F0EA2290
:10276900C2D5EC30E709B2D5E4C39DFDE49CFCEE8B
:1027790030E715B2D5E4C39FFFE49EFE122714C3C8
:10278900E49DFDE49CFC800312271430D507C3E4C3
:062799009FFFE49EFE22FA
:10279F00C5F0F8A3E028F0C5F0F8E58215827002C5
:0627AF001583E038F02262
:1027B500A3F8E0C5F025F0F0E582158270021583D7
:0627C500E0C838F0E82234
:1027CB00BB010A89828A83F0E5F0A3F0225006F759
:0F27DB0009A7F01922BBFE06F3E5F009F3192256
:0D27EA00EF2BFFEE3AFEED39FDEC38FC223E
:0E27F700C3EF9BFFEE9AFEED99FDEC98FC22DD
:10280500E88FF0A4CC8BF0A42CFCE98EF0A42CFC72
:102815008AF0EDA42CFCEA8EF0A4CDA8F08BF0A4F0
:102825002DCC3825F0FDE98FF0A42CCD35F0FCEB4F
:102835008EF0A4FEA9F0EB8FF0A4CFC5F02ECD3914
:0F284500FEE43CFCEAA42DCE35F0FDE43CFC2281
:1028540075F008758200EF2FFFEE33FECD33CDCC3B
:1028640033CCC58233C5829BED9AEC99E5829840BE
:102874000CF582EE9BFEED9AFDEC99FC0FD5F0D69B
:10288400E4CEFBE4CDFAE4CCF9A88222B800C1B9C5
:102894000059BA002DEC8BF084CFCECDFCE5F0CB03
:1028A400F97818EF2FFFEE33FEED33FDEC33FCEB3C
:1028B40033FB10D703994004EB99FB0FD8E5E4F9F7
:1028C400FA227818EF2FFFEE33FEED33FDEC33FCE4
:1028D400C933C910D7059BE99A4007EC9BFCE99AD8
:1028E400F90FD8E0E4C9FAE4CCFB2275F010EF2F1D
:1028F400FFEE33FEED33FDCC33CCC833C810D7071D
:102904009BEC9AE899400AED9BFDEC9AFCE899F857
:0E2914000FD5F0DAE4CDFBE4CCFAE4C8F922EA
:0E292200C3E49FFFE49EFEE49DFDE49CFC22C6
:10293000EB9FF5F0EA9E42F0E99D42F0E89C45F0FD
:012940002274
:10294100E8600FECC313FCED13FDEE13FEEF13FF74
:03295100D8F12298
:10295400E8600FEFC333FFEE33FEED33FDEC33FCE1
:03296400D8F12285
:10296700BB010789828A830229995005E9F8022F5A
:0A29770085BBFE05E9F8022F91224E
:0C298100E0FCA3E0FDA3E0FEA3E0FF22C9
:0C298D00E0F8A3E0F9A3E0FAA3E0FB22CD
:0C299900ECF0A3EDF0A3EEF0A3EFF022B1
:1029A500A8828583F0D083D0821229BC1229BC125B
:1029B50029BC1229BCE473E493A3C583C5F0C58380
:1029C500C8C582C8F0A3C583C5F0C583C8C582C87C
:0129D50022DF
:1029D600F5F0C582A4C582C5F0C583A42583F58319
:0129E60022CE
:0C29E700A42582F582E5F03583F58322FB
:0929F300E0FBA3E0FAA3E0F922E5
:1029FC00F8E0FBA3A3E0F925F0F0E5821582700264
:072A0C001583E0FA38F02207
:102A1300F8E0FBA3A3E025F0F9F0E582158270024C
:072A23001583E038FAF022F0
:092A2A00EBF0A3EAF0A3E9F022AD
:0C2A3300E493FB740193FA740293F922FF
:102A3F00BB010DE58229F582E5833AF5830229F37F
:102A4F005007E92582F8022F9DBBFE07E92582F882
:102A5F00022FAFE58229F582E5833AF583022A3307
:102A6F00BB0120E58229F582E5833AF583D0F0D0CA
:102A7F00E0F8D0E0F9D0E0FAD0E0FBE8C0E0C0F039
:102A8F00022A2A5018E92582F8D083D082D0E0F9A3
:102A9F00D0E0FAD0E0FBC082C083022FA6BBFE18A5
:102AAF00E92582F8D083D082D0E0F9D0E0FAD0E0E7
:092ABF00FBC082C083022FB82283
:102AC800D083D082F8E4937012740193700DA3A39D
:102AD80093F8740193F5828883E4737402936860B1
:062AE800EFA3A3A380DFB1
:102AEE00D083D082F8E4937012740193700DA3A377
:102AFE0093F8740193F5828883E473740293B5F0AE
:0D2B0E00067403936860E9A3A3A3A380D815
:062B1B008A838982E47345
:10FB180010780B12FD32BF0D027F0A02A486901ED8
:04FB280042E0FF2296
:08FDB400901E42EFF0D278220C
:10F87200EFC394414005EF945B400BEFC3946140AA
:0BF8820008EF947B5003D38001C322E9
:0FFC1600EFC394304007EF943A50028001C322AD
:10F4CA00EFC394414005EF945B4016EFC39461404B
:10F4DA0005EF947B400BEFC394304008EF943A5009
:06F4EA0003D38001C322E0
:0FFC2500EFC394204007EF947F50028001C32269
:0FFC3400EFC394414007EF945B50028001C3225D
:10FB2C00EFC394094005EF940E4004EFB42003D3C7
:04FB3C008001C3225F
:10F4F000EFC394414005EF94474016EFC394614039
:10F5000005EF9467400BEFC394304008EF943A50F6
:06F5100003D38001C322B9
:10D8F600901D04EBF0A3EAF0A3E9F0901D0AEBF00B
:10D90600A3EAF0A3E9F0901D04E0FBA3E475F0019F
:10D916001227B5A9F0FA12263370EB901D0574FF95
:10D92600F5F012279F901D07E0FBA3E475F00112A6
:10D9360027B5A9F0FA122633FF901D04E0FBA3E4F5
:10D9460075F0011227B5A9F0FAEF1226CE70D6901F
:0BD956001D0AE0FBA3E0FAA3E0F922A9
:10003A00901CBAEBF0A3EAF0A3E9F0E4901CC2F03A
:10004A00A3F0D3901CC1E09400901CC0E06480949B
:10005A008050030200F3901CBAE0FBA3E0FAA3E08D
:10006A00F9901CC2E0FEA3E0F5828E8312264C6052
:10007A0010901CC3E004F070DD901CC2E004F08014
:10008A00D5901CBDE0FBA3E0FAA3E0F91226336089
:10009A003E901CBDA3E475F0011227B5A9F0FA122F
:1000AA002633FF901CBAE0FBA3E0FAA3E0F9901C08
:1000BA00C2E475F0011227B585F082F583EF1226A6
:1000CA00E0901CC074FFF5F012279F45F070B290C3
:1000DA001CBAE0FBA3E0FAA3E0F9901CC2E0FEA37D
:1000EA00E0F5828E83E41226E0901CBAE0FBA3E0DE
:0500FA00FAA3E0F92269
:102B2100E3F5F009E208B5F06D606B80F3E3F5F0D1
:102B310009E608B5F060605E80F387F009E608B544
:102B4100F054605280F487F009E208B5F04860461D
:102B510080F488828C8387F009E0A3B5F038603671
:102B610080F488828C8387F009E493A3B5F0276011
:102B71002580F388828C83E3F5F009E0A3B5F01694
:102B8100601480F388828C83E3F5F009E493A3B5A4
:102B9100F004600280F2022C4C808580E7808E80F8
:102BA100D2803C8015806C807E809B80B5808B803C
:102BB100A1804F8070803A022C6289828A83ECFA6C
:102BC100E493F5F0A3C8C582C8CCC583CCE493A334
:102BD100C8C582C8CCC583CCB5F070606E80E18970
:102BE100828A83E493F5F0A3E208B5F05E605C802D
:102BF100F289828A83E0F5F0A3E608B5F04D604BD7
:102C010080F389828A83E0F5F0A3E208B5F03C60A5
:102C11003A80F389828A83E493F5F0A3E608B5F05C
:102C21002A602880F2805D89828A83ECFAE493F538
:102C3100F0A3C8C582C8CCC583CCE0A3C8C582C8EF
:102C4100CCC583CCB5F004600280E27F00F845F08A
:102C5100600EE863F0806480D395F01F40027F012D
:102C61002289828A83ECFAE0F5F0A3C8C582C8CC38
:102C7100C583CCE0A3C8C582C8CCC583CCB5F0CB95
:102C810060C980E389828A83ECFAE0F5F0A3C8C5C4
:102C910082C8CCC583CCE493A3C8C582C8CCC58304
:102CA100CCB5F0A760A580E288F0ED2402B4040061
:102CB1005099F582EB2402B40400508F23234582FE
:052CC10023902B9A7323
:10DB0300901D25EBF0A3EAF0A3E9F0901D28E0FBBC
:10DB1300A3E0FAA3E0F9122633FE901D25E0FBA350
:10DB2300E0FAA3E0F9122633FD6E702AED600E9041
:10DB33001D2B74FFF5F012279F45F070037F002221
:10DB4300901D26E475F00112279F901D29E475F0BE
:10DB53000112279F80B5D3EE6480F8ED648098406E
:07DB6300037F01227FFF2276
:102CC600E709F60870FA8046E709F20870FA803ECE
:102CD60088828C83E709F0A370FA807EE309F60800
:102CE60070FA8076E309F20870FA806E88828C8327
:102CF600E309F0A370FA806289828A83E0A3F6086A
:102D060070FA805689828A83E0A3F20870FA804AB4
:102D160080D280FA80C680D4806580F280318010AF
:102D260080A680EA809A80A880DA80E280CA803114
:102D360089828A83ECFAE493A3C8C582C8CCC5838A
:102D4600CCF0A3C8C582C8CCC583CC70E9800D89F8
:102D5600828A83E493A3F60870F9ECFAA9F0EDFBF6
:102D66002289828A83ECFAE0A3C8C582C8CCC583CF
:102D7600CCF0A3C8C582C8CCC583CC70EA80DD89F7
:102D8600828A83E493A3F20870F980CE88F0ED245A
:102D960002B4040050C4F582EB2402B4040050BA15
:092DA6002323458223902D1673AE
:10DA9B00901CC4EBF0A3EAF0A3E9F0E4901CCCF0EB
:10DAAB00A3F0901CCA74FFF5F01227B545F0603C4B
:10DABB00901CC7E0FBA3E0FAA3E0F9122633FF901A
:10DACB001CC4E0FBA3E0FAA3E0F9901CCCE475F0D6
:10DADB00011227B585F082F583EF1226E0EF60C2C5
:10DAEB00901CC8E475F00112279F80B6901CC4E00F
:08DAFB00FBA3E0FAA3E0F9220D
:10FADB00E4FFFE122633600C0FEF70010E09E97084
:05FAEB00F20A80EF2289
:10F82000E4FFFE800D6D60130FEF70010E09E970AB
:0CF83000010A12263370EE7EFF7FFF22DB
:102DAF00E3F5F009E208B5F06BDFF58067E3F5F0C6
:102DBF0009E608B5F05EDFF5805A87F009E608B539
:102DCF00F052DFF6804E87F009E208B5F046DFF6E5
:102DDF00804288828C8387F009E0A3B5F036DFF656
:102DEF00803288828C8387F009E493A3B5F025DFC6
:102DFF00F5802188828C83E3F5F009E0A3B5F01408
:102E0F00DFF5801088828C83E3F5F009E493A3B596
:102E1F00F002DFF4022EDE808780E9809080D4807C
:102E2F003E8015806E807E809D80B7808D80A380D0
:102E3F00518074803C022EEA89828A83ECFAE493F3
:102E4F00F5F0A3C8C582C8CCC583CCE493A3C8C58D
:102E5F0082C8CCC583CCB5F076DFE3DEE180708924
:102E6F00828A83E493F5F0A3E208B5F062DFF48081
:102E7F005E89828A83E0F5F0A3E608B5F051DFF5AD
:102E8F00804D89828A83E0F5F0A3E208B5F040DF38
:102E9F00F5803C89828A83E493F5F0A3E608B5F0C8
:102EAF002EDFF4802A8002805789828A83ECFAE42D
:102EBF0093F5F0A3C8C582C8CCC583CCE0A3C8C521
:102ECF0082C8CCC583CCB5F006DFE4DEE280007F9C
:102EDF00FFB5F0020F2240027F012289828A83EC24
:102EEF00FAE0F5F0A3C8C582C8CCC583CCE0A3C86F
:102EFF00C582C8CCC583CCB5F0D5DFE5DEE380CF86
:102F0F0089828A83ECFAE0F5F0A3C8C582C8CCC5E4
:102F1F0083CCE493A3C8C582C8CCC583CCB5F0AF2E
:102F2F00DFE4DEE280A988F0EF60010E4E60ABEDCA
:102F3F002402B404005098F582EB2402B40400502C
:0A2F4F008E2323458223902E267363
:102F5900EF4E6012EF60010EEDBB010B89828A838F
:102F6900F0A3DFFCDEFA2289F05007F709DFFCA99C
:0C2F7900F022BBFEFCF309DFFCA9F022F3
:0C2F8500ECF608EDF608EEF608EFF62278
:0C2F9100ECF208EDF208EEF208EFF2227C
:092F9D00E6FB08E6FA08E6F92259
:092FA600EBF608EAF608E9F62250
:092FAF00E2FB08E2FA08E2F92253
:092FB800EBF208EAF208E9F2224A
:0AFD32003098FDAF99C2987E0022C0
:00000001FF
